Archive member included to satisfy reference by file (symbol)

c:/program files (x86)/atollic/truestudio for stm32 9.2.0/armtools/bin/../lib/gcc/arm-atollic-eabi/6.3.1/../../../../arm-atollic-eabi/lib/armv7-m\libc_nano.a(lib_a-impure.o)
                              Src\main.o (_impure_ptr)
c:/program files (x86)/atollic/truestudio for stm32 9.2.0/armtools/bin/../lib/gcc/arm-atollic-eabi/6.3.1/../../../../arm-atollic-eabi/lib/armv7-m\libc_nano.a(lib_a-init.o)
                              startup\startup_stm32f207xx.o (__libc_init_array)
c:/program files (x86)/atollic/truestudio for stm32 9.2.0/armtools/bin/../lib/gcc/arm-atollic-eabi/6.3.1/../../../../arm-atollic-eabi/lib/armv7-m\libc_nano.a(lib_a-memset.o)
                              Src\atten_ctrl.o (memset)
c:/program files (x86)/atollic/truestudio for stm32 9.2.0/armtools/bin/../lib/gcc/arm-atollic-eabi/6.3.1/../../../../arm-atollic-eabi/lib/armv7-m\libc_nano.a(lib_a-printf.o)
                              Src\atten_ctrl.o (printf)
c:/program files (x86)/atollic/truestudio for stm32 9.2.0/armtools/bin/../lib/gcc/arm-atollic-eabi/6.3.1/../../../../arm-atollic-eabi/lib/armv7-m\libc_nano.a(lib_a-puts.o)
                              Src\atten_ctrl.o (puts)
c:/program files (x86)/atollic/truestudio for stm32 9.2.0/armtools/bin/../lib/gcc/arm-atollic-eabi/6.3.1/../../../../arm-atollic-eabi/lib/armv7-m\libc_nano.a(lib_a-setbuf.o)
                              Src\main.o (setbuf)
c:/program files (x86)/atollic/truestudio for stm32 9.2.0/armtools/bin/../lib/gcc/arm-atollic-eabi/6.3.1/../../../../arm-atollic-eabi/lib/armv7-m\libc_nano.a(lib_a-setvbuf.o)
                              c:/program files (x86)/atollic/truestudio for stm32 9.2.0/armtools/bin/../lib/gcc/arm-atollic-eabi/6.3.1/../../../../arm-atollic-eabi/lib/armv7-m\libc_nano.a(lib_a-setbuf.o) (setvbuf)
c:/program files (x86)/atollic/truestudio for stm32 9.2.0/armtools/bin/../lib/gcc/arm-atollic-eabi/6.3.1/../../../../arm-atollic-eabi/lib/armv7-m\libc_nano.a(lib_a-wbuf.o)
                              c:/program files (x86)/atollic/truestudio for stm32 9.2.0/armtools/bin/../lib/gcc/arm-atollic-eabi/6.3.1/../../../../arm-atollic-eabi/lib/armv7-m\libc_nano.a(lib_a-puts.o) (__swbuf_r)
c:/program files (x86)/atollic/truestudio for stm32 9.2.0/armtools/bin/../lib/gcc/arm-atollic-eabi/6.3.1/../../../../arm-atollic-eabi/lib/armv7-m\libc_nano.a(lib_a-wsetup.o)
                              c:/program files (x86)/atollic/truestudio for stm32 9.2.0/armtools/bin/../lib/gcc/arm-atollic-eabi/6.3.1/../../../../arm-atollic-eabi/lib/armv7-m\libc_nano.a(lib_a-puts.o) (__swsetup_r)
c:/program files (x86)/atollic/truestudio for stm32 9.2.0/armtools/bin/../lib/gcc/arm-atollic-eabi/6.3.1/../../../../arm-atollic-eabi/lib/armv7-m\libc_nano.a(lib_a-fflush.o)
                              c:/program files (x86)/atollic/truestudio for stm32 9.2.0/armtools/bin/../lib/gcc/arm-atollic-eabi/6.3.1/../../../../arm-atollic-eabi/lib/armv7-m\libc_nano.a(lib_a-setvbuf.o) (_fflush_r)
c:/program files (x86)/atollic/truestudio for stm32 9.2.0/armtools/bin/../lib/gcc/arm-atollic-eabi/6.3.1/../../../../arm-atollic-eabi/lib/armv7-m\libc_nano.a(lib_a-findfp.o)
                              c:/program files (x86)/atollic/truestudio for stm32 9.2.0/armtools/bin/../lib/gcc/arm-atollic-eabi/6.3.1/../../../../arm-atollic-eabi/lib/armv7-m\libc_nano.a(lib_a-printf.o) (__sinit)
c:/program files (x86)/atollic/truestudio for stm32 9.2.0/armtools/bin/../lib/gcc/arm-atollic-eabi/6.3.1/../../../../arm-atollic-eabi/lib/armv7-m\libc_nano.a(lib_a-fwalk.o)
                              c:/program files (x86)/atollic/truestudio for stm32 9.2.0/armtools/bin/../lib/gcc/arm-atollic-eabi/6.3.1/../../../../arm-atollic-eabi/lib/armv7-m\libc_nano.a(lib_a-findfp.o) (_fwalk)
c:/program files (x86)/atollic/truestudio for stm32 9.2.0/armtools/bin/../lib/gcc/arm-atollic-eabi/6.3.1/../../../../arm-atollic-eabi/lib/armv7-m\libc_nano.a(lib_a-makebuf.o)
                              c:/program files (x86)/atollic/truestudio for stm32 9.2.0/armtools/bin/../lib/gcc/arm-atollic-eabi/6.3.1/../../../../arm-atollic-eabi/lib/armv7-m\libc_nano.a(lib_a-setvbuf.o) (__swhatbuf_r)
c:/program files (x86)/atollic/truestudio for stm32 9.2.0/armtools/bin/../lib/gcc/arm-atollic-eabi/6.3.1/../../../../arm-atollic-eabi/lib/armv7-m\libc_nano.a(lib_a-malloc.o)
                              c:/program files (x86)/atollic/truestudio for stm32 9.2.0/armtools/bin/../lib/gcc/arm-atollic-eabi/6.3.1/../../../../arm-atollic-eabi/lib/armv7-m\libc_nano.a(lib_a-setvbuf.o) (malloc)
c:/program files (x86)/atollic/truestudio for stm32 9.2.0/armtools/bin/../lib/gcc/arm-atollic-eabi/6.3.1/../../../../arm-atollic-eabi/lib/armv7-m\libc_nano.a(lib_a-nano-freer.o)
                              c:/program files (x86)/atollic/truestudio for stm32 9.2.0/armtools/bin/../lib/gcc/arm-atollic-eabi/6.3.1/../../../../arm-atollic-eabi/lib/armv7-m\libc_nano.a(lib_a-setvbuf.o) (_free_r)
c:/program files (x86)/atollic/truestudio for stm32 9.2.0/armtools/bin/../lib/gcc/arm-atollic-eabi/6.3.1/../../../../arm-atollic-eabi/lib/armv7-m\libc_nano.a(lib_a-nano-mallocr.o)
                              c:/program files (x86)/atollic/truestudio for stm32 9.2.0/armtools/bin/../lib/gcc/arm-atollic-eabi/6.3.1/../../../../arm-atollic-eabi/lib/armv7-m\libc_nano.a(lib_a-findfp.o) (_malloc_r)
c:/program files (x86)/atollic/truestudio for stm32 9.2.0/armtools/bin/../lib/gcc/arm-atollic-eabi/6.3.1/../../../../arm-atollic-eabi/lib/armv7-m\libc_nano.a(lib_a-nano-vfprintf.o)
                              c:/program files (x86)/atollic/truestudio for stm32 9.2.0/armtools/bin/../lib/gcc/arm-atollic-eabi/6.3.1/../../../../arm-atollic-eabi/lib/armv7-m\libc_nano.a(lib_a-printf.o) (_vfprintf_r)
c:/program files (x86)/atollic/truestudio for stm32 9.2.0/armtools/bin/../lib/gcc/arm-atollic-eabi/6.3.1/../../../../arm-atollic-eabi/lib/armv7-m\libc_nano.a(lib_a-nano-vfprintf_i.o)
                              c:/program files (x86)/atollic/truestudio for stm32 9.2.0/armtools/bin/../lib/gcc/arm-atollic-eabi/6.3.1/../../../../arm-atollic-eabi/lib/armv7-m\libc_nano.a(lib_a-nano-vfprintf.o) (_printf_i)
c:/program files (x86)/atollic/truestudio for stm32 9.2.0/armtools/bin/../lib/gcc/arm-atollic-eabi/6.3.1/../../../../arm-atollic-eabi/lib/armv7-m\libc_nano.a(lib_a-sbrkr.o)
                              c:/program files (x86)/atollic/truestudio for stm32 9.2.0/armtools/bin/../lib/gcc/arm-atollic-eabi/6.3.1/../../../../arm-atollic-eabi/lib/armv7-m\libc_nano.a(lib_a-nano-mallocr.o) (_sbrk_r)
c:/program files (x86)/atollic/truestudio for stm32 9.2.0/armtools/bin/../lib/gcc/arm-atollic-eabi/6.3.1/../../../../arm-atollic-eabi/lib/armv7-m\libc_nano.a(lib_a-stdio.o)
                              c:/program files (x86)/atollic/truestudio for stm32 9.2.0/armtools/bin/../lib/gcc/arm-atollic-eabi/6.3.1/../../../../arm-atollic-eabi/lib/armv7-m\libc_nano.a(lib_a-findfp.o) (__sread)
c:/program files (x86)/atollic/truestudio for stm32 9.2.0/armtools/bin/../lib/gcc/arm-atollic-eabi/6.3.1/../../../../arm-atollic-eabi/lib/armv7-m\libc_nano.a(lib_a-writer.o)
                              c:/program files (x86)/atollic/truestudio for stm32 9.2.0/armtools/bin/../lib/gcc/arm-atollic-eabi/6.3.1/../../../../arm-atollic-eabi/lib/armv7-m\libc_nano.a(lib_a-stdio.o) (_write_r)
c:/program files (x86)/atollic/truestudio for stm32 9.2.0/armtools/bin/../lib/gcc/arm-atollic-eabi/6.3.1/../../../../arm-atollic-eabi/lib/armv7-m\libc_nano.a(lib_a-closer.o)
                              c:/program files (x86)/atollic/truestudio for stm32 9.2.0/armtools/bin/../lib/gcc/arm-atollic-eabi/6.3.1/../../../../arm-atollic-eabi/lib/armv7-m\libc_nano.a(lib_a-stdio.o) (_close_r)
c:/program files (x86)/atollic/truestudio for stm32 9.2.0/armtools/bin/../lib/gcc/arm-atollic-eabi/6.3.1/../../../../arm-atollic-eabi/lib/armv7-m\libc_nano.a(lib_a-fstatr.o)
                              c:/program files (x86)/atollic/truestudio for stm32 9.2.0/armtools/bin/../lib/gcc/arm-atollic-eabi/6.3.1/../../../../arm-atollic-eabi/lib/armv7-m\libc_nano.a(lib_a-makebuf.o) (_fstat_r)
c:/program files (x86)/atollic/truestudio for stm32 9.2.0/armtools/bin/../lib/gcc/arm-atollic-eabi/6.3.1/../../../../arm-atollic-eabi/lib/armv7-m\libc_nano.a(lib_a-fvwrite.o)
                              c:/program files (x86)/atollic/truestudio for stm32 9.2.0/armtools/bin/../lib/gcc/arm-atollic-eabi/6.3.1/../../../../arm-atollic-eabi/lib/armv7-m\libc_nano.a(lib_a-nano-vfprintf.o) (__sfvwrite_r)
c:/program files (x86)/atollic/truestudio for stm32 9.2.0/armtools/bin/../lib/gcc/arm-atollic-eabi/6.3.1/../../../../arm-atollic-eabi/lib/armv7-m\libc_nano.a(lib_a-isattyr.o)
                              c:/program files (x86)/atollic/truestudio for stm32 9.2.0/armtools/bin/../lib/gcc/arm-atollic-eabi/6.3.1/../../../../arm-atollic-eabi/lib/armv7-m\libc_nano.a(lib_a-makebuf.o) (_isatty_r)
c:/program files (x86)/atollic/truestudio for stm32 9.2.0/armtools/bin/../lib/gcc/arm-atollic-eabi/6.3.1/../../../../arm-atollic-eabi/lib/armv7-m\libc_nano.a(lib_a-lseekr.o)
                              c:/program files (x86)/atollic/truestudio for stm32 9.2.0/armtools/bin/../lib/gcc/arm-atollic-eabi/6.3.1/../../../../arm-atollic-eabi/lib/armv7-m\libc_nano.a(lib_a-stdio.o) (_lseek_r)
c:/program files (x86)/atollic/truestudio for stm32 9.2.0/armtools/bin/../lib/gcc/arm-atollic-eabi/6.3.1/../../../../arm-atollic-eabi/lib/armv7-m\libc_nano.a(lib_a-memchr-stub.o)
                              c:/program files (x86)/atollic/truestudio for stm32 9.2.0/armtools/bin/../lib/gcc/arm-atollic-eabi/6.3.1/../../../../arm-atollic-eabi/lib/armv7-m\libc_nano.a(lib_a-nano-vfprintf.o) (memchr)
c:/program files (x86)/atollic/truestudio for stm32 9.2.0/armtools/bin/../lib/gcc/arm-atollic-eabi/6.3.1/../../../../arm-atollic-eabi/lib/armv7-m\libc_nano.a(lib_a-memcpy-stub.o)
                              c:/program files (x86)/atollic/truestudio for stm32 9.2.0/armtools/bin/../lib/gcc/arm-atollic-eabi/6.3.1/../../../../arm-atollic-eabi/lib/armv7-m\libc_nano.a(lib_a-fvwrite.o) (memcpy)
c:/program files (x86)/atollic/truestudio for stm32 9.2.0/armtools/bin/../lib/gcc/arm-atollic-eabi/6.3.1/../../../../arm-atollic-eabi/lib/armv7-m\libc_nano.a(lib_a-memmove.o)
                              c:/program files (x86)/atollic/truestudio for stm32 9.2.0/armtools/bin/../lib/gcc/arm-atollic-eabi/6.3.1/../../../../arm-atollic-eabi/lib/armv7-m\libc_nano.a(lib_a-fvwrite.o) (memmove)
c:/program files (x86)/atollic/truestudio for stm32 9.2.0/armtools/bin/../lib/gcc/arm-atollic-eabi/6.3.1/../../../../arm-atollic-eabi/lib/armv7-m\libc_nano.a(lib_a-mlock.o)
                              c:/program files (x86)/atollic/truestudio for stm32 9.2.0/armtools/bin/../lib/gcc/arm-atollic-eabi/6.3.1/../../../../arm-atollic-eabi/lib/armv7-m\libc_nano.a(lib_a-nano-freer.o) (__malloc_lock)
c:/program files (x86)/atollic/truestudio for stm32 9.2.0/armtools/bin/../lib/gcc/arm-atollic-eabi/6.3.1/../../../../arm-atollic-eabi/lib/armv7-m\libc_nano.a(lib_a-nano-reallocr.o)
                              c:/program files (x86)/atollic/truestudio for stm32 9.2.0/armtools/bin/../lib/gcc/arm-atollic-eabi/6.3.1/../../../../arm-atollic-eabi/lib/armv7-m\libc_nano.a(lib_a-fvwrite.o) (_realloc_r)
c:/program files (x86)/atollic/truestudio for stm32 9.2.0/armtools/bin/../lib/gcc/arm-atollic-eabi/6.3.1/../../../../arm-atollic-eabi/lib/armv7-m\libc_nano.a(lib_a-readr.o)
                              c:/program files (x86)/atollic/truestudio for stm32 9.2.0/armtools/bin/../lib/gcc/arm-atollic-eabi/6.3.1/../../../../arm-atollic-eabi/lib/armv7-m\libc_nano.a(lib_a-stdio.o) (_read_r)
c:/program files (x86)/atollic/truestudio for stm32 9.2.0/armtools/bin/../lib/gcc/arm-atollic-eabi/6.3.1/../../../../arm-atollic-eabi/lib/armv7-m\libc_nano.a(lib_a-reent.o)
                              c:/program files (x86)/atollic/truestudio for stm32 9.2.0/armtools/bin/../lib/gcc/arm-atollic-eabi/6.3.1/../../../../arm-atollic-eabi/lib/armv7-m\libc_nano.a(lib_a-sbrkr.o) (errno)
c:/program files (x86)/atollic/truestudio for stm32 9.2.0/armtools/bin/../lib/gcc/arm-atollic-eabi/6.3.1/../../../../arm-atollic-eabi/lib/armv7-m\libc_nano.a(lib_a-nano-msizer.o)
                              c:/program files (x86)/atollic/truestudio for stm32 9.2.0/armtools/bin/../lib/gcc/arm-atollic-eabi/6.3.1/../../../../arm-atollic-eabi/lib/armv7-m\libc_nano.a(lib_a-nano-reallocr.o) (_malloc_usable_size_r)
c:/program files (x86)/atollic/truestudio for stm32 9.2.0/armtools/bin/../lib/gcc/arm-atollic-eabi/6.3.1/armv7-m\libgcc.a(_aeabi_uldivmod.o)
                              Drivers\STM32F2xx_HAL_Driver\Src\stm32f2xx_hal_rcc.o (__aeabi_uldivmod)
c:/program files (x86)/atollic/truestudio for stm32 9.2.0/armtools/bin/../lib/gcc/arm-atollic-eabi/6.3.1/armv7-m\libgcc.a(_udivmoddi4.o)
                              c:/program files (x86)/atollic/truestudio for stm32 9.2.0/armtools/bin/../lib/gcc/arm-atollic-eabi/6.3.1/armv7-m\libgcc.a(_aeabi_uldivmod.o) (__udivmoddi4)
c:/program files (x86)/atollic/truestudio for stm32 9.2.0/armtools/bin/../lib/gcc/arm-atollic-eabi/6.3.1/armv7-m\libgcc.a(_dvmd_tls.o)
                              c:/program files (x86)/atollic/truestudio for stm32 9.2.0/armtools/bin/../lib/gcc/arm-atollic-eabi/6.3.1/armv7-m\libgcc.a(_aeabi_uldivmod.o) (__aeabi_ldiv0)
c:/program files (x86)/atollic/truestudio for stm32 9.2.0/armtools/bin/../lib/gcc/arm-atollic-eabi/6.3.1/../../../../arm-atollic-eabi/lib/armv7-m\libnosys.a(close.o)
                              c:/program files (x86)/atollic/truestudio for stm32 9.2.0/armtools/bin/../lib/gcc/arm-atollic-eabi/6.3.1/../../../../arm-atollic-eabi/lib/armv7-m\libc_nano.a(lib_a-closer.o) (_close)
c:/program files (x86)/atollic/truestudio for stm32 9.2.0/armtools/bin/../lib/gcc/arm-atollic-eabi/6.3.1/../../../../arm-atollic-eabi/lib/armv7-m\libnosys.a(fstat.o)
                              c:/program files (x86)/atollic/truestudio for stm32 9.2.0/armtools/bin/../lib/gcc/arm-atollic-eabi/6.3.1/../../../../arm-atollic-eabi/lib/armv7-m\libc_nano.a(lib_a-fstatr.o) (_fstat)
c:/program files (x86)/atollic/truestudio for stm32 9.2.0/armtools/bin/../lib/gcc/arm-atollic-eabi/6.3.1/../../../../arm-atollic-eabi/lib/armv7-m\libnosys.a(isatty.o)
                              c:/program files (x86)/atollic/truestudio for stm32 9.2.0/armtools/bin/../lib/gcc/arm-atollic-eabi/6.3.1/../../../../arm-atollic-eabi/lib/armv7-m\libc_nano.a(lib_a-isattyr.o) (_isatty)
c:/program files (x86)/atollic/truestudio for stm32 9.2.0/armtools/bin/../lib/gcc/arm-atollic-eabi/6.3.1/../../../../arm-atollic-eabi/lib/armv7-m\libnosys.a(lseek.o)
                              c:/program files (x86)/atollic/truestudio for stm32 9.2.0/armtools/bin/../lib/gcc/arm-atollic-eabi/6.3.1/../../../../arm-atollic-eabi/lib/armv7-m\libc_nano.a(lib_a-lseekr.o) (_lseek)
c:/program files (x86)/atollic/truestudio for stm32 9.2.0/armtools/bin/../lib/gcc/arm-atollic-eabi/6.3.1/../../../../arm-atollic-eabi/lib/armv7-m\libnosys.a(read.o)
                              c:/program files (x86)/atollic/truestudio for stm32 9.2.0/armtools/bin/../lib/gcc/arm-atollic-eabi/6.3.1/../../../../arm-atollic-eabi/lib/armv7-m\libc_nano.a(lib_a-readr.o) (_read)
c:/program files (x86)/atollic/truestudio for stm32 9.2.0/armtools/bin/../lib/gcc/arm-atollic-eabi/6.3.1/../../../../arm-atollic-eabi/lib/armv7-m\libnosys.a(sbrk.o)
                              c:/program files (x86)/atollic/truestudio for stm32 9.2.0/armtools/bin/../lib/gcc/arm-atollic-eabi/6.3.1/../../../../arm-atollic-eabi/lib/armv7-m\libc_nano.a(lib_a-sbrkr.o) (_sbrk)

Allocating common symbols
Common symbol       size              file

ATT_B_EN_WIFI4_2_4Ghz_Table
                    0x40              Src\atten_ctrl.o
hi2c3               0x54              Src\main.o
ATT_A_EN_30G3_29_29_5Ghz_Table
                    0x40              Src\atten_ctrl.o
ATT_B_EN_30G1_28_28_5Ghz_Table
                    0x40              Src\atten_ctrl.o
ATT_A_EN_WIFI4_2_4Ghz_Table
                    0x40              Src\atten_ctrl.o
ATT_A_EN_30G3_29_5_30Ghz_Table
                    0x40              Src\atten_ctrl.o
errno               0x4               c:/program files (x86)/atollic/truestudio for stm32 9.2.0/armtools/bin/../lib/gcc/arm-atollic-eabi/6.3.1/../../../../arm-atollic-eabi/lib/armv7-m\libc_nano.a(lib_a-reent.o)
UartDataisReved     0x1               Src\main.o
ATT_B_EN_WIFI3_5_8Ghz_Table
                    0x40              Src\atten_ctrl.o
ATT_B_EN_30G3_28_5_29Ghz_Table
                    0x40              Src\atten_ctrl.o
ATT_A_EN_WIFI1_2_4Ghz_Table
                    0x40              Src\atten_ctrl.o
rx2_data            0x2               Src\main.o
ATT_B_EN_30G2_28_28_5Ghz_Table
                    0x40              Src\atten_ctrl.o
ATT_B_EN_WIFI4_5_8Ghz_Table
                    0x40              Src\atten_ctrl.o
ATT_A_EN_WIFI3_2_4Ghz_Table
                    0x40              Src\atten_ctrl.o
ATT_B_EN_WIFI2_2_4Ghz_Table
                    0x40              Src\atten_ctrl.o
ATT_B_EN_30G1_28_5_29Ghz_Table
                    0x40              Src\atten_ctrl.o
ATT_A_EN_30G2_28_5_29Ghz_Table
                    0x40              Src\atten_ctrl.o
ATT_B_EN_WIFI1_2_4Ghz_Table
                    0x40              Src\atten_ctrl.o
uwTick              0x4               Drivers\STM32F2xx_HAL_Driver\Src\stm32f2xx_hal.o
ATT_A_EN_30G2_29_29_5Ghz_Table
                    0x40              Src\atten_ctrl.o
ATT_B_EN_30G3_29_29_5Ghz_Table
                    0x40              Src\atten_ctrl.o
pFlash              0x20              Drivers\STM32F2xx_HAL_Driver\Src\stm32f2xx_hal_flash.o
count_out           0x1               Src\main.o
ATT_B_EN_30G2_28_5_29Ghz_Table
                    0x40              Src\atten_ctrl.o
ATT_A_EN_30G3_28_5_29Ghz_Table
                    0x40              Src\atten_ctrl.o
count_in            0x1               Src\main.o
ATT_B_EN_WIFI2_5_8Ghz_Table
                    0x40              Src\atten_ctrl.o
ATT_A_EN_30G1_28_28_5Ghz_Table
                    0x40              Src\atten_ctrl.o
ATT_B_EN_30G1_29_29_5Ghz_Table
                    0x40              Src\atten_ctrl.o
ATT_B_EN_30G2_29_29_5Ghz_Table
                    0x40              Src\atten_ctrl.o
ATT_A_EN_WIFI3_5_8Ghz_Table
                    0x40              Src\atten_ctrl.o
ATT_A_EN_30G3_28_28_5Ghz_Table
                    0x40              Src\atten_ctrl.o
ATT_A_EN_WIFI4_5_8Ghz_Table
                    0x40              Src\atten_ctrl.o
huart1              0x40              Src\main.o
Atten_Setting       0x31              Src\atten_ctrl.o
ATT_A_EN_150M_Table
                    0x40              Src\atten_ctrl.o
ATT_B_EN_WIFI3_2_4Ghz_Table
                    0x40              Src\atten_ctrl.o
ATT_A_EN_30G2_29_5_30Ghz_Table
                    0x40              Src\atten_ctrl.o
ring_buf            0x40              Src\main.o
ATT_A_EN_30G1_29_5_30Ghz_Table
                    0x40              Src\atten_ctrl.o
ATT_B_EN_30G3_29_5_30Ghz_Table
                    0x40              Src\atten_ctrl.o
ATT_A_EN_30G1_28_5_29Ghz_Table
                    0x40              Src\atten_ctrl.o
ATT_B_EN_30G1_29_5_30Ghz_Table
                    0x40              Src\atten_ctrl.o
ATT_B_EN_150M_Table
                    0x40              Src\atten_ctrl.o
htim6               0x40              Src\main.o
ATT_B_EN_30G3_28_28_5Ghz_Table
                    0x40              Src\atten_ctrl.o
Timer10ms           0x4               Src\main.o
ATT_A_EN_WIFI1_5_8Ghz_Table
                    0x40              Src\atten_ctrl.o
ATT_B_EN_WIFI1_5_8Ghz_Table
                    0x40              Src\atten_ctrl.o
ATT_B_EN_30G2_29_5_30Ghz_Table
                    0x40              Src\atten_ctrl.o
ATT_A_EN_30G2_28_28_5Ghz_Table
                    0x40              Src\atten_ctrl.o
ATT_A_EN_WIFI2_2_4Ghz_Table
                    0x40              Src\atten_ctrl.o
ATT_A_EN_30G1_29_29_5Ghz_Table
                    0x40              Src\atten_ctrl.o
ATT_A_EN_WIFI2_5_8Ghz_Table
                    0x40              Src\atten_ctrl.o

Discarded input sections

 .text          0x00000000        0x0 c:/program files (x86)/atollic/truestudio for stm32 9.2.0/armtools/bin/../lib/gcc/arm-atollic-eabi/6.3.1/armv7-m/crti.o
 .data          0x00000000        0x0 c:/program files (x86)/atollic/truestudio for stm32 9.2.0/armtools/bin/../lib/gcc/arm-atollic-eabi/6.3.1/armv7-m/crti.o
 .bss           0x00000000        0x0 c:/program files (x86)/atollic/truestudio for stm32 9.2.0/armtools/bin/../lib/gcc/arm-atollic-eabi/6.3.1/armv7-m/crti.o
 .data          0x00000000        0x4 c:/program files (x86)/atollic/truestudio for stm32 9.2.0/armtools/bin/../lib/gcc/arm-atollic-eabi/6.3.1/armv7-m/crtbegin.o
 .text          0x00000000        0x0 Drivers\STM32F2xx_HAL_Driver\Src\stm32f2xx_hal.o
 .data          0x00000000        0x0 Drivers\STM32F2xx_HAL_Driver\Src\stm32f2xx_hal.o
 .bss           0x00000000        0x0 Drivers\STM32F2xx_HAL_Driver\Src\stm32f2xx_hal.o
 .text.HAL_MspInit
                0x00000000        0x2 Drivers\STM32F2xx_HAL_Driver\Src\stm32f2xx_hal.o
 .text.HAL_MspDeInit
                0x00000000        0x2 Drivers\STM32F2xx_HAL_Driver\Src\stm32f2xx_hal.o
 .text.HAL_DeInit
                0x00000000       0x2c Drivers\STM32F2xx_HAL_Driver\Src\stm32f2xx_hal.o
 .text.HAL_SuspendTick
                0x00000000       0x10 Drivers\STM32F2xx_HAL_Driver\Src\stm32f2xx_hal.o
 .text.HAL_ResumeTick
                0x00000000       0x10 Drivers\STM32F2xx_HAL_Driver\Src\stm32f2xx_hal.o
 .text.HAL_GetHalVersion
                0x00000000        0x8 Drivers\STM32F2xx_HAL_Driver\Src\stm32f2xx_hal.o
 .text.HAL_GetREVID
                0x00000000        0xc Drivers\STM32F2xx_HAL_Driver\Src\stm32f2xx_hal.o
 .text.HAL_GetDEVID
                0x00000000       0x10 Drivers\STM32F2xx_HAL_Driver\Src\stm32f2xx_hal.o
 .text.HAL_DBGMCU_EnableDBGSleepMode
                0x00000000       0x10 Drivers\STM32F2xx_HAL_Driver\Src\stm32f2xx_hal.o
 .text.HAL_DBGMCU_DisableDBGSleepMode
                0x00000000       0x10 Drivers\STM32F2xx_HAL_Driver\Src\stm32f2xx_hal.o
 .text.HAL_DBGMCU_EnableDBGStopMode
                0x00000000       0x10 Drivers\STM32F2xx_HAL_Driver\Src\stm32f2xx_hal.o
 .text.HAL_DBGMCU_DisableDBGStopMode
                0x00000000       0x10 Drivers\STM32F2xx_HAL_Driver\Src\stm32f2xx_hal.o
 .text.HAL_DBGMCU_EnableDBGStandbyMode
                0x00000000       0x10 Drivers\STM32F2xx_HAL_Driver\Src\stm32f2xx_hal.o
 .text.HAL_DBGMCU_DisableDBGStandbyMode
                0x00000000       0x10 Drivers\STM32F2xx_HAL_Driver\Src\stm32f2xx_hal.o
 .text.HAL_EnableCompensationCell
                0x00000000       0x18 Drivers\STM32F2xx_HAL_Driver\Src\stm32f2xx_hal.o
 .text.HAL_DisableCompensationCell
                0x00000000       0x1c Drivers\STM32F2xx_HAL_Driver\Src\stm32f2xx_hal.o
 .text.HAL_GetUID
                0x00000000       0x20 Drivers\STM32F2xx_HAL_Driver\Src\stm32f2xx_hal.o
 .text          0x00000000        0x0 Drivers\STM32F2xx_HAL_Driver\Src\stm32f2xx_hal_cortex.o
 .data          0x00000000        0x0 Drivers\STM32F2xx_HAL_Driver\Src\stm32f2xx_hal_cortex.o
 .bss           0x00000000        0x0 Drivers\STM32F2xx_HAL_Driver\Src\stm32f2xx_hal_cortex.o
 .text.HAL_NVIC_DisableIRQ
                0x00000000       0x1c Drivers\STM32F2xx_HAL_Driver\Src\stm32f2xx_hal_cortex.o
 .text.HAL_NVIC_SystemReset
                0x00000000       0x24 Drivers\STM32F2xx_HAL_Driver\Src\stm32f2xx_hal_cortex.o
 .text.HAL_MPU_Disable
                0x00000000       0x20 Drivers\STM32F2xx_HAL_Driver\Src\stm32f2xx_hal_cortex.o
 .text.HAL_MPU_Enable
                0x00000000       0x24 Drivers\STM32F2xx_HAL_Driver\Src\stm32f2xx_hal_cortex.o
 .text.HAL_MPU_ConfigRegion
                0x00000000       0x50 Drivers\STM32F2xx_HAL_Driver\Src\stm32f2xx_hal_cortex.o
 .text.HAL_NVIC_GetPriorityGrouping
                0x00000000       0x10 Drivers\STM32F2xx_HAL_Driver\Src\stm32f2xx_hal_cortex.o
 .text.HAL_NVIC_GetPriority
                0x00000000       0x5c Drivers\STM32F2xx_HAL_Driver\Src\stm32f2xx_hal_cortex.o
 .text.HAL_NVIC_SetPendingIRQ
                0x00000000       0x1c Drivers\STM32F2xx_HAL_Driver\Src\stm32f2xx_hal_cortex.o
 .text.HAL_NVIC_GetPendingIRQ
                0x00000000       0x1c Drivers\STM32F2xx_HAL_Driver\Src\stm32f2xx_hal_cortex.o
 .text.HAL_NVIC_ClearPendingIRQ
                0x00000000       0x1c Drivers\STM32F2xx_HAL_Driver\Src\stm32f2xx_hal_cortex.o
 .text.HAL_NVIC_GetActive
                0x00000000       0x1c Drivers\STM32F2xx_HAL_Driver\Src\stm32f2xx_hal_cortex.o
 .text.HAL_SYSTICK_CLKSourceConfig
                0x00000000       0x18 Drivers\STM32F2xx_HAL_Driver\Src\stm32f2xx_hal_cortex.o
 .text.HAL_SYSTICK_Callback
                0x00000000        0x2 Drivers\STM32F2xx_HAL_Driver\Src\stm32f2xx_hal_cortex.o
 .text.HAL_SYSTICK_IRQHandler
                0x00000000        0x8 Drivers\STM32F2xx_HAL_Driver\Src\stm32f2xx_hal_cortex.o
 .text          0x00000000        0x0 Drivers\STM32F2xx_HAL_Driver\Src\stm32f2xx_hal_dma.o
 .data          0x00000000        0x0 Drivers\STM32F2xx_HAL_Driver\Src\stm32f2xx_hal_dma.o
 .bss           0x00000000        0x0 Drivers\STM32F2xx_HAL_Driver\Src\stm32f2xx_hal_dma.o
 .text.DMA_CalcBaseAndBitshift
                0x00000000       0x2c Drivers\STM32F2xx_HAL_Driver\Src\stm32f2xx_hal_dma.o
 .text.HAL_DMA_Init
                0x00000000       0xfc Drivers\STM32F2xx_HAL_Driver\Src\stm32f2xx_hal_dma.o
 .text.HAL_DMA_DeInit
                0x00000000       0x48 Drivers\STM32F2xx_HAL_Driver\Src\stm32f2xx_hal_dma.o
 .text.HAL_DMA_Start
                0x00000000       0x52 Drivers\STM32F2xx_HAL_Driver\Src\stm32f2xx_hal_dma.o
 .text.HAL_DMA_Start_IT
                0x00000000       0x7e Drivers\STM32F2xx_HAL_Driver\Src\stm32f2xx_hal_dma.o
 .text.HAL_DMA_Abort
                0x00000000       0x86 Drivers\STM32F2xx_HAL_Driver\Src\stm32f2xx_hal_dma.o
 .text.HAL_DMA_PollForTransfer
                0x00000000      0x112 Drivers\STM32F2xx_HAL_Driver\Src\stm32f2xx_hal_dma.o
 .text.HAL_DMA_IRQHandler
                0x00000000      0x174 Drivers\STM32F2xx_HAL_Driver\Src\stm32f2xx_hal_dma.o
 .text.HAL_DMA_RegisterCallback
                0x00000000       0x50 Drivers\STM32F2xx_HAL_Driver\Src\stm32f2xx_hal_dma.o
 .text.HAL_DMA_UnRegisterCallback
                0x00000000       0x5c Drivers\STM32F2xx_HAL_Driver\Src\stm32f2xx_hal_dma.o
 .text.HAL_DMA_GetState
                0x00000000        0x6 Drivers\STM32F2xx_HAL_Driver\Src\stm32f2xx_hal_dma.o
 .text.HAL_DMA_GetError
                0x00000000        0x4 Drivers\STM32F2xx_HAL_Driver\Src\stm32f2xx_hal_dma.o
 .rodata.flagBitshiftOffset.7572
                0x00000000        0x8 Drivers\STM32F2xx_HAL_Driver\Src\stm32f2xx_hal_dma.o
 .text          0x00000000        0x0 Drivers\STM32F2xx_HAL_Driver\Src\stm32f2xx_hal_dma_ex.o
 .data          0x00000000        0x0 Drivers\STM32F2xx_HAL_Driver\Src\stm32f2xx_hal_dma_ex.o
 .bss           0x00000000        0x0 Drivers\STM32F2xx_HAL_Driver\Src\stm32f2xx_hal_dma_ex.o
 .text.HAL_DMAEx_MultiBufferStart
                0x00000000       0x5a Drivers\STM32F2xx_HAL_Driver\Src\stm32f2xx_hal_dma_ex.o
 .text.HAL_DMAEx_MultiBufferStart_IT
                0x00000000      0x3e8 Drivers\STM32F2xx_HAL_Driver\Src\stm32f2xx_hal_dma_ex.o
 .text.HAL_DMAEx_ChangeMemory
                0x00000000        0xe Drivers\STM32F2xx_HAL_Driver\Src\stm32f2xx_hal_dma_ex.o
 .debug_info    0x00000000      0xdee Drivers\STM32F2xx_HAL_Driver\Src\stm32f2xx_hal_dma_ex.o
 .debug_abbrev  0x00000000      0x258 Drivers\STM32F2xx_HAL_Driver\Src\stm32f2xx_hal_dma_ex.o
 .debug_loc     0x00000000      0x452 Drivers\STM32F2xx_HAL_Driver\Src\stm32f2xx_hal_dma_ex.o
 .debug_aranges
                0x00000000       0x30 Drivers\STM32F2xx_HAL_Driver\Src\stm32f2xx_hal_dma_ex.o
 .debug_ranges  0x00000000       0x58 Drivers\STM32F2xx_HAL_Driver\Src\stm32f2xx_hal_dma_ex.o
 .debug_line    0x00000000      0x624 Drivers\STM32F2xx_HAL_Driver\Src\stm32f2xx_hal_dma_ex.o
 .debug_str     0x00000000      0x9b6 Drivers\STM32F2xx_HAL_Driver\Src\stm32f2xx_hal_dma_ex.o
 .comment       0x00000000       0x7d Drivers\STM32F2xx_HAL_Driver\Src\stm32f2xx_hal_dma_ex.o
 .debug_frame   0x00000000       0x58 Drivers\STM32F2xx_HAL_Driver\Src\stm32f2xx_hal_dma_ex.o
 .ARM.attributes
                0x00000000       0x33 Drivers\STM32F2xx_HAL_Driver\Src\stm32f2xx_hal_dma_ex.o
 .text          0x00000000        0x0 Drivers\STM32F2xx_HAL_Driver\Src\stm32f2xx_hal_flash.o
 .data          0x00000000        0x0 Drivers\STM32F2xx_HAL_Driver\Src\stm32f2xx_hal_flash.o
 .bss           0x00000000        0x0 Drivers\STM32F2xx_HAL_Driver\Src\stm32f2xx_hal_flash.o
 .text.FLASH_Program_DoubleWord
                0x00000000       0x28 Drivers\STM32F2xx_HAL_Driver\Src\stm32f2xx_hal_flash.o
 .text.FLASH_Program_Word
                0x00000000       0x24 Drivers\STM32F2xx_HAL_Driver\Src\stm32f2xx_hal_flash.o
 .text.FLASH_Program_HalfWord
                0x00000000       0x24 Drivers\STM32F2xx_HAL_Driver\Src\stm32f2xx_hal_flash.o
 .text.FLASH_SetErrorCode
                0x00000000       0x74 Drivers\STM32F2xx_HAL_Driver\Src\stm32f2xx_hal_flash.o
 .text.HAL_FLASH_Program_IT
                0x00000000       0x74 Drivers\STM32F2xx_HAL_Driver\Src\stm32f2xx_hal_flash.o
 .text.HAL_FLASH_EndOfOperationCallback
                0x00000000        0x2 Drivers\STM32F2xx_HAL_Driver\Src\stm32f2xx_hal_flash.o
 .text.HAL_FLASH_OperationErrorCallback
                0x00000000        0x2 Drivers\STM32F2xx_HAL_Driver\Src\stm32f2xx_hal_flash.o
 .text.HAL_FLASH_IRQHandler
                0x00000000       0xc4 Drivers\STM32F2xx_HAL_Driver\Src\stm32f2xx_hal_flash.o
 .text.HAL_FLASH_Unlock
                0x00000000       0x24 Drivers\STM32F2xx_HAL_Driver\Src\stm32f2xx_hal_flash.o
 .text.HAL_FLASH_Lock
                0x00000000       0x14 Drivers\STM32F2xx_HAL_Driver\Src\stm32f2xx_hal_flash.o
 .text.HAL_FLASH_OB_Unlock
                0x00000000       0x24 Drivers\STM32F2xx_HAL_Driver\Src\stm32f2xx_hal_flash.o
 .text.HAL_FLASH_OB_Lock
                0x00000000       0x14 Drivers\STM32F2xx_HAL_Driver\Src\stm32f2xx_hal_flash.o
 .text.HAL_FLASH_GetError
                0x00000000        0xc Drivers\STM32F2xx_HAL_Driver\Src\stm32f2xx_hal_flash.o
 .text.FLASH_WaitForLastOperation
                0x00000000       0x54 Drivers\STM32F2xx_HAL_Driver\Src\stm32f2xx_hal_flash.o
 .text.HAL_FLASH_Program
                0x00000000       0x90 Drivers\STM32F2xx_HAL_Driver\Src\stm32f2xx_hal_flash.o
 .text.HAL_FLASH_OB_Launch
                0x00000000       0x18 Drivers\STM32F2xx_HAL_Driver\Src\stm32f2xx_hal_flash.o
 .debug_info    0x00000000      0xf38 Drivers\STM32F2xx_HAL_Driver\Src\stm32f2xx_hal_flash.o
 .debug_abbrev  0x00000000      0x372 Drivers\STM32F2xx_HAL_Driver\Src\stm32f2xx_hal_flash.o
 .debug_loc     0x00000000      0x2c5 Drivers\STM32F2xx_HAL_Driver\Src\stm32f2xx_hal_flash.o
 .debug_aranges
                0x00000000       0x90 Drivers\STM32F2xx_HAL_Driver\Src\stm32f2xx_hal_flash.o
 .debug_ranges  0x00000000       0xb0 Drivers\STM32F2xx_HAL_Driver\Src\stm32f2xx_hal_flash.o
 .debug_line    0x00000000      0x4e9 Drivers\STM32F2xx_HAL_Driver\Src\stm32f2xx_hal_flash.o
 .debug_str     0x00000000      0x998 Drivers\STM32F2xx_HAL_Driver\Src\stm32f2xx_hal_flash.o
 .comment       0x00000000       0x7d Drivers\STM32F2xx_HAL_Driver\Src\stm32f2xx_hal_flash.o
 .debug_frame   0x00000000      0x154 Drivers\STM32F2xx_HAL_Driver\Src\stm32f2xx_hal_flash.o
 .ARM.attributes
                0x00000000       0x33 Drivers\STM32F2xx_HAL_Driver\Src\stm32f2xx_hal_flash.o
 COMMON         0x00000000       0x20 Drivers\STM32F2xx_HAL_Driver\Src\stm32f2xx_hal_flash.o
 .text          0x00000000        0x0 Drivers\STM32F2xx_HAL_Driver\Src\stm32f2xx_hal_flash_ex.o
 .data          0x00000000        0x0 Drivers\STM32F2xx_HAL_Driver\Src\stm32f2xx_hal_flash_ex.o
 .bss           0x00000000        0x0 Drivers\STM32F2xx_HAL_Driver\Src\stm32f2xx_hal_flash_ex.o
 .text.FLASH_MassErase.isra.0
                0x00000000       0x24 Drivers\STM32F2xx_HAL_Driver\Src\stm32f2xx_hal_flash_ex.o
 .text.HAL_FLASHEx_OBProgram
                0x00000000       0xb8 Drivers\STM32F2xx_HAL_Driver\Src\stm32f2xx_hal_flash_ex.o
 .text.HAL_FLASHEx_OBGetConfig
                0x00000000       0x48 Drivers\STM32F2xx_HAL_Driver\Src\stm32f2xx_hal_flash_ex.o
 .text.FLASH_Erase_Sector
                0x00000000       0x54 Drivers\STM32F2xx_HAL_Driver\Src\stm32f2xx_hal_flash_ex.o
 .text.HAL_FLASHEx_Erase_IT
                0x00000000       0x60 Drivers\STM32F2xx_HAL_Driver\Src\stm32f2xx_hal_flash_ex.o
 .text.FLASH_FlushCaches
                0x00000000       0x58 Drivers\STM32F2xx_HAL_Driver\Src\stm32f2xx_hal_flash_ex.o
 .text.HAL_FLASHEx_Erase
                0x00000000       0x9c Drivers\STM32F2xx_HAL_Driver\Src\stm32f2xx_hal_flash_ex.o
 .debug_info    0x00000000     0x10e7 Drivers\STM32F2xx_HAL_Driver\Src\stm32f2xx_hal_flash_ex.o
 .debug_abbrev  0x00000000      0x36c Drivers\STM32F2xx_HAL_Driver\Src\stm32f2xx_hal_flash_ex.o
 .debug_loc     0x00000000      0x3fa Drivers\STM32F2xx_HAL_Driver\Src\stm32f2xx_hal_flash_ex.o
 .debug_aranges
                0x00000000       0x50 Drivers\STM32F2xx_HAL_Driver\Src\stm32f2xx_hal_flash_ex.o
 .debug_ranges  0x00000000       0xd8 Drivers\STM32F2xx_HAL_Driver\Src\stm32f2xx_hal_flash_ex.o
 .debug_line    0x00000000      0x4aa Drivers\STM32F2xx_HAL_Driver\Src\stm32f2xx_hal_flash_ex.o
 .debug_str     0x00000000      0xa02 Drivers\STM32F2xx_HAL_Driver\Src\stm32f2xx_hal_flash_ex.o
 .comment       0x00000000       0x7d Drivers\STM32F2xx_HAL_Driver\Src\stm32f2xx_hal_flash_ex.o
 .debug_frame   0x00000000       0xa8 Drivers\STM32F2xx_HAL_Driver\Src\stm32f2xx_hal_flash_ex.o
 .ARM.attributes
                0x00000000       0x33 Drivers\STM32F2xx_HAL_Driver\Src\stm32f2xx_hal_flash_ex.o
 .text          0x00000000        0x0 Drivers\STM32F2xx_HAL_Driver\Src\stm32f2xx_hal_gpio.o
 .data          0x00000000        0x0 Drivers\STM32F2xx_HAL_Driver\Src\stm32f2xx_hal_gpio.o
 .bss           0x00000000        0x0 Drivers\STM32F2xx_HAL_Driver\Src\stm32f2xx_hal_gpio.o
 .text.HAL_GPIO_DeInit
                0x00000000      0x13c Drivers\STM32F2xx_HAL_Driver\Src\stm32f2xx_hal_gpio.o
 .text.HAL_GPIO_ReadPin
                0x00000000        0xc Drivers\STM32F2xx_HAL_Driver\Src\stm32f2xx_hal_gpio.o
 .text.HAL_GPIO_LockPin
                0x00000000       0x2a Drivers\STM32F2xx_HAL_Driver\Src\stm32f2xx_hal_gpio.o
 .text.HAL_GPIO_EXTI_Callback
                0x00000000        0x2 Drivers\STM32F2xx_HAL_Driver\Src\stm32f2xx_hal_gpio.o
 .text.HAL_GPIO_EXTI_IRQHandler
                0x00000000       0x18 Drivers\STM32F2xx_HAL_Driver\Src\stm32f2xx_hal_gpio.o
 .text          0x00000000        0x0 Drivers\STM32F2xx_HAL_Driver\Src\stm32f2xx_hal_i2c.o
 .data          0x00000000        0x0 Drivers\STM32F2xx_HAL_Driver\Src\stm32f2xx_hal_i2c.o
 .bss           0x00000000        0x0 Drivers\STM32F2xx_HAL_Driver\Src\stm32f2xx_hal_i2c.o
 .text.HAL_I2C_MspInit
                0x00000000        0x2 Drivers\STM32F2xx_HAL_Driver\Src\stm32f2xx_hal_i2c.o
 .text.HAL_I2C_MspDeInit
                0x00000000        0x2 Drivers\STM32F2xx_HAL_Driver\Src\stm32f2xx_hal_i2c.o
 .text.HAL_I2C_DeInit
                0x00000000       0x32 Drivers\STM32F2xx_HAL_Driver\Src\stm32f2xx_hal_i2c.o
 .text.HAL_I2C_Master_Transmit
                0x00000000      0x1ac Drivers\STM32F2xx_HAL_Driver\Src\stm32f2xx_hal_i2c.o
 .text.HAL_I2C_Master_Receive
                0x00000000      0x2ec Drivers\STM32F2xx_HAL_Driver\Src\stm32f2xx_hal_i2c.o
 .text.HAL_I2C_Slave_Transmit
                0x00000000      0x15c Drivers\STM32F2xx_HAL_Driver\Src\stm32f2xx_hal_i2c.o
 .text.HAL_I2C_Slave_Receive
                0x00000000      0x178 Drivers\STM32F2xx_HAL_Driver\Src\stm32f2xx_hal_i2c.o
 .text.HAL_I2C_Master_Transmit_IT
                0x00000000       0xa8 Drivers\STM32F2xx_HAL_Driver\Src\stm32f2xx_hal_i2c.o
 .text.HAL_I2C_Master_Receive_IT
                0x00000000       0xb0 Drivers\STM32F2xx_HAL_Driver\Src\stm32f2xx_hal_i2c.o
 .text.HAL_I2C_Master_Sequential_Transmit_IT
                0x00000000       0xc4 Drivers\STM32F2xx_HAL_Driver\Src\stm32f2xx_hal_i2c.o
 .text.HAL_I2C_Master_Sequential_Receive_IT
                0x00000000       0xdc Drivers\STM32F2xx_HAL_Driver\Src\stm32f2xx_hal_i2c.o
 .text.HAL_I2C_Slave_Transmit_IT
                0x00000000       0xb4 Drivers\STM32F2xx_HAL_Driver\Src\stm32f2xx_hal_i2c.o
 .text.HAL_I2C_Slave_Receive_IT
                0x00000000       0xb0 Drivers\STM32F2xx_HAL_Driver\Src\stm32f2xx_hal_i2c.o
 .text.HAL_I2C_Slave_Sequential_Transmit_IT
                0x00000000       0x78 Drivers\STM32F2xx_HAL_Driver\Src\stm32f2xx_hal_i2c.o
 .text.HAL_I2C_Slave_Sequential_Receive_IT
                0x00000000       0x78 Drivers\STM32F2xx_HAL_Driver\Src\stm32f2xx_hal_i2c.o
 .text.HAL_I2C_EnableListen_IT
                0x00000000       0x36 Drivers\STM32F2xx_HAL_Driver\Src\stm32f2xx_hal_i2c.o
 .text.HAL_I2C_DisableListen_IT
                0x00000000       0x3e Drivers\STM32F2xx_HAL_Driver\Src\stm32f2xx_hal_i2c.o
 .text.HAL_I2C_Master_Transmit_DMA
                0x00000000      0x104 Drivers\STM32F2xx_HAL_Driver\Src\stm32f2xx_hal_i2c.o
 .text.HAL_I2C_Master_Receive_DMA
                0x00000000      0x104 Drivers\STM32F2xx_HAL_Driver\Src\stm32f2xx_hal_i2c.o
 .text.HAL_I2C_Slave_Transmit_DMA
                0x00000000       0xe8 Drivers\STM32F2xx_HAL_Driver\Src\stm32f2xx_hal_i2c.o
 .text.HAL_I2C_Slave_Receive_DMA
                0x00000000       0xe8 Drivers\STM32F2xx_HAL_Driver\Src\stm32f2xx_hal_i2c.o
 .text.HAL_I2C_Mem_Write_IT
                0x00000000       0xb4 Drivers\STM32F2xx_HAL_Driver\Src\stm32f2xx_hal_i2c.o
 .text.HAL_I2C_Mem_Read_IT
                0x00000000       0xc0 Drivers\STM32F2xx_HAL_Driver\Src\stm32f2xx_hal_i2c.o
 .text.HAL_I2C_Mem_Write_DMA
                0x00000000      0x11c Drivers\STM32F2xx_HAL_Driver\Src\stm32f2xx_hal_i2c.o
 .text.HAL_I2C_Mem_Read_DMA
                0x00000000      0x180 Drivers\STM32F2xx_HAL_Driver\Src\stm32f2xx_hal_i2c.o
 .text.HAL_I2C_IsDeviceReady
                0x00000000      0x160 Drivers\STM32F2xx_HAL_Driver\Src\stm32f2xx_hal_i2c.o
 .text.HAL_I2C_MasterTxCpltCallback
                0x00000000        0x2 Drivers\STM32F2xx_HAL_Driver\Src\stm32f2xx_hal_i2c.o
 .text.HAL_I2C_MasterRxCpltCallback
                0x00000000        0x2 Drivers\STM32F2xx_HAL_Driver\Src\stm32f2xx_hal_i2c.o
 .text.HAL_I2C_SlaveTxCpltCallback
                0x00000000        0x2 Drivers\STM32F2xx_HAL_Driver\Src\stm32f2xx_hal_i2c.o
 .text.HAL_I2C_SlaveRxCpltCallback
                0x00000000        0x2 Drivers\STM32F2xx_HAL_Driver\Src\stm32f2xx_hal_i2c.o
 .text.HAL_I2C_AddrCallback
                0x00000000        0x2 Drivers\STM32F2xx_HAL_Driver\Src\stm32f2xx_hal_i2c.o
 .text.HAL_I2C_ListenCpltCallback
                0x00000000        0x2 Drivers\STM32F2xx_HAL_Driver\Src\stm32f2xx_hal_i2c.o
 .text.HAL_I2C_MemTxCpltCallback
                0x00000000        0x2 Drivers\STM32F2xx_HAL_Driver\Src\stm32f2xx_hal_i2c.o
 .text.HAL_I2C_MemRxCpltCallback
                0x00000000        0x2 Drivers\STM32F2xx_HAL_Driver\Src\stm32f2xx_hal_i2c.o
 .text.HAL_I2C_ErrorCallback
                0x00000000        0x2 Drivers\STM32F2xx_HAL_Driver\Src\stm32f2xx_hal_i2c.o
 .text.I2C_DMAError
                0x00000000       0x34 Drivers\STM32F2xx_HAL_Driver\Src\stm32f2xx_hal_i2c.o
 .text.I2C_DMAXferCplt
                0x00000000       0x80 Drivers\STM32F2xx_HAL_Driver\Src\stm32f2xx_hal_i2c.o
 .text.HAL_I2C_AbortCpltCallback
                0x00000000        0x2 Drivers\STM32F2xx_HAL_Driver\Src\stm32f2xx_hal_i2c.o
 .text.I2C_ITError
                0x00000000      0x128 Drivers\STM32F2xx_HAL_Driver\Src\stm32f2xx_hal_i2c.o
 .text.HAL_I2C_Master_Abort_IT
                0x00000000       0x4c Drivers\STM32F2xx_HAL_Driver\Src\stm32f2xx_hal_i2c.o
 .text.HAL_I2C_EV_IRQHandler
                0x00000000      0x6d4 Drivers\STM32F2xx_HAL_Driver\Src\stm32f2xx_hal_i2c.o
 .text.HAL_I2C_ER_IRQHandler
                0x00000000      0x134 Drivers\STM32F2xx_HAL_Driver\Src\stm32f2xx_hal_i2c.o
 .text.I2C_DMAAbort
                0x00000000       0x4c Drivers\STM32F2xx_HAL_Driver\Src\stm32f2xx_hal_i2c.o
 .text.HAL_I2C_GetState
                0x00000000        0x6 Drivers\STM32F2xx_HAL_Driver\Src\stm32f2xx_hal_i2c.o
 .text.HAL_I2C_GetMode
                0x00000000        0x6 Drivers\STM32F2xx_HAL_Driver\Src\stm32f2xx_hal_i2c.o
 .text.HAL_I2C_GetError
                0x00000000        0x4 Drivers\STM32F2xx_HAL_Driver\Src\stm32f2xx_hal_i2c.o
 .text          0x00000000        0x0 Drivers\STM32F2xx_HAL_Driver\Src\stm32f2xx_hal_pwr.o
 .data          0x00000000        0x0 Drivers\STM32F2xx_HAL_Driver\Src\stm32f2xx_hal_pwr.o
 .bss           0x00000000        0x0 Drivers\STM32F2xx_HAL_Driver\Src\stm32f2xx_hal_pwr.o
 .text.HAL_PWR_DeInit
                0x00000000       0x18 Drivers\STM32F2xx_HAL_Driver\Src\stm32f2xx_hal_pwr.o
 .text.HAL_PWR_EnableBkUpAccess
                0x00000000       0x1c Drivers\STM32F2xx_HAL_Driver\Src\stm32f2xx_hal_pwr.o
 .text.HAL_PWR_DisableBkUpAccess
                0x00000000       0x1c Drivers\STM32F2xx_HAL_Driver\Src\stm32f2xx_hal_pwr.o
 .text.HAL_PWR_ConfigPVD
                0x00000000       0x70 Drivers\STM32F2xx_HAL_Driver\Src\stm32f2xx_hal_pwr.o
 .text.HAL_PWR_EnablePVD
                0x00000000       0x1a Drivers\STM32F2xx_HAL_Driver\Src\stm32f2xx_hal_pwr.o
 .text.HAL_PWR_DisablePVD
                0x00000000       0x1a Drivers\STM32F2xx_HAL_Driver\Src\stm32f2xx_hal_pwr.o
 .text.HAL_PWR_EnableWakeUpPin
                0x00000000       0x10 Drivers\STM32F2xx_HAL_Driver\Src\stm32f2xx_hal_pwr.o
 .text.HAL_PWR_DisableWakeUpPin
                0x00000000       0x10 Drivers\STM32F2xx_HAL_Driver\Src\stm32f2xx_hal_pwr.o
 .text.HAL_PWR_EnterSLEEPMode
                0x00000000       0x20 Drivers\STM32F2xx_HAL_Driver\Src\stm32f2xx_hal_pwr.o
 .text.HAL_PWR_EnterSTOPMode
                0x00000000       0x38 Drivers\STM32F2xx_HAL_Driver\Src\stm32f2xx_hal_pwr.o
 .text.HAL_PWR_EnterSTANDBYMode
                0x00000000       0x20 Drivers\STM32F2xx_HAL_Driver\Src\stm32f2xx_hal_pwr.o
 .text.HAL_PWR_PVDCallback
                0x00000000        0x2 Drivers\STM32F2xx_HAL_Driver\Src\stm32f2xx_hal_pwr.o
 .text.HAL_PWR_PVD_IRQHandler
                0x00000000       0x1c Drivers\STM32F2xx_HAL_Driver\Src\stm32f2xx_hal_pwr.o
 .text.HAL_PWR_EnableSleepOnExit
                0x00000000       0x10 Drivers\STM32F2xx_HAL_Driver\Src\stm32f2xx_hal_pwr.o
 .text.HAL_PWR_DisableSleepOnExit
                0x00000000       0x10 Drivers\STM32F2xx_HAL_Driver\Src\stm32f2xx_hal_pwr.o
 .text.HAL_PWR_EnableSEVOnPend
                0x00000000       0x10 Drivers\STM32F2xx_HAL_Driver\Src\stm32f2xx_hal_pwr.o
 .text.HAL_PWR_DisableSEVOnPend
                0x00000000       0x10 Drivers\STM32F2xx_HAL_Driver\Src\stm32f2xx_hal_pwr.o
 .debug_info    0x00000000     0x10c9 Drivers\STM32F2xx_HAL_Driver\Src\stm32f2xx_hal_pwr.o
 .debug_abbrev  0x00000000      0x29d Drivers\STM32F2xx_HAL_Driver\Src\stm32f2xx_hal_pwr.o
 .debug_loc     0x00000000       0xd8 Drivers\STM32F2xx_HAL_Driver\Src\stm32f2xx_hal_pwr.o
 .debug_aranges
                0x00000000       0xa0 Drivers\STM32F2xx_HAL_Driver\Src\stm32f2xx_hal_pwr.o
 .debug_ranges  0x00000000       0x90 Drivers\STM32F2xx_HAL_Driver\Src\stm32f2xx_hal_pwr.o
 .debug_line    0x00000000      0x433 Drivers\STM32F2xx_HAL_Driver\Src\stm32f2xx_hal_pwr.o
 .debug_str     0x00000000      0x9b8 Drivers\STM32F2xx_HAL_Driver\Src\stm32f2xx_hal_pwr.o
 .comment       0x00000000       0x7d Drivers\STM32F2xx_HAL_Driver\Src\stm32f2xx_hal_pwr.o
 .debug_frame   0x00000000      0x128 Drivers\STM32F2xx_HAL_Driver\Src\stm32f2xx_hal_pwr.o
 .ARM.attributes
                0x00000000       0x33 Drivers\STM32F2xx_HAL_Driver\Src\stm32f2xx_hal_pwr.o
 .text          0x00000000        0x0 Drivers\STM32F2xx_HAL_Driver\Src\stm32f2xx_hal_pwr_ex.o
 .data          0x00000000        0x0 Drivers\STM32F2xx_HAL_Driver\Src\stm32f2xx_hal_pwr_ex.o
 .bss           0x00000000        0x0 Drivers\STM32F2xx_HAL_Driver\Src\stm32f2xx_hal_pwr_ex.o
 .text.HAL_PWREx_EnableBkUpReg
                0x00000000       0x44 Drivers\STM32F2xx_HAL_Driver\Src\stm32f2xx_hal_pwr_ex.o
 .text.HAL_PWREx_DisableBkUpReg
                0x00000000       0x44 Drivers\STM32F2xx_HAL_Driver\Src\stm32f2xx_hal_pwr_ex.o
 .text.HAL_PWREx_EnableFlashPowerDown
                0x00000000       0x1c Drivers\STM32F2xx_HAL_Driver\Src\stm32f2xx_hal_pwr_ex.o
 .text.HAL_PWREx_DisableFlashPowerDown
                0x00000000       0x1c Drivers\STM32F2xx_HAL_Driver\Src\stm32f2xx_hal_pwr_ex.o
 .debug_info    0x00000000      0xb44 Drivers\STM32F2xx_HAL_Driver\Src\stm32f2xx_hal_pwr_ex.o
 .debug_abbrev  0x00000000      0x255 Drivers\STM32F2xx_HAL_Driver\Src\stm32f2xx_hal_pwr_ex.o
 .debug_loc     0x00000000       0x96 Drivers\STM32F2xx_HAL_Driver\Src\stm32f2xx_hal_pwr_ex.o
 .debug_aranges
                0x00000000       0x38 Drivers\STM32F2xx_HAL_Driver\Src\stm32f2xx_hal_pwr_ex.o
 .debug_ranges  0x00000000       0x28 Drivers\STM32F2xx_HAL_Driver\Src\stm32f2xx_hal_pwr_ex.o
 .debug_line    0x00000000      0x341 Drivers\STM32F2xx_HAL_Driver\Src\stm32f2xx_hal_pwr_ex.o
 .debug_str     0x00000000      0x727 Drivers\STM32F2xx_HAL_Driver\Src\stm32f2xx_hal_pwr_ex.o
 .comment       0x00000000       0x7d Drivers\STM32F2xx_HAL_Driver\Src\stm32f2xx_hal_pwr_ex.o
 .debug_frame   0x00000000       0x68 Drivers\STM32F2xx_HAL_Driver\Src\stm32f2xx_hal_pwr_ex.o
 .ARM.attributes
                0x00000000       0x33 Drivers\STM32F2xx_HAL_Driver\Src\stm32f2xx_hal_pwr_ex.o
 .text          0x00000000        0x0 Drivers\STM32F2xx_HAL_Driver\Src\stm32f2xx_hal_rcc.o
 .data          0x00000000        0x0 Drivers\STM32F2xx_HAL_Driver\Src\stm32f2xx_hal_rcc.o
 .bss           0x00000000        0x0 Drivers\STM32F2xx_HAL_Driver\Src\stm32f2xx_hal_rcc.o
 .text.HAL_RCC_DeInit
                0x00000000       0xf4 Drivers\STM32F2xx_HAL_Driver\Src\stm32f2xx_hal_rcc.o
 .text.HAL_RCC_MCOConfig
                0x00000000       0x98 Drivers\STM32F2xx_HAL_Driver\Src\stm32f2xx_hal_rcc.o
 .text.HAL_RCC_EnableCSS
                0x00000000        0xc Drivers\STM32F2xx_HAL_Driver\Src\stm32f2xx_hal_rcc.o
 .text.HAL_RCC_DisableCSS
                0x00000000        0xc Drivers\STM32F2xx_HAL_Driver\Src\stm32f2xx_hal_rcc.o
 .text.HAL_RCC_GetHCLKFreq
                0x00000000        0xc Drivers\STM32F2xx_HAL_Driver\Src\stm32f2xx_hal_rcc.o
 .text.HAL_RCC_GetOscConfig
                0x00000000       0xcc Drivers\STM32F2xx_HAL_Driver\Src\stm32f2xx_hal_rcc.o
 .text.HAL_RCC_GetClockConfig
                0x00000000       0x3c Drivers\STM32F2xx_HAL_Driver\Src\stm32f2xx_hal_rcc.o
 .text.HAL_RCC_CSSCallback
                0x00000000        0x2 Drivers\STM32F2xx_HAL_Driver\Src\stm32f2xx_hal_rcc.o
 .text.HAL_RCC_NMI_IRQHandler
                0x00000000       0x20 Drivers\STM32F2xx_HAL_Driver\Src\stm32f2xx_hal_rcc.o
 .text          0x00000000        0x0 Drivers\STM32F2xx_HAL_Driver\Src\stm32f2xx_hal_rcc_ex.o
 .data          0x00000000        0x0 Drivers\STM32F2xx_HAL_Driver\Src\stm32f2xx_hal_rcc_ex.o
 .bss           0x00000000        0x0 Drivers\STM32F2xx_HAL_Driver\Src\stm32f2xx_hal_rcc_ex.o
 .text.HAL_RCCEx_PeriphCLKConfig
                0x00000000      0x14c Drivers\STM32F2xx_HAL_Driver\Src\stm32f2xx_hal_rcc_ex.o
 .text.HAL_RCCEx_GetPeriphCLKConfig
                0x00000000       0x4c Drivers\STM32F2xx_HAL_Driver\Src\stm32f2xx_hal_rcc_ex.o
 .debug_info    0x00000000      0xd9c Drivers\STM32F2xx_HAL_Driver\Src\stm32f2xx_hal_rcc_ex.o
 .debug_abbrev  0x00000000      0x2a3 Drivers\STM32F2xx_HAL_Driver\Src\stm32f2xx_hal_rcc_ex.o
 .debug_loc     0x00000000      0x17e Drivers\STM32F2xx_HAL_Driver\Src\stm32f2xx_hal_rcc_ex.o
 .debug_aranges
                0x00000000       0x28 Drivers\STM32F2xx_HAL_Driver\Src\stm32f2xx_hal_rcc_ex.o
 .debug_ranges  0x00000000       0x48 Drivers\STM32F2xx_HAL_Driver\Src\stm32f2xx_hal_rcc_ex.o
 .debug_line    0x00000000      0x390 Drivers\STM32F2xx_HAL_Driver\Src\stm32f2xx_hal_rcc_ex.o
 .debug_str     0x00000000      0x88d Drivers\STM32F2xx_HAL_Driver\Src\stm32f2xx_hal_rcc_ex.o
 .comment       0x00000000       0x7d Drivers\STM32F2xx_HAL_Driver\Src\stm32f2xx_hal_rcc_ex.o
 .debug_frame   0x00000000       0x4c Drivers\STM32F2xx_HAL_Driver\Src\stm32f2xx_hal_rcc_ex.o
 .ARM.attributes
                0x00000000       0x33 Drivers\STM32F2xx_HAL_Driver\Src\stm32f2xx_hal_rcc_ex.o
 .text          0x00000000        0x0 Drivers\STM32F2xx_HAL_Driver\Src\stm32f2xx_hal_tim.o
 .data          0x00000000        0x0 Drivers\STM32F2xx_HAL_Driver\Src\stm32f2xx_hal_tim.o
 .bss           0x00000000        0x0 Drivers\STM32F2xx_HAL_Driver\Src\stm32f2xx_hal_tim.o
 .text.TIM_OC1_SetConfig
                0x00000000       0x58 Drivers\STM32F2xx_HAL_Driver\Src\stm32f2xx_hal_tim.o
 .text.TIM_OC3_SetConfig
                0x00000000       0x60 Drivers\STM32F2xx_HAL_Driver\Src\stm32f2xx_hal_tim.o
 .text.TIM_OC4_SetConfig
                0x00000000       0x50 Drivers\STM32F2xx_HAL_Driver\Src\stm32f2xx_hal_tim.o
 .text.TIM_SlaveTimer_SetConfig
                0x00000000       0xaa Drivers\STM32F2xx_HAL_Driver\Src\stm32f2xx_hal_tim.o
 .text.HAL_TIM_Base_MspInit
                0x00000000        0x2 Drivers\STM32F2xx_HAL_Driver\Src\stm32f2xx_hal_tim.o
 .text.HAL_TIM_Base_MspDeInit
                0x00000000        0x2 Drivers\STM32F2xx_HAL_Driver\Src\stm32f2xx_hal_tim.o
 .text.HAL_TIM_Base_DeInit
                0x00000000       0x3a Drivers\STM32F2xx_HAL_Driver\Src\stm32f2xx_hal_tim.o
 .text.HAL_TIM_Base_Start
                0x00000000       0x1a Drivers\STM32F2xx_HAL_Driver\Src\stm32f2xx_hal_tim.o
 .text.HAL_TIM_Base_Stop
                0x00000000       0x2e Drivers\STM32F2xx_HAL_Driver\Src\stm32f2xx_hal_tim.o
 .text.HAL_TIM_Base_Stop_IT
                0x00000000       0x2a Drivers\STM32F2xx_HAL_Driver\Src\stm32f2xx_hal_tim.o
 .text.HAL_TIM_Base_Start_DMA
                0x00000000       0x54 Drivers\STM32F2xx_HAL_Driver\Src\stm32f2xx_hal_tim.o
 .text.HAL_TIM_Base_Stop_DMA
                0x00000000       0x30 Drivers\STM32F2xx_HAL_Driver\Src\stm32f2xx_hal_tim.o
 .text.HAL_TIM_OC_MspInit
                0x00000000        0x2 Drivers\STM32F2xx_HAL_Driver\Src\stm32f2xx_hal_tim.o
 .text.HAL_TIM_OC_MspDeInit
                0x00000000        0x2 Drivers\STM32F2xx_HAL_Driver\Src\stm32f2xx_hal_tim.o
 .text.HAL_TIM_OC_DeInit
                0x00000000       0x3a Drivers\STM32F2xx_HAL_Driver\Src\stm32f2xx_hal_tim.o
 .text.HAL_TIM_PWM_MspInit
                0x00000000        0x2 Drivers\STM32F2xx_HAL_Driver\Src\stm32f2xx_hal_tim.o
 .text.HAL_TIM_PWM_MspDeInit
                0x00000000        0x2 Drivers\STM32F2xx_HAL_Driver\Src\stm32f2xx_hal_tim.o
 .text.HAL_TIM_PWM_DeInit
                0x00000000       0x3a Drivers\STM32F2xx_HAL_Driver\Src\stm32f2xx_hal_tim.o
 .text.HAL_TIM_IC_MspInit
                0x00000000        0x2 Drivers\STM32F2xx_HAL_Driver\Src\stm32f2xx_hal_tim.o
 .text.HAL_TIM_IC_MspDeInit
                0x00000000        0x2 Drivers\STM32F2xx_HAL_Driver\Src\stm32f2xx_hal_tim.o
 .text.HAL_TIM_IC_DeInit
                0x00000000       0x3a Drivers\STM32F2xx_HAL_Driver\Src\stm32f2xx_hal_tim.o
 .text.HAL_TIM_OnePulse_MspInit
                0x00000000        0x2 Drivers\STM32F2xx_HAL_Driver\Src\stm32f2xx_hal_tim.o
 .text.HAL_TIM_OnePulse_MspDeInit
                0x00000000        0x2 Drivers\STM32F2xx_HAL_Driver\Src\stm32f2xx_hal_tim.o
 .text.HAL_TIM_OnePulse_DeInit
                0x00000000       0x3a Drivers\STM32F2xx_HAL_Driver\Src\stm32f2xx_hal_tim.o
 .text.HAL_TIM_OnePulse_Start
                0x00000000       0x40 Drivers\STM32F2xx_HAL_Driver\Src\stm32f2xx_hal_tim.o
 .text.HAL_TIM_OnePulse_Stop
                0x00000000       0x68 Drivers\STM32F2xx_HAL_Driver\Src\stm32f2xx_hal_tim.o
 .text.HAL_TIM_OnePulse_Start_IT
                0x00000000       0x50 Drivers\STM32F2xx_HAL_Driver\Src\stm32f2xx_hal_tim.o
 .text.HAL_TIM_OnePulse_Stop_IT
                0x00000000       0x78 Drivers\STM32F2xx_HAL_Driver\Src\stm32f2xx_hal_tim.o
 .text.HAL_TIM_Encoder_MspInit
                0x00000000        0x2 Drivers\STM32F2xx_HAL_Driver\Src\stm32f2xx_hal_tim.o
 .text.HAL_TIM_Encoder_MspDeInit
                0x00000000        0x2 Drivers\STM32F2xx_HAL_Driver\Src\stm32f2xx_hal_tim.o
 .text.HAL_TIM_Encoder_DeInit
                0x00000000       0x3a Drivers\STM32F2xx_HAL_Driver\Src\stm32f2xx_hal_tim.o
 .text.HAL_TIM_Encoder_Start
                0x00000000       0x44 Drivers\STM32F2xx_HAL_Driver\Src\stm32f2xx_hal_tim.o
 .text.HAL_TIM_Encoder_Stop
                0x00000000       0x48 Drivers\STM32F2xx_HAL_Driver\Src\stm32f2xx_hal_tim.o
 .text.HAL_TIM_Encoder_Start_IT
                0x00000000       0x6e Drivers\STM32F2xx_HAL_Driver\Src\stm32f2xx_hal_tim.o
 .text.HAL_TIM_Encoder_Stop_IT
                0x00000000       0x74 Drivers\STM32F2xx_HAL_Driver\Src\stm32f2xx_hal_tim.o
 .text.HAL_TIM_Encoder_Start_DMA
                0x00000000      0x124 Drivers\STM32F2xx_HAL_Driver\Src\stm32f2xx_hal_tim.o
 .text.HAL_TIM_Encoder_Stop_DMA
                0x00000000       0x74 Drivers\STM32F2xx_HAL_Driver\Src\stm32f2xx_hal_tim.o
 .text.HAL_TIM_DMABurst_WriteStart
                0x00000000       0xb4 Drivers\STM32F2xx_HAL_Driver\Src\stm32f2xx_hal_tim.o
 .text.HAL_TIM_DMABurst_ReadStart
                0x00000000       0xb4 Drivers\STM32F2xx_HAL_Driver\Src\stm32f2xx_hal_tim.o
 .text.HAL_TIM_DMABurst_ReadStop
                0x00000000       0x5e Drivers\STM32F2xx_HAL_Driver\Src\stm32f2xx_hal_tim.o
 .text.HAL_TIM_DMABurst_WriteStop
                0x00000000        0x4 Drivers\STM32F2xx_HAL_Driver\Src\stm32f2xx_hal_tim.o
 .text.HAL_TIM_GenerateEvent
                0x00000000       0x24 Drivers\STM32F2xx_HAL_Driver\Src\stm32f2xx_hal_tim.o
 .text.HAL_TIM_ConfigOCrefClear
                0x00000000       0xb6 Drivers\STM32F2xx_HAL_Driver\Src\stm32f2xx_hal_tim.o
 .text.HAL_TIM_ConfigClockSource
                0x00000000      0x172 Drivers\STM32F2xx_HAL_Driver\Src\stm32f2xx_hal_tim.o
 .text.HAL_TIM_ConfigTI1Input
                0x00000000       0x10 Drivers\STM32F2xx_HAL_Driver\Src\stm32f2xx_hal_tim.o
 .text.HAL_TIM_SlaveConfigSynchronization
                0x00000000       0x40 Drivers\STM32F2xx_HAL_Driver\Src\stm32f2xx_hal_tim.o
 .text.HAL_TIM_SlaveConfigSynchronization_IT
                0x00000000       0x40 Drivers\STM32F2xx_HAL_Driver\Src\stm32f2xx_hal_tim.o
 .text.HAL_TIM_ReadCapturedValue
                0x00000000       0x46 Drivers\STM32F2xx_HAL_Driver\Src\stm32f2xx_hal_tim.o
 .text.HAL_TIM_PeriodElapsedCallback
                0x00000000        0x2 Drivers\STM32F2xx_HAL_Driver\Src\stm32f2xx_hal_tim.o
 .text.TIM_DMAPeriodElapsedCplt
                0x00000000       0x10 Drivers\STM32F2xx_HAL_Driver\Src\stm32f2xx_hal_tim.o
 .text.TIM_DMACaptureCplt
                0x00000000       0x3c Drivers\STM32F2xx_HAL_Driver\Src\stm32f2xx_hal_tim.o
 .text.TIM_DMADelayPulseCplt
                0x00000000       0x3c Drivers\STM32F2xx_HAL_Driver\Src\stm32f2xx_hal_tim.o
 .text.TIM_DMATriggerCplt
                0x00000000       0x10 Drivers\STM32F2xx_HAL_Driver\Src\stm32f2xx_hal_tim.o
 .text.HAL_TIM_ErrorCallback
                0x00000000        0x2 Drivers\STM32F2xx_HAL_Driver\Src\stm32f2xx_hal_tim.o
 .text.TIM_DMAError
                0x00000000       0x10 Drivers\STM32F2xx_HAL_Driver\Src\stm32f2xx_hal_tim.o
 .text.HAL_TIM_Base_GetState
                0x00000000        0x6 Drivers\STM32F2xx_HAL_Driver\Src\stm32f2xx_hal_tim.o
 .text.HAL_TIM_OC_GetState
                0x00000000        0x6 Drivers\STM32F2xx_HAL_Driver\Src\stm32f2xx_hal_tim.o
 .text.HAL_TIM_PWM_GetState
                0x00000000        0x6 Drivers\STM32F2xx_HAL_Driver\Src\stm32f2xx_hal_tim.o
 .text.HAL_TIM_IC_GetState
                0x00000000        0x6 Drivers\STM32F2xx_HAL_Driver\Src\stm32f2xx_hal_tim.o
 .text.HAL_TIM_OnePulse_GetState
                0x00000000        0x6 Drivers\STM32F2xx_HAL_Driver\Src\stm32f2xx_hal_tim.o
 .text.HAL_TIM_Encoder_GetState
                0x00000000        0x6 Drivers\STM32F2xx_HAL_Driver\Src\stm32f2xx_hal_tim.o
 .text.HAL_TIM_OC_Init
                0x00000000       0x34 Drivers\STM32F2xx_HAL_Driver\Src\stm32f2xx_hal_tim.o
 .text.HAL_TIM_PWM_Init
                0x00000000       0x34 Drivers\STM32F2xx_HAL_Driver\Src\stm32f2xx_hal_tim.o
 .text.HAL_TIM_IC_Init
                0x00000000       0x34 Drivers\STM32F2xx_HAL_Driver\Src\stm32f2xx_hal_tim.o
 .text.HAL_TIM_OnePulse_Init
                0x00000000       0x46 Drivers\STM32F2xx_HAL_Driver\Src\stm32f2xx_hal_tim.o
 .text.HAL_TIM_Encoder_Init
                0x00000000       0x92 Drivers\STM32F2xx_HAL_Driver\Src\stm32f2xx_hal_tim.o
 .text.TIM_TI1_SetConfig
                0x00000000       0x74 Drivers\STM32F2xx_HAL_Driver\Src\stm32f2xx_hal_tim.o
 .text.HAL_TIM_IC_ConfigChannel
                0x00000000      0x110 Drivers\STM32F2xx_HAL_Driver\Src\stm32f2xx_hal_tim.o
 .text.TIM_OC2_SetConfig
                0x00000000       0x60 Drivers\STM32F2xx_HAL_Driver\Src\stm32f2xx_hal_tim.o
 .text.HAL_TIM_OC_ConfigChannel
                0x00000000       0x5c Drivers\STM32F2xx_HAL_Driver\Src\stm32f2xx_hal_tim.o
 .text.HAL_TIM_PWM_ConfigChannel
                0x00000000       0xc4 Drivers\STM32F2xx_HAL_Driver\Src\stm32f2xx_hal_tim.o
 .text.HAL_TIM_OnePulse_ConfigChannel
                0x00000000       0xf4 Drivers\STM32F2xx_HAL_Driver\Src\stm32f2xx_hal_tim.o
 .text.TIM_CCxChannelCmd
                0x00000000       0x18 Drivers\STM32F2xx_HAL_Driver\Src\stm32f2xx_hal_tim.o
 .text.HAL_TIM_OC_Stop
                0x00000000       0x5c Drivers\STM32F2xx_HAL_Driver\Src\stm32f2xx_hal_tim.o
 .text.HAL_TIM_PWM_Start
                0x00000000       0x34 Drivers\STM32F2xx_HAL_Driver\Src\stm32f2xx_hal_tim.o
 .text.HAL_TIM_OC_Start
                0x00000000        0x4 Drivers\STM32F2xx_HAL_Driver\Src\stm32f2xx_hal_tim.o
 .text.HAL_TIM_PWM_Stop
                0x00000000       0x64 Drivers\STM32F2xx_HAL_Driver\Src\stm32f2xx_hal_tim.o
 .text.HAL_TIM_PWM_Start_IT
                0x00000000       0x74 Drivers\STM32F2xx_HAL_Driver\Src\stm32f2xx_hal_tim.o
 .text.HAL_TIM_OC_Start_IT
                0x00000000        0x4 Drivers\STM32F2xx_HAL_Driver\Src\stm32f2xx_hal_tim.o
 .text.HAL_TIM_PWM_Stop_IT
                0x00000000       0x9c Drivers\STM32F2xx_HAL_Driver\Src\stm32f2xx_hal_tim.o
 .text.HAL_TIM_OC_Stop_IT
                0x00000000        0x4 Drivers\STM32F2xx_HAL_Driver\Src\stm32f2xx_hal_tim.o
 .text.HAL_TIM_PWM_Start_DMA
                0x00000000       0xec Drivers\STM32F2xx_HAL_Driver\Src\stm32f2xx_hal_tim.o
 .text.HAL_TIM_OC_Start_DMA
                0x00000000        0x4 Drivers\STM32F2xx_HAL_Driver\Src\stm32f2xx_hal_tim.o
 .text.HAL_TIM_PWM_Stop_DMA
                0x00000000       0xa0 Drivers\STM32F2xx_HAL_Driver\Src\stm32f2xx_hal_tim.o
 .text.HAL_TIM_OC_Stop_DMA
                0x00000000        0x4 Drivers\STM32F2xx_HAL_Driver\Src\stm32f2xx_hal_tim.o
 .text.HAL_TIM_IC_Start
                0x00000000       0x1a Drivers\STM32F2xx_HAL_Driver\Src\stm32f2xx_hal_tim.o
 .text.HAL_TIM_IC_Stop
                0x00000000       0x2e Drivers\STM32F2xx_HAL_Driver\Src\stm32f2xx_hal_tim.o
 .text.HAL_TIM_IC_Start_IT
                0x00000000       0x58 Drivers\STM32F2xx_HAL_Driver\Src\stm32f2xx_hal_tim.o
 .text.HAL_TIM_IC_Stop_IT
                0x00000000       0x6c Drivers\STM32F2xx_HAL_Driver\Src\stm32f2xx_hal_tim.o
 .text.HAL_TIM_IC_Start_DMA
                0x00000000       0xcc Drivers\STM32F2xx_HAL_Driver\Src\stm32f2xx_hal_tim.o
 .text.HAL_TIM_IC_Stop_DMA
                0x00000000       0x72 Drivers\STM32F2xx_HAL_Driver\Src\stm32f2xx_hal_tim.o
 .text          0x00000000        0x0 Drivers\STM32F2xx_HAL_Driver\Src\stm32f2xx_hal_tim_ex.o
 .data          0x00000000        0x0 Drivers\STM32F2xx_HAL_Driver\Src\stm32f2xx_hal_tim_ex.o
 .bss           0x00000000        0x0 Drivers\STM32F2xx_HAL_Driver\Src\stm32f2xx_hal_tim_ex.o
 .text.TIM_CCxNChannelCmd
                0x00000000       0x18 Drivers\STM32F2xx_HAL_Driver\Src\stm32f2xx_hal_tim_ex.o
 .text.HAL_TIMEx_HallSensor_MspInit
                0x00000000        0x2 Drivers\STM32F2xx_HAL_Driver\Src\stm32f2xx_hal_tim_ex.o
 .text.HAL_TIMEx_HallSensor_Init
                0x00000000       0xa0 Drivers\STM32F2xx_HAL_Driver\Src\stm32f2xx_hal_tim_ex.o
 .text.HAL_TIMEx_HallSensor_MspDeInit
                0x00000000        0x2 Drivers\STM32F2xx_HAL_Driver\Src\stm32f2xx_hal_tim_ex.o
 .text.HAL_TIMEx_HallSensor_DeInit
                0x00000000       0x3a Drivers\STM32F2xx_HAL_Driver\Src\stm32f2xx_hal_tim_ex.o
 .text.HAL_TIMEx_HallSensor_Start
                0x00000000       0x1c Drivers\STM32F2xx_HAL_Driver\Src\stm32f2xx_hal_tim_ex.o
 .text.HAL_TIMEx_HallSensor_Stop
                0x00000000       0x30 Drivers\STM32F2xx_HAL_Driver\Src\stm32f2xx_hal_tim_ex.o
 .text.HAL_TIMEx_HallSensor_Start_IT
                0x00000000       0x24 Drivers\STM32F2xx_HAL_Driver\Src\stm32f2xx_hal_tim_ex.o
 .text.HAL_TIMEx_HallSensor_Stop_IT
                0x00000000       0x38 Drivers\STM32F2xx_HAL_Driver\Src\stm32f2xx_hal_tim_ex.o
 .text.HAL_TIMEx_HallSensor_Start_DMA
                0x00000000       0x64 Drivers\STM32F2xx_HAL_Driver\Src\stm32f2xx_hal_tim_ex.o
 .text.HAL_TIMEx_HallSensor_Stop_DMA
                0x00000000       0x38 Drivers\STM32F2xx_HAL_Driver\Src\stm32f2xx_hal_tim_ex.o
 .text.HAL_TIMEx_PWMN_Start
                0x00000000       0x22 Drivers\STM32F2xx_HAL_Driver\Src\stm32f2xx_hal_tim_ex.o
 .text.HAL_TIMEx_OCN_Start
                0x00000000        0x4 Drivers\STM32F2xx_HAL_Driver\Src\stm32f2xx_hal_tim_ex.o
 .text.HAL_TIMEx_PWMN_Start_IT
                0x00000000       0x60 Drivers\STM32F2xx_HAL_Driver\Src\stm32f2xx_hal_tim_ex.o
 .text.HAL_TIMEx_OCN_Start_IT
                0x00000000        0x4 Drivers\STM32F2xx_HAL_Driver\Src\stm32f2xx_hal_tim_ex.o
 .text.HAL_TIMEx_PWMN_Stop_IT
                0x00000000       0x9a Drivers\STM32F2xx_HAL_Driver\Src\stm32f2xx_hal_tim_ex.o
 .text.HAL_TIMEx_OCN_Stop_IT
                0x00000000        0x4 Drivers\STM32F2xx_HAL_Driver\Src\stm32f2xx_hal_tim_ex.o
 .text.HAL_TIMEx_PWMN_Start_DMA
                0x00000000       0xd4 Drivers\STM32F2xx_HAL_Driver\Src\stm32f2xx_hal_tim_ex.o
 .text.HAL_TIMEx_OCN_Start_DMA
                0x00000000        0x4 Drivers\STM32F2xx_HAL_Driver\Src\stm32f2xx_hal_tim_ex.o
 .text.HAL_TIMEx_PWMN_Stop_DMA
                0x00000000       0x8e Drivers\STM32F2xx_HAL_Driver\Src\stm32f2xx_hal_tim_ex.o
 .text.HAL_TIMEx_OCN_Stop_DMA
                0x00000000        0x4 Drivers\STM32F2xx_HAL_Driver\Src\stm32f2xx_hal_tim_ex.o
 .text.HAL_TIMEx_OnePulseN_Start
                0x00000000       0x1a Drivers\STM32F2xx_HAL_Driver\Src\stm32f2xx_hal_tim_ex.o
 .text.HAL_TIMEx_OnePulseN_Stop
                0x00000000       0x4a Drivers\STM32F2xx_HAL_Driver\Src\stm32f2xx_hal_tim_ex.o
 .text.HAL_TIMEx_PWMN_Stop
                0x00000000        0x4 Drivers\STM32F2xx_HAL_Driver\Src\stm32f2xx_hal_tim_ex.o
 .text.HAL_TIMEx_OCN_Stop
                0x00000000        0x4 Drivers\STM32F2xx_HAL_Driver\Src\stm32f2xx_hal_tim_ex.o
 .text.HAL_TIMEx_OnePulseN_Start_IT
                0x00000000       0x2a Drivers\STM32F2xx_HAL_Driver\Src\stm32f2xx_hal_tim_ex.o
 .text.HAL_TIMEx_OnePulseN_Stop_IT
                0x00000000       0x5a Drivers\STM32F2xx_HAL_Driver\Src\stm32f2xx_hal_tim_ex.o
 .text.HAL_TIMEx_ConfigCommutationEvent
                0x00000000       0x4a Drivers\STM32F2xx_HAL_Driver\Src\stm32f2xx_hal_tim_ex.o
 .text.HAL_TIMEx_ConfigCommutationEvent_IT
                0x00000000       0x52 Drivers\STM32F2xx_HAL_Driver\Src\stm32f2xx_hal_tim_ex.o
 .text.HAL_TIMEx_ConfigCommutationEvent_DMA
                0x00000000       0x64 Drivers\STM32F2xx_HAL_Driver\Src\stm32f2xx_hal_tim_ex.o
 .text.HAL_TIMEx_ConfigBreakDeadTime
                0x00000000       0x4c Drivers\STM32F2xx_HAL_Driver\Src\stm32f2xx_hal_tim_ex.o
 .text.HAL_TIMEx_RemapConfig
                0x00000000       0x20 Drivers\STM32F2xx_HAL_Driver\Src\stm32f2xx_hal_tim_ex.o
 .text.TIMEx_DMACommutationCplt
                0x00000000       0x10 Drivers\STM32F2xx_HAL_Driver\Src\stm32f2xx_hal_tim_ex.o
 .text.HAL_TIMEx_HallSensor_GetState
                0x00000000        0x6 Drivers\STM32F2xx_HAL_Driver\Src\stm32f2xx_hal_tim_ex.o
 .text          0x00000000        0x0 Drivers\STM32F2xx_HAL_Driver\Src\stm32f2xx_hal_uart.o
 .data          0x00000000        0x0 Drivers\STM32F2xx_HAL_Driver\Src\stm32f2xx_hal_uart.o
 .bss           0x00000000        0x0 Drivers\STM32F2xx_HAL_Driver\Src\stm32f2xx_hal_uart.o
 .text.HAL_UART_MspInit
                0x00000000        0x2 Drivers\STM32F2xx_HAL_Driver\Src\stm32f2xx_hal_uart.o
 .text.HAL_HalfDuplex_Init
                0x00000000       0x64 Drivers\STM32F2xx_HAL_Driver\Src\stm32f2xx_hal_uart.o
 .text.HAL_LIN_Init
                0x00000000       0x76 Drivers\STM32F2xx_HAL_Driver\Src\stm32f2xx_hal_uart.o
 .text.HAL_MultiProcessor_Init
                0x00000000       0x7e Drivers\STM32F2xx_HAL_Driver\Src\stm32f2xx_hal_uart.o
 .text.HAL_UART_MspDeInit
                0x00000000        0x2 Drivers\STM32F2xx_HAL_Driver\Src\stm32f2xx_hal_uart.o
 .text.HAL_UART_DeInit
                0x00000000       0x26 Drivers\STM32F2xx_HAL_Driver\Src\stm32f2xx_hal_uart.o
 .text.HAL_UART_Receive
                0x00000000       0xbe Drivers\STM32F2xx_HAL_Driver\Src\stm32f2xx_hal_uart.o
 .text.HAL_UART_Transmit_IT
                0x00000000       0x3e Drivers\STM32F2xx_HAL_Driver\Src\stm32f2xx_hal_uart.o
 .text.HAL_UART_Transmit_DMA
                0x00000000       0x74 Drivers\STM32F2xx_HAL_Driver\Src\stm32f2xx_hal_uart.o
 .text.HAL_UART_Receive_DMA
                0x00000000       0x90 Drivers\STM32F2xx_HAL_Driver\Src\stm32f2xx_hal_uart.o
 .text.HAL_UART_DMAPause
                0x00000000       0x5a Drivers\STM32F2xx_HAL_Driver\Src\stm32f2xx_hal_uart.o
 .text.HAL_UART_DMAResume
                0x00000000       0x62 Drivers\STM32F2xx_HAL_Driver\Src\stm32f2xx_hal_uart.o
 .text.HAL_UART_DMAStop
                0x00000000       0x5e Drivers\STM32F2xx_HAL_Driver\Src\stm32f2xx_hal_uart.o
 .text.HAL_UART_Abort
                0x00000000       0x60 Drivers\STM32F2xx_HAL_Driver\Src\stm32f2xx_hal_uart.o
 .text.HAL_UART_AbortTransmit
                0x00000000       0x34 Drivers\STM32F2xx_HAL_Driver\Src\stm32f2xx_hal_uart.o
 .text.HAL_UART_AbortReceive
                0x00000000       0x3c Drivers\STM32F2xx_HAL_Driver\Src\stm32f2xx_hal_uart.o
 .text.UART_DMATransmitCplt
                0x00000000       0x2c Drivers\STM32F2xx_HAL_Driver\Src\stm32f2xx_hal_uart.o
 .text.HAL_UART_TxHalfCpltCallback
                0x00000000        0x2 Drivers\STM32F2xx_HAL_Driver\Src\stm32f2xx_hal_uart.o
 .text.UART_DMATxHalfCplt
                0x00000000        0xa Drivers\STM32F2xx_HAL_Driver\Src\stm32f2xx_hal_uart.o
 .text.HAL_UART_RxCpltCallback
                0x00000000        0x2 Drivers\STM32F2xx_HAL_Driver\Src\stm32f2xx_hal_uart.o
 .text.UART_DMAReceiveCplt
                0x00000000       0x38 Drivers\STM32F2xx_HAL_Driver\Src\stm32f2xx_hal_uart.o
 .text.HAL_UART_RxHalfCpltCallback
                0x00000000        0x2 Drivers\STM32F2xx_HAL_Driver\Src\stm32f2xx_hal_uart.o
 .text.UART_DMARxHalfCplt
                0x00000000        0xa Drivers\STM32F2xx_HAL_Driver\Src\stm32f2xx_hal_uart.o
 .text.UART_DMAError
                0x00000000       0x4e Drivers\STM32F2xx_HAL_Driver\Src\stm32f2xx_hal_uart.o
 .text.HAL_UART_AbortCpltCallback
                0x00000000        0x2 Drivers\STM32F2xx_HAL_Driver\Src\stm32f2xx_hal_uart.o
 .text.HAL_UART_Abort_IT
                0x00000000       0xa8 Drivers\STM32F2xx_HAL_Driver\Src\stm32f2xx_hal_uart.o
 .text.UART_DMARxAbortCallback
                0x00000000       0x28 Drivers\STM32F2xx_HAL_Driver\Src\stm32f2xx_hal_uart.o
 .text.UART_DMATxAbortCallback
                0x00000000       0x28 Drivers\STM32F2xx_HAL_Driver\Src\stm32f2xx_hal_uart.o
 .text.HAL_UART_AbortTransmitCpltCallback
                0x00000000        0x2 Drivers\STM32F2xx_HAL_Driver\Src\stm32f2xx_hal_uart.o
 .text.HAL_UART_AbortTransmit_IT
                0x00000000       0x50 Drivers\STM32F2xx_HAL_Driver\Src\stm32f2xx_hal_uart.o
 .text.UART_DMATxOnlyAbortCallback
                0x00000000       0x14 Drivers\STM32F2xx_HAL_Driver\Src\stm32f2xx_hal_uart.o
 .text.HAL_UART_AbortReceiveCpltCallback
                0x00000000        0x2 Drivers\STM32F2xx_HAL_Driver\Src\stm32f2xx_hal_uart.o
 .text.HAL_UART_AbortReceive_IT
                0x00000000       0x58 Drivers\STM32F2xx_HAL_Driver\Src\stm32f2xx_hal_uart.o
 .text.UART_DMARxOnlyAbortCallback
                0x00000000       0x14 Drivers\STM32F2xx_HAL_Driver\Src\stm32f2xx_hal_uart.o
 .text.HAL_LIN_SendBreak
                0x00000000       0x2c Drivers\STM32F2xx_HAL_Driver\Src\stm32f2xx_hal_uart.o
 .text.HAL_MultiProcessor_EnterMuteMode
                0x00000000       0x2c Drivers\STM32F2xx_HAL_Driver\Src\stm32f2xx_hal_uart.o
 .text.HAL_MultiProcessor_ExitMuteMode
                0x00000000       0x2c Drivers\STM32F2xx_HAL_Driver\Src\stm32f2xx_hal_uart.o
 .text.HAL_HalfDuplex_EnableTransmitter
                0x00000000       0x30 Drivers\STM32F2xx_HAL_Driver\Src\stm32f2xx_hal_uart.o
 .text.HAL_HalfDuplex_EnableReceiver
                0x00000000       0x30 Drivers\STM32F2xx_HAL_Driver\Src\stm32f2xx_hal_uart.o
 .text.HAL_UART_GetState
                0x00000000        0xc Drivers\STM32F2xx_HAL_Driver\Src\stm32f2xx_hal_uart.o
 .text.HAL_UART_GetError
                0x00000000        0x4 Drivers\STM32F2xx_HAL_Driver\Src\stm32f2xx_hal_uart.o
 .text          0x00000000        0x0 Src\atten_ctrl.o
 .data          0x00000000        0x0 Src\atten_ctrl.o
 .bss           0x00000000        0x0 Src\atten_ctrl.o
 .text.Atten_Test
                0x00000000       0x1a Src\atten_ctrl.o
 .text.Atten_Offset_Calc
                0x00000000       0x86 Src\atten_ctrl.o
 .text.Atten_Table_Read
                0x00000000       0x4a Src\atten_ctrl.o
 .text          0x00000000        0x0 Src\eeprom.o
 .data          0x00000000        0x0 Src\eeprom.o
 .bss           0x00000000        0x0 Src\eeprom.o
 .text          0x00000000        0x0 Src\main.o
 .data          0x00000000        0x0 Src\main.o
 .bss           0x00000000        0x0 Src\main.o
 .text.UartDataRecvSet
                0x00000000        0xc Src\main.o
 .text.UartDataRecvGet
                0x00000000        0xc Src\main.o
 .text.Error_Handler
                0x00000000        0x2 Src\main.o
 .bss.data_complete
                0x00000000        0x1 Src\main.o
 .text          0x00000000        0x0 Src\sth30_crc.o
 .data          0x00000000        0x0 Src\sth30_crc.o
 .bss           0x00000000        0x0 Src\sth30_crc.o
 .text.genCRC16
                0x00000000       0x48 Src\sth30_crc.o
 .data.Table_CRC16
                0x00000000      0x200 Src\sth30_crc.o
 .text          0x00000000        0x0 Src\stm32f2xx_hal_msp.o
 .data          0x00000000        0x0 Src\stm32f2xx_hal_msp.o
 .bss           0x00000000        0x0 Src\stm32f2xx_hal_msp.o
 .text.HAL_I2C_MspDeInit
                0x00000000       0x40 Src\stm32f2xx_hal_msp.o
 .text.HAL_TIM_Base_MspDeInit
                0x00000000       0x24 Src\stm32f2xx_hal_msp.o
 .text.HAL_UART_MspDeInit
                0x00000000       0x38 Src\stm32f2xx_hal_msp.o
 .text          0x00000000        0x0 Src\stm32f2xx_it.o
 .data          0x00000000        0x0 Src\stm32f2xx_it.o
 .bss           0x00000000        0x0 Src\stm32f2xx_it.o
 .text          0x00000000        0x0 Src\system_stm32f2xx.o
 .data          0x00000000        0x0 Src\system_stm32f2xx.o
 .bss           0x00000000        0x0 Src\system_stm32f2xx.o
 .text.SystemCoreClockUpdate
                0x00000000       0x74 Src\system_stm32f2xx.o
 .text          0x00000000       0x14 startup\startup_stm32f207xx.o
 .data          0x00000000        0x0 startup\startup_stm32f207xx.o
 .bss           0x00000000        0x0 startup\startup_stm32f207xx.o
 .text          0x00000000        0x0 c:/program files (x86)/atollic/truestudio for stm32 9.2.0/armtools/bin/../lib/gcc/arm-atollic-eabi/6.3.1/../../../../arm-atollic-eabi/lib/armv7-m\libc_nano.a(lib_a-impure.o)
 .data          0x00000000        0x0 c:/program files (x86)/atollic/truestudio for stm32 9.2.0/armtools/bin/../lib/gcc/arm-atollic-eabi/6.3.1/../../../../arm-atollic-eabi/lib/armv7-m\libc_nano.a(lib_a-impure.o)
 .bss           0x00000000        0x0 c:/program files (x86)/atollic/truestudio for stm32 9.2.0/armtools/bin/../lib/gcc/arm-atollic-eabi/6.3.1/../../../../arm-atollic-eabi/lib/armv7-m\libc_nano.a(lib_a-impure.o)
 .text          0x00000000        0x0 c:/program files (x86)/atollic/truestudio for stm32 9.2.0/armtools/bin/../lib/gcc/arm-atollic-eabi/6.3.1/../../../../arm-atollic-eabi/lib/armv7-m\libc_nano.a(lib_a-init.o)
 .data          0x00000000        0x0 c:/program files (x86)/atollic/truestudio for stm32 9.2.0/armtools/bin/../lib/gcc/arm-atollic-eabi/6.3.1/../../../../arm-atollic-eabi/lib/armv7-m\libc_nano.a(lib_a-init.o)
 .bss           0x00000000        0x0 c:/program files (x86)/atollic/truestudio for stm32 9.2.0/armtools/bin/../lib/gcc/arm-atollic-eabi/6.3.1/../../../../arm-atollic-eabi/lib/armv7-m\libc_nano.a(lib_a-init.o)
 .text          0x00000000        0x0 c:/program files (x86)/atollic/truestudio for stm32 9.2.0/armtools/bin/../lib/gcc/arm-atollic-eabi/6.3.1/../../../../arm-atollic-eabi/lib/armv7-m\libc_nano.a(lib_a-memset.o)
 .data          0x00000000        0x0 c:/program files (x86)/atollic/truestudio for stm32 9.2.0/armtools/bin/../lib/gcc/arm-atollic-eabi/6.3.1/../../../../arm-atollic-eabi/lib/armv7-m\libc_nano.a(lib_a-memset.o)
 .bss           0x00000000        0x0 c:/program files (x86)/atollic/truestudio for stm32 9.2.0/armtools/bin/../lib/gcc/arm-atollic-eabi/6.3.1/../../../../arm-atollic-eabi/lib/armv7-m\libc_nano.a(lib_a-memset.o)
 .text          0x00000000        0x0 c:/program files (x86)/atollic/truestudio for stm32 9.2.0/armtools/bin/../lib/gcc/arm-atollic-eabi/6.3.1/../../../../arm-atollic-eabi/lib/armv7-m\libc_nano.a(lib_a-printf.o)
 .data          0x00000000        0x0 c:/program files (x86)/atollic/truestudio for stm32 9.2.0/armtools/bin/../lib/gcc/arm-atollic-eabi/6.3.1/../../../../arm-atollic-eabi/lib/armv7-m\libc_nano.a(lib_a-printf.o)
 .bss           0x00000000        0x0 c:/program files (x86)/atollic/truestudio for stm32 9.2.0/armtools/bin/../lib/gcc/arm-atollic-eabi/6.3.1/../../../../arm-atollic-eabi/lib/armv7-m\libc_nano.a(lib_a-printf.o)
 .text._printf_r
                0x00000000       0x28 c:/program files (x86)/atollic/truestudio for stm32 9.2.0/armtools/bin/../lib/gcc/arm-atollic-eabi/6.3.1/../../../../arm-atollic-eabi/lib/armv7-m\libc_nano.a(lib_a-printf.o)
 .text          0x00000000        0x0 c:/program files (x86)/atollic/truestudio for stm32 9.2.0/armtools/bin/../lib/gcc/arm-atollic-eabi/6.3.1/../../../../arm-atollic-eabi/lib/armv7-m\libc_nano.a(lib_a-puts.o)
 .data          0x00000000        0x0 c:/program files (x86)/atollic/truestudio for stm32 9.2.0/armtools/bin/../lib/gcc/arm-atollic-eabi/6.3.1/../../../../arm-atollic-eabi/lib/armv7-m\libc_nano.a(lib_a-puts.o)
 .bss           0x00000000        0x0 c:/program files (x86)/atollic/truestudio for stm32 9.2.0/armtools/bin/../lib/gcc/arm-atollic-eabi/6.3.1/../../../../arm-atollic-eabi/lib/armv7-m\libc_nano.a(lib_a-puts.o)
 .text          0x00000000        0x0 c:/program files (x86)/atollic/truestudio for stm32 9.2.0/armtools/bin/../lib/gcc/arm-atollic-eabi/6.3.1/../../../../arm-atollic-eabi/lib/armv7-m\libc_nano.a(lib_a-setbuf.o)
 .data          0x00000000        0x0 c:/program files (x86)/atollic/truestudio for stm32 9.2.0/armtools/bin/../lib/gcc/arm-atollic-eabi/6.3.1/../../../../arm-atollic-eabi/lib/armv7-m\libc_nano.a(lib_a-setbuf.o)
 .bss           0x00000000        0x0 c:/program files (x86)/atollic/truestudio for stm32 9.2.0/armtools/bin/../lib/gcc/arm-atollic-eabi/6.3.1/../../../../arm-atollic-eabi/lib/armv7-m\libc_nano.a(lib_a-setbuf.o)
 .text          0x00000000        0x0 c:/program files (x86)/atollic/truestudio for stm32 9.2.0/armtools/bin/../lib/gcc/arm-atollic-eabi/6.3.1/../../../../arm-atollic-eabi/lib/armv7-m\libc_nano.a(lib_a-setvbuf.o)
 .data          0x00000000        0x0 c:/program files (x86)/atollic/truestudio for stm32 9.2.0/armtools/bin/../lib/gcc/arm-atollic-eabi/6.3.1/../../../../arm-atollic-eabi/lib/armv7-m\libc_nano.a(lib_a-setvbuf.o)
 .bss           0x00000000        0x0 c:/program files (x86)/atollic/truestudio for stm32 9.2.0/armtools/bin/../lib/gcc/arm-atollic-eabi/6.3.1/../../../../arm-atollic-eabi/lib/armv7-m\libc_nano.a(lib_a-setvbuf.o)
 .text          0x00000000        0x0 c:/program files (x86)/atollic/truestudio for stm32 9.2.0/armtools/bin/../lib/gcc/arm-atollic-eabi/6.3.1/../../../../arm-atollic-eabi/lib/armv7-m\libc_nano.a(lib_a-wbuf.o)
 .data          0x00000000        0x0 c:/program files (x86)/atollic/truestudio for stm32 9.2.0/armtools/bin/../lib/gcc/arm-atollic-eabi/6.3.1/../../../../arm-atollic-eabi/lib/armv7-m\libc_nano.a(lib_a-wbuf.o)
 .bss           0x00000000        0x0 c:/program files (x86)/atollic/truestudio for stm32 9.2.0/armtools/bin/../lib/gcc/arm-atollic-eabi/6.3.1/../../../../arm-atollic-eabi/lib/armv7-m\libc_nano.a(lib_a-wbuf.o)
 .text.__swbuf  0x00000000       0x10 c:/program files (x86)/atollic/truestudio for stm32 9.2.0/armtools/bin/../lib/gcc/arm-atollic-eabi/6.3.1/../../../../arm-atollic-eabi/lib/armv7-m\libc_nano.a(lib_a-wbuf.o)
 .text          0x00000000        0x0 c:/program files (x86)/atollic/truestudio for stm32 9.2.0/armtools/bin/../lib/gcc/arm-atollic-eabi/6.3.1/../../../../arm-atollic-eabi/lib/armv7-m\libc_nano.a(lib_a-wsetup.o)
 .data          0x00000000        0x0 c:/program files (x86)/atollic/truestudio for stm32 9.2.0/armtools/bin/../lib/gcc/arm-atollic-eabi/6.3.1/../../../../arm-atollic-eabi/lib/armv7-m\libc_nano.a(lib_a-wsetup.o)
 .bss           0x00000000        0x0 c:/program files (x86)/atollic/truestudio for stm32 9.2.0/armtools/bin/../lib/gcc/arm-atollic-eabi/6.3.1/../../../../arm-atollic-eabi/lib/armv7-m\libc_nano.a(lib_a-wsetup.o)
 .text          0x00000000        0x0 c:/program files (x86)/atollic/truestudio for stm32 9.2.0/armtools/bin/../lib/gcc/arm-atollic-eabi/6.3.1/../../../../arm-atollic-eabi/lib/armv7-m\libc_nano.a(lib_a-fflush.o)
 .data          0x00000000        0x0 c:/program files (x86)/atollic/truestudio for stm32 9.2.0/armtools/bin/../lib/gcc/arm-atollic-eabi/6.3.1/../../../../arm-atollic-eabi/lib/armv7-m\libc_nano.a(lib_a-fflush.o)
 .bss           0x00000000        0x0 c:/program files (x86)/atollic/truestudio for stm32 9.2.0/armtools/bin/../lib/gcc/arm-atollic-eabi/6.3.1/../../../../arm-atollic-eabi/lib/armv7-m\libc_nano.a(lib_a-fflush.o)
 .text.fflush   0x00000000       0x24 c:/program files (x86)/atollic/truestudio for stm32 9.2.0/armtools/bin/../lib/gcc/arm-atollic-eabi/6.3.1/../../../../arm-atollic-eabi/lib/armv7-m\libc_nano.a(lib_a-fflush.o)
 .text          0x00000000        0x0 c:/program files (x86)/atollic/truestudio for stm32 9.2.0/armtools/bin/../lib/gcc/arm-atollic-eabi/6.3.1/../../../../arm-atollic-eabi/lib/armv7-m\libc_nano.a(lib_a-findfp.o)
 .data          0x00000000        0x0 c:/program files (x86)/atollic/truestudio for stm32 9.2.0/armtools/bin/../lib/gcc/arm-atollic-eabi/6.3.1/../../../../arm-atollic-eabi/lib/armv7-m\libc_nano.a(lib_a-findfp.o)
 .bss           0x00000000        0x0 c:/program files (x86)/atollic/truestudio for stm32 9.2.0/armtools/bin/../lib/gcc/arm-atollic-eabi/6.3.1/../../../../arm-atollic-eabi/lib/armv7-m\libc_nano.a(lib_a-findfp.o)
 .text.__fp_unlock
                0x00000000        0x4 c:/program files (x86)/atollic/truestudio for stm32 9.2.0/armtools/bin/../lib/gcc/arm-atollic-eabi/6.3.1/../../../../arm-atollic-eabi/lib/armv7-m\libc_nano.a(lib_a-findfp.o)
 .text.__fp_lock
                0x00000000        0x4 c:/program files (x86)/atollic/truestudio for stm32 9.2.0/armtools/bin/../lib/gcc/arm-atollic-eabi/6.3.1/../../../../arm-atollic-eabi/lib/armv7-m\libc_nano.a(lib_a-findfp.o)
 .text._cleanup
                0x00000000        0xc c:/program files (x86)/atollic/truestudio for stm32 9.2.0/armtools/bin/../lib/gcc/arm-atollic-eabi/6.3.1/../../../../arm-atollic-eabi/lib/armv7-m\libc_nano.a(lib_a-findfp.o)
 .text.__sfp_lock_acquire
                0x00000000        0x2 c:/program files (x86)/atollic/truestudio for stm32 9.2.0/armtools/bin/../lib/gcc/arm-atollic-eabi/6.3.1/../../../../arm-atollic-eabi/lib/armv7-m\libc_nano.a(lib_a-findfp.o)
 .text.__sfp_lock_release
                0x00000000        0x2 c:/program files (x86)/atollic/truestudio for stm32 9.2.0/armtools/bin/../lib/gcc/arm-atollic-eabi/6.3.1/../../../../arm-atollic-eabi/lib/armv7-m\libc_nano.a(lib_a-findfp.o)
 .text.__sinit_lock_acquire
                0x00000000        0x2 c:/program files (x86)/atollic/truestudio for stm32 9.2.0/armtools/bin/../lib/gcc/arm-atollic-eabi/6.3.1/../../../../arm-atollic-eabi/lib/armv7-m\libc_nano.a(lib_a-findfp.o)
 .text.__sinit_lock_release
                0x00000000        0x2 c:/program files (x86)/atollic/truestudio for stm32 9.2.0/armtools/bin/../lib/gcc/arm-atollic-eabi/6.3.1/../../../../arm-atollic-eabi/lib/armv7-m\libc_nano.a(lib_a-findfp.o)
 .text.__fp_lock_all
                0x00000000       0x14 c:/program files (x86)/atollic/truestudio for stm32 9.2.0/armtools/bin/../lib/gcc/arm-atollic-eabi/6.3.1/../../../../arm-atollic-eabi/lib/armv7-m\libc_nano.a(lib_a-findfp.o)
 .text.__fp_unlock_all
                0x00000000       0x14 c:/program files (x86)/atollic/truestudio for stm32 9.2.0/armtools/bin/../lib/gcc/arm-atollic-eabi/6.3.1/../../../../arm-atollic-eabi/lib/armv7-m\libc_nano.a(lib_a-findfp.o)
 .text          0x00000000        0x0 c:/program files (x86)/atollic/truestudio for stm32 9.2.0/armtools/bin/../lib/gcc/arm-atollic-eabi/6.3.1/../../../../arm-atollic-eabi/lib/armv7-m\libc_nano.a(lib_a-fwalk.o)
 .data          0x00000000        0x0 c:/program files (x86)/atollic/truestudio for stm32 9.2.0/armtools/bin/../lib/gcc/arm-atollic-eabi/6.3.1/../../../../arm-atollic-eabi/lib/armv7-m\libc_nano.a(lib_a-fwalk.o)
 .bss           0x00000000        0x0 c:/program files (x86)/atollic/truestudio for stm32 9.2.0/armtools/bin/../lib/gcc/arm-atollic-eabi/6.3.1/../../../../arm-atollic-eabi/lib/armv7-m\libc_nano.a(lib_a-fwalk.o)
 .text._fwalk   0x00000000       0x38 c:/program files (x86)/atollic/truestudio for stm32 9.2.0/armtools/bin/../lib/gcc/arm-atollic-eabi/6.3.1/../../../../arm-atollic-eabi/lib/armv7-m\libc_nano.a(lib_a-fwalk.o)
 .text          0x00000000        0x0 c:/program files (x86)/atollic/truestudio for stm32 9.2.0/armtools/bin/../lib/gcc/arm-atollic-eabi/6.3.1/../../../../arm-atollic-eabi/lib/armv7-m\libc_nano.a(lib_a-makebuf.o)
 .data          0x00000000        0x0 c:/program files (x86)/atollic/truestudio for stm32 9.2.0/armtools/bin/../lib/gcc/arm-atollic-eabi/6.3.1/../../../../arm-atollic-eabi/lib/armv7-m\libc_nano.a(lib_a-makebuf.o)
 .bss           0x00000000        0x0 c:/program files (x86)/atollic/truestudio for stm32 9.2.0/armtools/bin/../lib/gcc/arm-atollic-eabi/6.3.1/../../../../arm-atollic-eabi/lib/armv7-m\libc_nano.a(lib_a-makebuf.o)
 .text          0x00000000        0x0 c:/program files (x86)/atollic/truestudio for stm32 9.2.0/armtools/bin/../lib/gcc/arm-atollic-eabi/6.3.1/../../../../arm-atollic-eabi/lib/armv7-m\libc_nano.a(lib_a-malloc.o)
 .data          0x00000000        0x0 c:/program files (x86)/atollic/truestudio for stm32 9.2.0/armtools/bin/../lib/gcc/arm-atollic-eabi/6.3.1/../../../../arm-atollic-eabi/lib/armv7-m\libc_nano.a(lib_a-malloc.o)
 .bss           0x00000000        0x0 c:/program files (x86)/atollic/truestudio for stm32 9.2.0/armtools/bin/../lib/gcc/arm-atollic-eabi/6.3.1/../../../../arm-atollic-eabi/lib/armv7-m\libc_nano.a(lib_a-malloc.o)
 .text.free     0x00000000       0x10 c:/program files (x86)/atollic/truestudio for stm32 9.2.0/armtools/bin/../lib/gcc/arm-atollic-eabi/6.3.1/../../../../arm-atollic-eabi/lib/armv7-m\libc_nano.a(lib_a-malloc.o)
 .text          0x00000000        0x0 c:/program files (x86)/atollic/truestudio for stm32 9.2.0/armtools/bin/../lib/gcc/arm-atollic-eabi/6.3.1/../../../../arm-atollic-eabi/lib/armv7-m\libc_nano.a(lib_a-nano-freer.o)
 .data          0x00000000        0x0 c:/program files (x86)/atollic/truestudio for stm32 9.2.0/armtools/bin/../lib/gcc/arm-atollic-eabi/6.3.1/../../../../arm-atollic-eabi/lib/armv7-m\libc_nano.a(lib_a-nano-freer.o)
 .bss           0x00000000        0x0 c:/program files (x86)/atollic/truestudio for stm32 9.2.0/armtools/bin/../lib/gcc/arm-atollic-eabi/6.3.1/../../../../arm-atollic-eabi/lib/armv7-m\libc_nano.a(lib_a-nano-freer.o)
 .text          0x00000000        0x0 c:/program files (x86)/atollic/truestudio for stm32 9.2.0/armtools/bin/../lib/gcc/arm-atollic-eabi/6.3.1/../../../../arm-atollic-eabi/lib/armv7-m\libc_nano.a(lib_a-nano-mallocr.o)
 .data          0x00000000        0x0 c:/program files (x86)/atollic/truestudio for stm32 9.2.0/armtools/bin/../lib/gcc/arm-atollic-eabi/6.3.1/../../../../arm-atollic-eabi/lib/armv7-m\libc_nano.a(lib_a-nano-mallocr.o)
 .bss           0x00000000        0x0 c:/program files (x86)/atollic/truestudio for stm32 9.2.0/armtools/bin/../lib/gcc/arm-atollic-eabi/6.3.1/../../../../arm-atollic-eabi/lib/armv7-m\libc_nano.a(lib_a-nano-mallocr.o)
 .text          0x00000000        0x0 c:/program files (x86)/atollic/truestudio for stm32 9.2.0/armtools/bin/../lib/gcc/arm-atollic-eabi/6.3.1/../../../../arm-atollic-eabi/lib/armv7-m\libc_nano.a(lib_a-nano-vfprintf.o)
 .data          0x00000000        0x0 c:/program files (x86)/atollic/truestudio for stm32 9.2.0/armtools/bin/../lib/gcc/arm-atollic-eabi/6.3.1/../../../../arm-atollic-eabi/lib/armv7-m\libc_nano.a(lib_a-nano-vfprintf.o)
 .bss           0x00000000        0x0 c:/program files (x86)/atollic/truestudio for stm32 9.2.0/armtools/bin/../lib/gcc/arm-atollic-eabi/6.3.1/../../../../arm-atollic-eabi/lib/armv7-m\libc_nano.a(lib_a-nano-vfprintf.o)
 .text.__sprint_r
                0x00000000       0x1a c:/program files (x86)/atollic/truestudio for stm32 9.2.0/armtools/bin/../lib/gcc/arm-atollic-eabi/6.3.1/../../../../arm-atollic-eabi/lib/armv7-m\libc_nano.a(lib_a-nano-vfprintf.o)
 .text.vfprintf
                0x00000000       0x14 c:/program files (x86)/atollic/truestudio for stm32 9.2.0/armtools/bin/../lib/gcc/arm-atollic-eabi/6.3.1/../../../../arm-atollic-eabi/lib/armv7-m\libc_nano.a(lib_a-nano-vfprintf.o)
 .text          0x00000000        0x0 c:/program files (x86)/atollic/truestudio for stm32 9.2.0/armtools/bin/../lib/gcc/arm-atollic-eabi/6.3.1/../../../../arm-atollic-eabi/lib/armv7-m\libc_nano.a(lib_a-nano-vfprintf_i.o)
 .data          0x00000000        0x0 c:/program files (x86)/atollic/truestudio for stm32 9.2.0/armtools/bin/../lib/gcc/arm-atollic-eabi/6.3.1/../../../../arm-atollic-eabi/lib/armv7-m\libc_nano.a(lib_a-nano-vfprintf_i.o)
 .bss           0x00000000        0x0 c:/program files (x86)/atollic/truestudio for stm32 9.2.0/armtools/bin/../lib/gcc/arm-atollic-eabi/6.3.1/../../../../arm-atollic-eabi/lib/armv7-m\libc_nano.a(lib_a-nano-vfprintf_i.o)
 .text          0x00000000        0x0 c:/program files (x86)/atollic/truestudio for stm32 9.2.0/armtools/bin/../lib/gcc/arm-atollic-eabi/6.3.1/../../../../arm-atollic-eabi/lib/armv7-m\libc_nano.a(lib_a-sbrkr.o)
 .data          0x00000000        0x0 c:/program files (x86)/atollic/truestudio for stm32 9.2.0/armtools/bin/../lib/gcc/arm-atollic-eabi/6.3.1/../../../../arm-atollic-eabi/lib/armv7-m\libc_nano.a(lib_a-sbrkr.o)
 .bss           0x00000000        0x0 c:/program files (x86)/atollic/truestudio for stm32 9.2.0/armtools/bin/../lib/gcc/arm-atollic-eabi/6.3.1/../../../../arm-atollic-eabi/lib/armv7-m\libc_nano.a(lib_a-sbrkr.o)
 .text          0x00000000        0x0 c:/program files (x86)/atollic/truestudio for stm32 9.2.0/armtools/bin/../lib/gcc/arm-atollic-eabi/6.3.1/../../../../arm-atollic-eabi/lib/armv7-m\libc_nano.a(lib_a-stdio.o)
 .data          0x00000000        0x0 c:/program files (x86)/atollic/truestudio for stm32 9.2.0/armtools/bin/../lib/gcc/arm-atollic-eabi/6.3.1/../../../../arm-atollic-eabi/lib/armv7-m\libc_nano.a(lib_a-stdio.o)
 .bss           0x00000000        0x0 c:/program files (x86)/atollic/truestudio for stm32 9.2.0/armtools/bin/../lib/gcc/arm-atollic-eabi/6.3.1/../../../../arm-atollic-eabi/lib/armv7-m\libc_nano.a(lib_a-stdio.o)
 .text.__seofread
                0x00000000        0x4 c:/program files (x86)/atollic/truestudio for stm32 9.2.0/armtools/bin/../lib/gcc/arm-atollic-eabi/6.3.1/../../../../arm-atollic-eabi/lib/armv7-m\libc_nano.a(lib_a-stdio.o)
 .text          0x00000000        0x0 c:/program files (x86)/atollic/truestudio for stm32 9.2.0/armtools/bin/../lib/gcc/arm-atollic-eabi/6.3.1/../../../../arm-atollic-eabi/lib/armv7-m\libc_nano.a(lib_a-writer.o)
 .data          0x00000000        0x0 c:/program files (x86)/atollic/truestudio for stm32 9.2.0/armtools/bin/../lib/gcc/arm-atollic-eabi/6.3.1/../../../../arm-atollic-eabi/lib/armv7-m\libc_nano.a(lib_a-writer.o)
 .bss           0x00000000        0x0 c:/program files (x86)/atollic/truestudio for stm32 9.2.0/armtools/bin/../lib/gcc/arm-atollic-eabi/6.3.1/../../../../arm-atollic-eabi/lib/armv7-m\libc_nano.a(lib_a-writer.o)
 .text          0x00000000        0x0 c:/program files (x86)/atollic/truestudio for stm32 9.2.0/armtools/bin/../lib/gcc/arm-atollic-eabi/6.3.1/../../../../arm-atollic-eabi/lib/armv7-m\libc_nano.a(lib_a-closer.o)
 .data          0x00000000        0x0 c:/program files (x86)/atollic/truestudio for stm32 9.2.0/armtools/bin/../lib/gcc/arm-atollic-eabi/6.3.1/../../../../arm-atollic-eabi/lib/armv7-m\libc_nano.a(lib_a-closer.o)
 .bss           0x00000000        0x0 c:/program files (x86)/atollic/truestudio for stm32 9.2.0/armtools/bin/../lib/gcc/arm-atollic-eabi/6.3.1/../../../../arm-atollic-eabi/lib/armv7-m\libc_nano.a(lib_a-closer.o)
 .text          0x00000000        0x0 c:/program files (x86)/atollic/truestudio for stm32 9.2.0/armtools/bin/../lib/gcc/arm-atollic-eabi/6.3.1/../../../../arm-atollic-eabi/lib/armv7-m\libc_nano.a(lib_a-fstatr.o)
 .data          0x00000000        0x0 c:/program files (x86)/atollic/truestudio for stm32 9.2.0/armtools/bin/../lib/gcc/arm-atollic-eabi/6.3.1/../../../../arm-atollic-eabi/lib/armv7-m\libc_nano.a(lib_a-fstatr.o)
 .bss           0x00000000        0x0 c:/program files (x86)/atollic/truestudio for stm32 9.2.0/armtools/bin/../lib/gcc/arm-atollic-eabi/6.3.1/../../../../arm-atollic-eabi/lib/armv7-m\libc_nano.a(lib_a-fstatr.o)
 .text          0x00000000        0x0 c:/program files (x86)/atollic/truestudio for stm32 9.2.0/armtools/bin/../lib/gcc/arm-atollic-eabi/6.3.1/../../../../arm-atollic-eabi/lib/armv7-m\libc_nano.a(lib_a-fvwrite.o)
 .data          0x00000000        0x0 c:/program files (x86)/atollic/truestudio for stm32 9.2.0/armtools/bin/../lib/gcc/arm-atollic-eabi/6.3.1/../../../../arm-atollic-eabi/lib/armv7-m\libc_nano.a(lib_a-fvwrite.o)
 .bss           0x00000000        0x0 c:/program files (x86)/atollic/truestudio for stm32 9.2.0/armtools/bin/../lib/gcc/arm-atollic-eabi/6.3.1/../../../../arm-atollic-eabi/lib/armv7-m\libc_nano.a(lib_a-fvwrite.o)
 .text.__sfvwrite_r
                0x00000000      0x29c c:/program files (x86)/atollic/truestudio for stm32 9.2.0/armtools/bin/../lib/gcc/arm-atollic-eabi/6.3.1/../../../../arm-atollic-eabi/lib/armv7-m\libc_nano.a(lib_a-fvwrite.o)
 .debug_frame   0x00000000       0x3c c:/program files (x86)/atollic/truestudio for stm32 9.2.0/armtools/bin/../lib/gcc/arm-atollic-eabi/6.3.1/../../../../arm-atollic-eabi/lib/armv7-m\libc_nano.a(lib_a-fvwrite.o)
 .ARM.attributes
                0x00000000       0x2d c:/program files (x86)/atollic/truestudio for stm32 9.2.0/armtools/bin/../lib/gcc/arm-atollic-eabi/6.3.1/../../../../arm-atollic-eabi/lib/armv7-m\libc_nano.a(lib_a-fvwrite.o)
 .text          0x00000000        0x0 c:/program files (x86)/atollic/truestudio for stm32 9.2.0/armtools/bin/../lib/gcc/arm-atollic-eabi/6.3.1/../../../../arm-atollic-eabi/lib/armv7-m\libc_nano.a(lib_a-isattyr.o)
 .data          0x00000000        0x0 c:/program files (x86)/atollic/truestudio for stm32 9.2.0/armtools/bin/../lib/gcc/arm-atollic-eabi/6.3.1/../../../../arm-atollic-eabi/lib/armv7-m\libc_nano.a(lib_a-isattyr.o)
 .bss           0x00000000        0x0 c:/program files (x86)/atollic/truestudio for stm32 9.2.0/armtools/bin/../lib/gcc/arm-atollic-eabi/6.3.1/../../../../arm-atollic-eabi/lib/armv7-m\libc_nano.a(lib_a-isattyr.o)
 .text          0x00000000        0x0 c:/program files (x86)/atollic/truestudio for stm32 9.2.0/armtools/bin/../lib/gcc/arm-atollic-eabi/6.3.1/../../../../arm-atollic-eabi/lib/armv7-m\libc_nano.a(lib_a-lseekr.o)
 .data          0x00000000        0x0 c:/program files (x86)/atollic/truestudio for stm32 9.2.0/armtools/bin/../lib/gcc/arm-atollic-eabi/6.3.1/../../../../arm-atollic-eabi/lib/armv7-m\libc_nano.a(lib_a-lseekr.o)
 .bss           0x00000000        0x0 c:/program files (x86)/atollic/truestudio for stm32 9.2.0/armtools/bin/../lib/gcc/arm-atollic-eabi/6.3.1/../../../../arm-atollic-eabi/lib/armv7-m\libc_nano.a(lib_a-lseekr.o)
 .text          0x00000000        0x0 c:/program files (x86)/atollic/truestudio for stm32 9.2.0/armtools/bin/../lib/gcc/arm-atollic-eabi/6.3.1/../../../../arm-atollic-eabi/lib/armv7-m\libc_nano.a(lib_a-memchr-stub.o)
 .data          0x00000000        0x0 c:/program files (x86)/atollic/truestudio for stm32 9.2.0/armtools/bin/../lib/gcc/arm-atollic-eabi/6.3.1/../../../../arm-atollic-eabi/lib/armv7-m\libc_nano.a(lib_a-memchr-stub.o)
 .bss           0x00000000        0x0 c:/program files (x86)/atollic/truestudio for stm32 9.2.0/armtools/bin/../lib/gcc/arm-atollic-eabi/6.3.1/../../../../arm-atollic-eabi/lib/armv7-m\libc_nano.a(lib_a-memchr-stub.o)
 .text          0x00000000        0x0 c:/program files (x86)/atollic/truestudio for stm32 9.2.0/armtools/bin/../lib/gcc/arm-atollic-eabi/6.3.1/../../../../arm-atollic-eabi/lib/armv7-m\libc_nano.a(lib_a-memcpy-stub.o)
 .data          0x00000000        0x0 c:/program files (x86)/atollic/truestudio for stm32 9.2.0/armtools/bin/../lib/gcc/arm-atollic-eabi/6.3.1/../../../../arm-atollic-eabi/lib/armv7-m\libc_nano.a(lib_a-memcpy-stub.o)
 .bss           0x00000000        0x0 c:/program files (x86)/atollic/truestudio for stm32 9.2.0/armtools/bin/../lib/gcc/arm-atollic-eabi/6.3.1/../../../../arm-atollic-eabi/lib/armv7-m\libc_nano.a(lib_a-memcpy-stub.o)
 .text.memcpy   0x00000000       0x16 c:/program files (x86)/atollic/truestudio for stm32 9.2.0/armtools/bin/../lib/gcc/arm-atollic-eabi/6.3.1/../../../../arm-atollic-eabi/lib/armv7-m\libc_nano.a(lib_a-memcpy-stub.o)
 .debug_frame   0x00000000       0x28 c:/program files (x86)/atollic/truestudio for stm32 9.2.0/armtools/bin/../lib/gcc/arm-atollic-eabi/6.3.1/../../../../arm-atollic-eabi/lib/armv7-m\libc_nano.a(lib_a-memcpy-stub.o)
 .ARM.attributes
                0x00000000       0x2d c:/program files (x86)/atollic/truestudio for stm32 9.2.0/armtools/bin/../lib/gcc/arm-atollic-eabi/6.3.1/../../../../arm-atollic-eabi/lib/armv7-m\libc_nano.a(lib_a-memcpy-stub.o)
 .text          0x00000000        0x0 c:/program files (x86)/atollic/truestudio for stm32 9.2.0/armtools/bin/../lib/gcc/arm-atollic-eabi/6.3.1/../../../../arm-atollic-eabi/lib/armv7-m\libc_nano.a(lib_a-memmove.o)
 .data          0x00000000        0x0 c:/program files (x86)/atollic/truestudio for stm32 9.2.0/armtools/bin/../lib/gcc/arm-atollic-eabi/6.3.1/../../../../arm-atollic-eabi/lib/armv7-m\libc_nano.a(lib_a-memmove.o)
 .bss           0x00000000        0x0 c:/program files (x86)/atollic/truestudio for stm32 9.2.0/armtools/bin/../lib/gcc/arm-atollic-eabi/6.3.1/../../../../arm-atollic-eabi/lib/armv7-m\libc_nano.a(lib_a-memmove.o)
 .text.memmove  0x00000000       0x34 c:/program files (x86)/atollic/truestudio for stm32 9.2.0/armtools/bin/../lib/gcc/arm-atollic-eabi/6.3.1/../../../../arm-atollic-eabi/lib/armv7-m\libc_nano.a(lib_a-memmove.o)
 .debug_frame   0x00000000       0x28 c:/program files (x86)/atollic/truestudio for stm32 9.2.0/armtools/bin/../lib/gcc/arm-atollic-eabi/6.3.1/../../../../arm-atollic-eabi/lib/armv7-m\libc_nano.a(lib_a-memmove.o)
 .ARM.attributes
                0x00000000       0x2d c:/program files (x86)/atollic/truestudio for stm32 9.2.0/armtools/bin/../lib/gcc/arm-atollic-eabi/6.3.1/../../../../arm-atollic-eabi/lib/armv7-m\libc_nano.a(lib_a-memmove.o)
 .text          0x00000000        0x0 c:/program files (x86)/atollic/truestudio for stm32 9.2.0/armtools/bin/../lib/gcc/arm-atollic-eabi/6.3.1/../../../../arm-atollic-eabi/lib/armv7-m\libc_nano.a(lib_a-mlock.o)
 .data          0x00000000        0x0 c:/program files (x86)/atollic/truestudio for stm32 9.2.0/armtools/bin/../lib/gcc/arm-atollic-eabi/6.3.1/../../../../arm-atollic-eabi/lib/armv7-m\libc_nano.a(lib_a-mlock.o)
 .bss           0x00000000        0x0 c:/program files (x86)/atollic/truestudio for stm32 9.2.0/armtools/bin/../lib/gcc/arm-atollic-eabi/6.3.1/../../../../arm-atollic-eabi/lib/armv7-m\libc_nano.a(lib_a-mlock.o)
 .text          0x00000000        0x0 c:/program files (x86)/atollic/truestudio for stm32 9.2.0/armtools/bin/../lib/gcc/arm-atollic-eabi/6.3.1/../../../../arm-atollic-eabi/lib/armv7-m\libc_nano.a(lib_a-nano-reallocr.o)
 .data          0x00000000        0x0 c:/program files (x86)/atollic/truestudio for stm32 9.2.0/armtools/bin/../lib/gcc/arm-atollic-eabi/6.3.1/../../../../arm-atollic-eabi/lib/armv7-m\libc_nano.a(lib_a-nano-reallocr.o)
 .bss           0x00000000        0x0 c:/program files (x86)/atollic/truestudio for stm32 9.2.0/armtools/bin/../lib/gcc/arm-atollic-eabi/6.3.1/../../../../arm-atollic-eabi/lib/armv7-m\libc_nano.a(lib_a-nano-reallocr.o)
 .text._realloc_r
                0x00000000       0x4c c:/program files (x86)/atollic/truestudio for stm32 9.2.0/armtools/bin/../lib/gcc/arm-atollic-eabi/6.3.1/../../../../arm-atollic-eabi/lib/armv7-m\libc_nano.a(lib_a-nano-reallocr.o)
 .debug_frame   0x00000000       0x3c c:/program files (x86)/atollic/truestudio for stm32 9.2.0/armtools/bin/../lib/gcc/arm-atollic-eabi/6.3.1/../../../../arm-atollic-eabi/lib/armv7-m\libc_nano.a(lib_a-nano-reallocr.o)
 .ARM.attributes
                0x00000000       0x2d c:/program files (x86)/atollic/truestudio for stm32 9.2.0/armtools/bin/../lib/gcc/arm-atollic-eabi/6.3.1/../../../../arm-atollic-eabi/lib/armv7-m\libc_nano.a(lib_a-nano-reallocr.o)
 .text          0x00000000        0x0 c:/program files (x86)/atollic/truestudio for stm32 9.2.0/armtools/bin/../lib/gcc/arm-atollic-eabi/6.3.1/../../../../arm-atollic-eabi/lib/armv7-m\libc_nano.a(lib_a-readr.o)
 .data          0x00000000        0x0 c:/program files (x86)/atollic/truestudio for stm32 9.2.0/armtools/bin/../lib/gcc/arm-atollic-eabi/6.3.1/../../../../arm-atollic-eabi/lib/armv7-m\libc_nano.a(lib_a-readr.o)
 .bss           0x00000000        0x0 c:/program files (x86)/atollic/truestudio for stm32 9.2.0/armtools/bin/../lib/gcc/arm-atollic-eabi/6.3.1/../../../../arm-atollic-eabi/lib/armv7-m\libc_nano.a(lib_a-readr.o)
 .text          0x00000000        0x0 c:/program files (x86)/atollic/truestudio for stm32 9.2.0/armtools/bin/../lib/gcc/arm-atollic-eabi/6.3.1/../../../../arm-atollic-eabi/lib/armv7-m\libc_nano.a(lib_a-reent.o)
 .data          0x00000000        0x0 c:/program files (x86)/atollic/truestudio for stm32 9.2.0/armtools/bin/../lib/gcc/arm-atollic-eabi/6.3.1/../../../../arm-atollic-eabi/lib/armv7-m\libc_nano.a(lib_a-reent.o)
 .bss           0x00000000        0x0 c:/program files (x86)/atollic/truestudio for stm32 9.2.0/armtools/bin/../lib/gcc/arm-atollic-eabi/6.3.1/../../../../arm-atollic-eabi/lib/armv7-m\libc_nano.a(lib_a-reent.o)
 .text.cleanup_glue
                0x00000000       0x1a c:/program files (x86)/atollic/truestudio for stm32 9.2.0/armtools/bin/../lib/gcc/arm-atollic-eabi/6.3.1/../../../../arm-atollic-eabi/lib/armv7-m\libc_nano.a(lib_a-reent.o)
 .text._reclaim_reent
                0x00000000       0xb8 c:/program files (x86)/atollic/truestudio for stm32 9.2.0/armtools/bin/../lib/gcc/arm-atollic-eabi/6.3.1/../../../../arm-atollic-eabi/lib/armv7-m\libc_nano.a(lib_a-reent.o)
 .text          0x00000000        0x0 c:/program files (x86)/atollic/truestudio for stm32 9.2.0/armtools/bin/../lib/gcc/arm-atollic-eabi/6.3.1/../../../../arm-atollic-eabi/lib/armv7-m\libc_nano.a(lib_a-nano-msizer.o)
 .data          0x00000000        0x0 c:/program files (x86)/atollic/truestudio for stm32 9.2.0/armtools/bin/../lib/gcc/arm-atollic-eabi/6.3.1/../../../../arm-atollic-eabi/lib/armv7-m\libc_nano.a(lib_a-nano-msizer.o)
 .bss           0x00000000        0x0 c:/program files (x86)/atollic/truestudio for stm32 9.2.0/armtools/bin/../lib/gcc/arm-atollic-eabi/6.3.1/../../../../arm-atollic-eabi/lib/armv7-m\libc_nano.a(lib_a-nano-msizer.o)
 .text._malloc_usable_size_r
                0x00000000       0x12 c:/program files (x86)/atollic/truestudio for stm32 9.2.0/armtools/bin/../lib/gcc/arm-atollic-eabi/6.3.1/../../../../arm-atollic-eabi/lib/armv7-m\libc_nano.a(lib_a-nano-msizer.o)
 .debug_frame   0x00000000       0x20 c:/program files (x86)/atollic/truestudio for stm32 9.2.0/armtools/bin/../lib/gcc/arm-atollic-eabi/6.3.1/../../../../arm-atollic-eabi/lib/armv7-m\libc_nano.a(lib_a-nano-msizer.o)
 .ARM.attributes
                0x00000000       0x2d c:/program files (x86)/atollic/truestudio for stm32 9.2.0/armtools/bin/../lib/gcc/arm-atollic-eabi/6.3.1/../../../../arm-atollic-eabi/lib/armv7-m\libc_nano.a(lib_a-nano-msizer.o)
 .data          0x00000000        0x0 c:/program files (x86)/atollic/truestudio for stm32 9.2.0/armtools/bin/../lib/gcc/arm-atollic-eabi/6.3.1/armv7-m\libgcc.a(_aeabi_uldivmod.o)
 .bss           0x00000000        0x0 c:/program files (x86)/atollic/truestudio for stm32 9.2.0/armtools/bin/../lib/gcc/arm-atollic-eabi/6.3.1/armv7-m\libgcc.a(_aeabi_uldivmod.o)
 .data          0x00000000        0x0 c:/program files (x86)/atollic/truestudio for stm32 9.2.0/armtools/bin/../lib/gcc/arm-atollic-eabi/6.3.1/armv7-m\libgcc.a(_udivmoddi4.o)
 .bss           0x00000000        0x0 c:/program files (x86)/atollic/truestudio for stm32 9.2.0/armtools/bin/../lib/gcc/arm-atollic-eabi/6.3.1/armv7-m\libgcc.a(_udivmoddi4.o)
 .ARM.extab     0x00000000        0x0 c:/program files (x86)/atollic/truestudio for stm32 9.2.0/armtools/bin/../lib/gcc/arm-atollic-eabi/6.3.1/armv7-m\libgcc.a(_udivmoddi4.o)
 .data          0x00000000        0x0 c:/program files (x86)/atollic/truestudio for stm32 9.2.0/armtools/bin/../lib/gcc/arm-atollic-eabi/6.3.1/armv7-m\libgcc.a(_dvmd_tls.o)
 .bss           0x00000000        0x0 c:/program files (x86)/atollic/truestudio for stm32 9.2.0/armtools/bin/../lib/gcc/arm-atollic-eabi/6.3.1/armv7-m\libgcc.a(_dvmd_tls.o)
 .text          0x00000000        0x0 c:/program files (x86)/atollic/truestudio for stm32 9.2.0/armtools/bin/../lib/gcc/arm-atollic-eabi/6.3.1/../../../../arm-atollic-eabi/lib/armv7-m\libnosys.a(close.o)
 .data          0x00000000        0x0 c:/program files (x86)/atollic/truestudio for stm32 9.2.0/armtools/bin/../lib/gcc/arm-atollic-eabi/6.3.1/../../../../arm-atollic-eabi/lib/armv7-m\libnosys.a(close.o)
 .bss           0x00000000        0x0 c:/program files (x86)/atollic/truestudio for stm32 9.2.0/armtools/bin/../lib/gcc/arm-atollic-eabi/6.3.1/../../../../arm-atollic-eabi/lib/armv7-m\libnosys.a(close.o)
 .text          0x00000000        0x0 c:/program files (x86)/atollic/truestudio for stm32 9.2.0/armtools/bin/../lib/gcc/arm-atollic-eabi/6.3.1/../../../../arm-atollic-eabi/lib/armv7-m\libnosys.a(fstat.o)
 .data          0x00000000        0x0 c:/program files (x86)/atollic/truestudio for stm32 9.2.0/armtools/bin/../lib/gcc/arm-atollic-eabi/6.3.1/../../../../arm-atollic-eabi/lib/armv7-m\libnosys.a(fstat.o)
 .bss           0x00000000        0x0 c:/program files (x86)/atollic/truestudio for stm32 9.2.0/armtools/bin/../lib/gcc/arm-atollic-eabi/6.3.1/../../../../arm-atollic-eabi/lib/armv7-m\libnosys.a(fstat.o)
 .text          0x00000000        0x0 c:/program files (x86)/atollic/truestudio for stm32 9.2.0/armtools/bin/../lib/gcc/arm-atollic-eabi/6.3.1/../../../../arm-atollic-eabi/lib/armv7-m\libnosys.a(isatty.o)
 .data          0x00000000        0x0 c:/program files (x86)/atollic/truestudio for stm32 9.2.0/armtools/bin/../lib/gcc/arm-atollic-eabi/6.3.1/../../../../arm-atollic-eabi/lib/armv7-m\libnosys.a(isatty.o)
 .bss           0x00000000        0x0 c:/program files (x86)/atollic/truestudio for stm32 9.2.0/armtools/bin/../lib/gcc/arm-atollic-eabi/6.3.1/../../../../arm-atollic-eabi/lib/armv7-m\libnosys.a(isatty.o)
 .text          0x00000000        0x0 c:/program files (x86)/atollic/truestudio for stm32 9.2.0/armtools/bin/../lib/gcc/arm-atollic-eabi/6.3.1/../../../../arm-atollic-eabi/lib/armv7-m\libnosys.a(lseek.o)
 .data          0x00000000        0x0 c:/program files (x86)/atollic/truestudio for stm32 9.2.0/armtools/bin/../lib/gcc/arm-atollic-eabi/6.3.1/../../../../arm-atollic-eabi/lib/armv7-m\libnosys.a(lseek.o)
 .bss           0x00000000        0x0 c:/program files (x86)/atollic/truestudio for stm32 9.2.0/armtools/bin/../lib/gcc/arm-atollic-eabi/6.3.1/../../../../arm-atollic-eabi/lib/armv7-m\libnosys.a(lseek.o)
 .text          0x00000000        0x0 c:/program files (x86)/atollic/truestudio for stm32 9.2.0/armtools/bin/../lib/gcc/arm-atollic-eabi/6.3.1/../../../../arm-atollic-eabi/lib/armv7-m\libnosys.a(read.o)
 .data          0x00000000        0x0 c:/program files (x86)/atollic/truestudio for stm32 9.2.0/armtools/bin/../lib/gcc/arm-atollic-eabi/6.3.1/../../../../arm-atollic-eabi/lib/armv7-m\libnosys.a(read.o)
 .bss           0x00000000        0x0 c:/program files (x86)/atollic/truestudio for stm32 9.2.0/armtools/bin/../lib/gcc/arm-atollic-eabi/6.3.1/../../../../arm-atollic-eabi/lib/armv7-m\libnosys.a(read.o)
 .text          0x00000000        0x0 c:/program files (x86)/atollic/truestudio for stm32 9.2.0/armtools/bin/../lib/gcc/arm-atollic-eabi/6.3.1/../../../../arm-atollic-eabi/lib/armv7-m\libnosys.a(sbrk.o)
 .data          0x00000000        0x0 c:/program files (x86)/atollic/truestudio for stm32 9.2.0/armtools/bin/../lib/gcc/arm-atollic-eabi/6.3.1/../../../../arm-atollic-eabi/lib/armv7-m\libnosys.a(sbrk.o)
 .bss           0x00000000        0x0 c:/program files (x86)/atollic/truestudio for stm32 9.2.0/armtools/bin/../lib/gcc/arm-atollic-eabi/6.3.1/../../../../arm-atollic-eabi/lib/armv7-m\libnosys.a(sbrk.o)
 .text          0x00000000        0x0 c:/program files (x86)/atollic/truestudio for stm32 9.2.0/armtools/bin/../lib/gcc/arm-atollic-eabi/6.3.1/armv7-m/crtend.o
 .data          0x00000000        0x0 c:/program files (x86)/atollic/truestudio for stm32 9.2.0/armtools/bin/../lib/gcc/arm-atollic-eabi/6.3.1/armv7-m/crtend.o
 .bss           0x00000000        0x0 c:/program files (x86)/atollic/truestudio for stm32 9.2.0/armtools/bin/../lib/gcc/arm-atollic-eabi/6.3.1/armv7-m/crtend.o
 .eh_frame      0x00000000        0x4 c:/program files (x86)/atollic/truestudio for stm32 9.2.0/armtools/bin/../lib/gcc/arm-atollic-eabi/6.3.1/armv7-m/crtend.o
 .ARM.attributes
                0x00000000       0x2d c:/program files (x86)/atollic/truestudio for stm32 9.2.0/armtools/bin/../lib/gcc/arm-atollic-eabi/6.3.1/armv7-m/crtend.o
 .text          0x00000000        0x0 c:/program files (x86)/atollic/truestudio for stm32 9.2.0/armtools/bin/../lib/gcc/arm-atollic-eabi/6.3.1/armv7-m/crtn.o
 .data          0x00000000        0x0 c:/program files (x86)/atollic/truestudio for stm32 9.2.0/armtools/bin/../lib/gcc/arm-atollic-eabi/6.3.1/armv7-m/crtn.o
 .bss           0x00000000        0x0 c:/program files (x86)/atollic/truestudio for stm32 9.2.0/armtools/bin/../lib/gcc/arm-atollic-eabi/6.3.1/armv7-m/crtn.o

Memory Configuration

Name             Origin             Length             Attributes
RAM              0x20000000         0x00020000         xrw
FLASH            0x08000000         0x00040000         xr
*default*        0x00000000         0xffffffff

Linker script and memory map

LOAD c:/program files (x86)/atollic/truestudio for stm32 9.2.0/armtools/bin/../lib/gcc/arm-atollic-eabi/6.3.1/armv7-m/crti.o
LOAD c:/program files (x86)/atollic/truestudio for stm32 9.2.0/armtools/bin/../lib/gcc/arm-atollic-eabi/6.3.1/armv7-m/crtbegin.o
LOAD Drivers\STM32F2xx_HAL_Driver\Src\stm32f2xx_hal.o
LOAD Drivers\STM32F2xx_HAL_Driver\Src\stm32f2xx_hal_cortex.o
LOAD Drivers\STM32F2xx_HAL_Driver\Src\stm32f2xx_hal_dma.o
LOAD Drivers\STM32F2xx_HAL_Driver\Src\stm32f2xx_hal_dma_ex.o
LOAD Drivers\STM32F2xx_HAL_Driver\Src\stm32f2xx_hal_flash.o
LOAD Drivers\STM32F2xx_HAL_Driver\Src\stm32f2xx_hal_flash_ex.o
LOAD Drivers\STM32F2xx_HAL_Driver\Src\stm32f2xx_hal_gpio.o
LOAD Drivers\STM32F2xx_HAL_Driver\Src\stm32f2xx_hal_i2c.o
LOAD Drivers\STM32F2xx_HAL_Driver\Src\stm32f2xx_hal_pwr.o
LOAD Drivers\STM32F2xx_HAL_Driver\Src\stm32f2xx_hal_pwr_ex.o
LOAD Drivers\STM32F2xx_HAL_Driver\Src\stm32f2xx_hal_rcc.o
LOAD Drivers\STM32F2xx_HAL_Driver\Src\stm32f2xx_hal_rcc_ex.o
LOAD Drivers\STM32F2xx_HAL_Driver\Src\stm32f2xx_hal_tim.o
LOAD Drivers\STM32F2xx_HAL_Driver\Src\stm32f2xx_hal_tim_ex.o
LOAD Drivers\STM32F2xx_HAL_Driver\Src\stm32f2xx_hal_uart.o
LOAD Src\atten_ctrl.o
LOAD Src\eeprom.o
LOAD Src\main.o
LOAD Src\sth30_crc.o
LOAD Src\stm32f2xx_hal_msp.o
LOAD Src\stm32f2xx_it.o
LOAD Src\system_stm32f2xx.o
LOAD startup\startup_stm32f207xx.o
                0x00000080                malloc_getpagesize_P = 0x80
START GROUP
LOAD c:/program files (x86)/atollic/truestudio for stm32 9.2.0/armtools/bin/../lib/gcc/arm-atollic-eabi/6.3.1/../../../../arm-atollic-eabi/lib/armv7-m\libc_nano.a
LOAD c:/program files (x86)/atollic/truestudio for stm32 9.2.0/armtools/bin/../lib/gcc/arm-atollic-eabi/6.3.1/../../../../arm-atollic-eabi/lib/armv7-m\libm.a
END GROUP
START GROUP
LOAD c:/program files (x86)/atollic/truestudio for stm32 9.2.0/armtools/bin/../lib/gcc/arm-atollic-eabi/6.3.1/armv7-m\libgcc.a
LOAD c:/program files (x86)/atollic/truestudio for stm32 9.2.0/armtools/bin/../lib/gcc/arm-atollic-eabi/6.3.1/../../../../arm-atollic-eabi/lib/armv7-m\libc_nano.a
END GROUP
START GROUP
LOAD c:/program files (x86)/atollic/truestudio for stm32 9.2.0/armtools/bin/../lib/gcc/arm-atollic-eabi/6.3.1/armv7-m\libgcc.a
LOAD c:/program files (x86)/atollic/truestudio for stm32 9.2.0/armtools/bin/../lib/gcc/arm-atollic-eabi/6.3.1/../../../../arm-atollic-eabi/lib/armv7-m\libc_nano.a
LOAD c:/program files (x86)/atollic/truestudio for stm32 9.2.0/armtools/bin/../lib/gcc/arm-atollic-eabi/6.3.1/../../../../arm-atollic-eabi/lib/armv7-m\libnosys.a
END GROUP
START GROUP
LOAD c:/program files (x86)/atollic/truestudio for stm32 9.2.0/armtools/bin/../lib/gcc/arm-atollic-eabi/6.3.1/armv7-m\libgcc.a
LOAD c:/program files (x86)/atollic/truestudio for stm32 9.2.0/armtools/bin/../lib/gcc/arm-atollic-eabi/6.3.1/../../../../arm-atollic-eabi/lib/armv7-m\libc_nano.a
LOAD c:/program files (x86)/atollic/truestudio for stm32 9.2.0/armtools/bin/../lib/gcc/arm-atollic-eabi/6.3.1/../../../../arm-atollic-eabi/lib/armv7-m\libnosys.a
END GROUP
LOAD c:/program files (x86)/atollic/truestudio for stm32 9.2.0/armtools/bin/../lib/gcc/arm-atollic-eabi/6.3.1/armv7-m/crtend.o
LOAD c:/program files (x86)/atollic/truestudio for stm32 9.2.0/armtools/bin/../lib/gcc/arm-atollic-eabi/6.3.1/armv7-m/crtn.o
                0x20020000                _estack = 0x20020000
                0x00000200                _Min_Heap_Size = 0x200
                0x00000400                _Min_Stack_Size = 0x400

.isr_vector     0x08000000      0x184
                0x08000000                . = ALIGN (0x4)
 *(.isr_vector)
 .isr_vector    0x08000000      0x184 startup\startup_stm32f207xx.o
                0x08000000                g_pfnVectors
                0x08000184                . = ALIGN (0x4)

.text           0x08000184     0x5fe4
                0x08000184                . = ALIGN (0x4)
 *(.text)
 .text          0x08000184       0x40 c:/program files (x86)/atollic/truestudio for stm32 9.2.0/armtools/bin/../lib/gcc/arm-atollic-eabi/6.3.1/armv7-m/crtbegin.o
 .text          0x080001c4       0x30 c:/program files (x86)/atollic/truestudio for stm32 9.2.0/armtools/bin/../lib/gcc/arm-atollic-eabi/6.3.1/armv7-m\libgcc.a(_aeabi_uldivmod.o)
                0x080001c4                __aeabi_uldivmod
 .text          0x080001f4      0x2dc c:/program files (x86)/atollic/truestudio for stm32 9.2.0/armtools/bin/../lib/gcc/arm-atollic-eabi/6.3.1/armv7-m\libgcc.a(_udivmoddi4.o)
                0x080001f4                __udivmoddi4
 .text          0x080004d0        0x4 c:/program files (x86)/atollic/truestudio for stm32 9.2.0/armtools/bin/../lib/gcc/arm-atollic-eabi/6.3.1/armv7-m\libgcc.a(_dvmd_tls.o)
                0x080004d0                __aeabi_idiv0
                0x080004d0                __aeabi_ldiv0
 *(.text*)
 .text.HAL_InitTick
                0x080004d4       0x28 Drivers\STM32F2xx_HAL_Driver\Src\stm32f2xx_hal.o
                0x080004d4                HAL_InitTick
 .text.HAL_Init
                0x080004fc       0x34 Drivers\STM32F2xx_HAL_Driver\Src\stm32f2xx_hal.o
                0x080004fc                HAL_Init
 .text.HAL_IncTick
                0x08000530       0x10 Drivers\STM32F2xx_HAL_Driver\Src\stm32f2xx_hal.o
                0x08000530                HAL_IncTick
 .text.HAL_GetTick
                0x08000540        0xc Drivers\STM32F2xx_HAL_Driver\Src\stm32f2xx_hal.o
                0x08000540                HAL_GetTick
 .text.HAL_Delay
                0x0800054c       0x20 Drivers\STM32F2xx_HAL_Driver\Src\stm32f2xx_hal.o
                0x0800054c                HAL_Delay
 .text.HAL_NVIC_SetPriorityGrouping
                0x0800056c       0x24 Drivers\STM32F2xx_HAL_Driver\Src\stm32f2xx_hal_cortex.o
                0x0800056c                HAL_NVIC_SetPriorityGrouping
 .text.HAL_NVIC_SetPriority
                0x08000590       0x68 Drivers\STM32F2xx_HAL_Driver\Src\stm32f2xx_hal_cortex.o
                0x08000590                HAL_NVIC_SetPriority
 .text.HAL_NVIC_EnableIRQ
                0x080005f8       0x18 Drivers\STM32F2xx_HAL_Driver\Src\stm32f2xx_hal_cortex.o
                0x080005f8                HAL_NVIC_EnableIRQ
 .text.HAL_SYSTICK_Config
                0x08000610       0x2c Drivers\STM32F2xx_HAL_Driver\Src\stm32f2xx_hal_cortex.o
                0x08000610                HAL_SYSTICK_Config
 .text.HAL_DMA_Abort_IT
                0x0800063c       0x24 Drivers\STM32F2xx_HAL_Driver\Src\stm32f2xx_hal_dma.o
                0x0800063c                HAL_DMA_Abort_IT
 .text.HAL_GPIO_Init
                0x08000660      0x1cc Drivers\STM32F2xx_HAL_Driver\Src\stm32f2xx_hal_gpio.o
                0x08000660                HAL_GPIO_Init
 .text.HAL_GPIO_WritePin
                0x0800082c        0xa Drivers\STM32F2xx_HAL_Driver\Src\stm32f2xx_hal_gpio.o
                0x0800082c                HAL_GPIO_WritePin
 .text.HAL_GPIO_TogglePin
                0x08000836        0x8 Drivers\STM32F2xx_HAL_Driver\Src\stm32f2xx_hal_gpio.o
                0x08000836                HAL_GPIO_TogglePin
 .text.I2C_IsAcknowledgeFailed
                0x0800083e       0x2a Drivers\STM32F2xx_HAL_Driver\Src\stm32f2xx_hal_i2c.o
 .text.I2C_WaitOnMasterAddressFlagUntilTimeout
                0x08000868       0x80 Drivers\STM32F2xx_HAL_Driver\Src\stm32f2xx_hal_i2c.o
 .text.I2C_WaitOnFlagUntilTimeout
                0x080008e8       0x5c Drivers\STM32F2xx_HAL_Driver\Src\stm32f2xx_hal_i2c.o
 .text.I2C_WaitOnTXEFlagUntilTimeout
                0x08000944       0x4c Drivers\STM32F2xx_HAL_Driver\Src\stm32f2xx_hal_i2c.o
 .text.I2C_RequestMemoryWrite
                0x08000990       0xa4 Drivers\STM32F2xx_HAL_Driver\Src\stm32f2xx_hal_i2c.o
 .text.I2C_RequestMemoryRead
                0x08000a34       0xf4 Drivers\STM32F2xx_HAL_Driver\Src\stm32f2xx_hal_i2c.o
 .text.I2C_WaitOnRXNEFlagUntilTimeout
                0x08000b28       0x5a Drivers\STM32F2xx_HAL_Driver\Src\stm32f2xx_hal_i2c.o
 .text.I2C_WaitOnBTFFlagUntilTimeout
                0x08000b82       0x4c Drivers\STM32F2xx_HAL_Driver\Src\stm32f2xx_hal_i2c.o
 *fill*         0x08000bce        0x2 
 .text.HAL_I2C_Init
                0x08000bd0       0xdc Drivers\STM32F2xx_HAL_Driver\Src\stm32f2xx_hal_i2c.o
                0x08000bd0                HAL_I2C_Init
 .text.HAL_I2C_Mem_Write
                0x08000cac      0x12c Drivers\STM32F2xx_HAL_Driver\Src\stm32f2xx_hal_i2c.o
                0x08000cac                HAL_I2C_Mem_Write
 .text.HAL_I2C_Mem_Read
                0x08000dd8      0x224 Drivers\STM32F2xx_HAL_Driver\Src\stm32f2xx_hal_i2c.o
                0x08000dd8                HAL_I2C_Mem_Read
 .text.HAL_RCC_OscConfig
                0x08000ffc      0x2dc Drivers\STM32F2xx_HAL_Driver\Src\stm32f2xx_hal_rcc.o
                0x08000ffc                HAL_RCC_OscConfig
 .text.HAL_RCC_GetSysClockFreq
                0x080012d8       0x5c Drivers\STM32F2xx_HAL_Driver\Src\stm32f2xx_hal_rcc.o
                0x080012d8                HAL_RCC_GetSysClockFreq
 .text.HAL_RCC_ClockConfig
                0x08001334      0x13c Drivers\STM32F2xx_HAL_Driver\Src\stm32f2xx_hal_rcc.o
                0x08001334                HAL_RCC_ClockConfig
 .text.HAL_RCC_GetPCLK1Freq
                0x08001470       0x30 Drivers\STM32F2xx_HAL_Driver\Src\stm32f2xx_hal_rcc.o
                0x08001470                HAL_RCC_GetPCLK1Freq
 .text.HAL_RCC_GetPCLK2Freq
                0x080014a0       0x30 Drivers\STM32F2xx_HAL_Driver\Src\stm32f2xx_hal_rcc.o
                0x080014a0                HAL_RCC_GetPCLK2Freq
 .text.HAL_TIM_Base_Start_IT
                0x080014d0       0x16 Drivers\STM32F2xx_HAL_Driver\Src\stm32f2xx_hal_tim.o
                0x080014d0                HAL_TIM_Base_Start_IT
 .text.HAL_TIM_OC_DelayElapsedCallback
                0x080014e6        0x2 Drivers\STM32F2xx_HAL_Driver\Src\stm32f2xx_hal_tim.o
                0x080014e6                HAL_TIM_OC_DelayElapsedCallback
 .text.HAL_TIM_IC_CaptureCallback
                0x080014e8        0x2 Drivers\STM32F2xx_HAL_Driver\Src\stm32f2xx_hal_tim.o
                0x080014e8                HAL_TIM_IC_CaptureCallback
 .text.HAL_TIM_PWM_PulseFinishedCallback
                0x080014ea        0x2 Drivers\STM32F2xx_HAL_Driver\Src\stm32f2xx_hal_tim.o
                0x080014ea                HAL_TIM_PWM_PulseFinishedCallback
 .text.HAL_TIM_TriggerCallback
                0x080014ec        0x2 Drivers\STM32F2xx_HAL_Driver\Src\stm32f2xx_hal_tim.o
                0x080014ec                HAL_TIM_TriggerCallback
 .text.HAL_TIM_IRQHandler
                0x080014ee      0x144 Drivers\STM32F2xx_HAL_Driver\Src\stm32f2xx_hal_tim.o
                0x080014ee                HAL_TIM_IRQHandler
 *fill*         0x08001632        0x2 
 .text.TIM_Base_SetConfig
                0x08001634       0xd0 Drivers\STM32F2xx_HAL_Driver\Src\stm32f2xx_hal_tim.o
                0x08001634                TIM_Base_SetConfig
 .text.HAL_TIM_Base_Init
                0x08001704       0x34 Drivers\STM32F2xx_HAL_Driver\Src\stm32f2xx_hal_tim.o
                0x08001704                HAL_TIM_Base_Init
 .text.HAL_TIMEx_MasterConfigSynchronization
                0x08001738       0x44 Drivers\STM32F2xx_HAL_Driver\Src\stm32f2xx_hal_tim_ex.o
                0x08001738                HAL_TIMEx_MasterConfigSynchronization
 .text.HAL_TIMEx_CommutationCallback
                0x0800177c        0x2 Drivers\STM32F2xx_HAL_Driver\Src\stm32f2xx_hal_tim_ex.o
                0x0800177c                HAL_TIMEx_CommutationCallback
 .text.HAL_TIMEx_BreakCallback
                0x0800177e        0x2 Drivers\STM32F2xx_HAL_Driver\Src\stm32f2xx_hal_tim_ex.o
                0x0800177e                HAL_TIMEx_BreakCallback
 .text.UART_EndRxTransfer
                0x08001780       0x1a Drivers\STM32F2xx_HAL_Driver\Src\stm32f2xx_hal_uart.o
 *fill*         0x0800179a        0x2 
 .text.UART_SetConfig
                0x0800179c      0x234 Drivers\STM32F2xx_HAL_Driver\Src\stm32f2xx_hal_uart.o
 .text.UART_WaitOnFlagUntilTimeout.constprop.3
                0x080019d0       0x50 Drivers\STM32F2xx_HAL_Driver\Src\stm32f2xx_hal_uart.o
 .text.HAL_UART_Init
                0x08001a20       0x5c Drivers\STM32F2xx_HAL_Driver\Src\stm32f2xx_hal_uart.o
                0x08001a20                HAL_UART_Init
 .text.HAL_UART_Transmit
                0x08001a7c       0xb8 Drivers\STM32F2xx_HAL_Driver\Src\stm32f2xx_hal_uart.o
                0x08001a7c                HAL_UART_Transmit
 .text.HAL_UART_Receive_IT
                0x08001b34       0x46 Drivers\STM32F2xx_HAL_Driver\Src\stm32f2xx_hal_uart.o
                0x08001b34                HAL_UART_Receive_IT
 .text.HAL_UART_TxCpltCallback
                0x08001b7a        0x2 Drivers\STM32F2xx_HAL_Driver\Src\stm32f2xx_hal_uart.o
                0x08001b7a                HAL_UART_TxCpltCallback
 .text.UART_Receive_IT
                0x08001b7c       0x74 Drivers\STM32F2xx_HAL_Driver\Src\stm32f2xx_hal_uart.o
 .text.HAL_UART_ErrorCallback
                0x08001bf0        0x2 Drivers\STM32F2xx_HAL_Driver\Src\stm32f2xx_hal_uart.o
                0x08001bf0                HAL_UART_ErrorCallback
 *fill*         0x08001bf2        0x2 
 .text.HAL_UART_IRQHandler
                0x08001bf4      0x140 Drivers\STM32F2xx_HAL_Driver\Src\stm32f2xx_hal_uart.o
                0x08001bf4                HAL_UART_IRQHandler
 .text.UART_DMAAbortOnError
                0x08001d34       0x10 Drivers\STM32F2xx_HAL_Driver\Src\stm32f2xx_hal_uart.o
 .text.QPC6614_atten_ctrl
                0x08001d44       0x94 Src\atten_ctrl.o
                0x08001d44                QPC6614_atten_ctrl
 .text.ADRF5720_atten_ctrl
                0x08001dd8       0xa4 Src\atten_ctrl.o
                0x08001dd8                ADRF5720_atten_ctrl
 .text.HMC939_atten_ctrl
                0x08001e7c       0xa4 Src\atten_ctrl.o
                0x08001e7c                HMC939_atten_ctrl
 .text.Uart_Data_Send
                0x08001f20       0x10 Src\atten_ctrl.o
                0x08001f20                Uart_Data_Send
 .text.Atten_Table_Read.constprop.0
                0x08001f30       0x4a Src\atten_ctrl.o
 *fill*         0x08001f7a        0x2 
 .text.Atten_Offset_QPC6614
                0x08001f7c      0x1f0 Src\atten_ctrl.o
                0x08001f7c                Atten_Offset_QPC6614
 .text.Atten_Offset_ADRF5720
                0x0800216c      0x1f0 Src\atten_ctrl.o
                0x0800216c                Atten_Offset_ADRF5720
 .text.Atten_Offset_HMC939
                0x0800235c      0x10c Src\atten_ctrl.o
                0x0800235c                Atten_Offset_HMC939
 .text.Atten_Operate
                0x08002468      0xe50 Src\atten_ctrl.o
                0x08002468                Atten_Operate
 .text.Atten_Operate_Mem_RW
                0x080032b8     0x1378 Src\atten_ctrl.o
                0x080032b8                Atten_Operate_Mem_RW
 .text.EEPROM_IM24CM01P_write
                0x08004630       0x28 Src\eeprom.o
                0x08004630                EEPROM_IM24CM01P_write
 .text.EEPROM_IM24CM01P_Read
                0x08004658       0x28 Src\eeprom.o
                0x08004658                EEPROM_IM24CM01P_Read
 .text.EEPROM_IM24CM01P_Init
                0x08004680      0x2f4 Src\eeprom.o
                0x08004680                EEPROM_IM24CM01P_Init
 .text._write   0x08004974       0x14 Src\main.o
                0x08004974                _write
 .text.HAL_TIM_PeriodElapsedCallback
                0x08004988       0x4c Src\main.o
                0x08004988                HAL_TIM_PeriodElapsedCallback
 .text.HAL_UART_RxCpltCallback
                0x080049d4       0x40 Src\main.o
                0x080049d4                HAL_UART_RxCpltCallback
 .text.SystemClock_Config
                0x08004a14       0x48 Src\main.o
                0x08004a14                SystemClock_Config
 .text.startup.main
                0x08004a5c      0x32c Src\main.o
                0x08004a5c                main
 .text.STH30_CreateCrc
                0x08004d88       0x36 Src\sth30_crc.o
                0x08004d88                STH30_CreateCrc
 .text.STH30_CheckCrc
                0x08004dbe       0x3a Src\sth30_crc.o
                0x08004dbe                STH30_CheckCrc
 .text.HAL_MspInit
                0x08004df8       0x38 Src\stm32f2xx_hal_msp.o
                0x08004df8                HAL_MspInit
 .text.HAL_I2C_MspInit
                0x08004e30       0xb0 Src\stm32f2xx_hal_msp.o
                0x08004e30                HAL_I2C_MspInit
 .text.HAL_TIM_Base_MspInit
                0x08004ee0       0x30 Src\stm32f2xx_hal_msp.o
                0x08004ee0                HAL_TIM_Base_MspInit
 .text.HAL_UART_MspInit
                0x08004f10       0x70 Src\stm32f2xx_hal_msp.o
                0x08004f10                HAL_UART_MspInit
 .text.NMI_Handler
                0x08004f80        0x2 Src\stm32f2xx_it.o
                0x08004f80                NMI_Handler
 .text.HardFault_Handler
                0x08004f82        0x2 Src\stm32f2xx_it.o
                0x08004f82                HardFault_Handler
 .text.MemManage_Handler
                0x08004f84        0x2 Src\stm32f2xx_it.o
                0x08004f84                MemManage_Handler
 .text.BusFault_Handler
                0x08004f86        0x2 Src\stm32f2xx_it.o
                0x08004f86                BusFault_Handler
 .text.UsageFault_Handler
                0x08004f88        0x2 Src\stm32f2xx_it.o
                0x08004f88                UsageFault_Handler
 .text.SVC_Handler
                0x08004f8a        0x2 Src\stm32f2xx_it.o
                0x08004f8a                SVC_Handler
 .text.DebugMon_Handler
                0x08004f8c        0x2 Src\stm32f2xx_it.o
                0x08004f8c                DebugMon_Handler
 .text.PendSV_Handler
                0x08004f8e        0x2 Src\stm32f2xx_it.o
                0x08004f8e                PendSV_Handler
 .text.SysTick_Handler
                0x08004f90        0x4 Src\stm32f2xx_it.o
                0x08004f90                SysTick_Handler
 .text.USART1_IRQHandler
                0x08004f94        0xc Src\stm32f2xx_it.o
                0x08004f94                USART1_IRQHandler
 .text.TIM6_DAC_IRQHandler
                0x08004fa0        0xc Src\stm32f2xx_it.o
                0x08004fa0                TIM6_DAC_IRQHandler
 .text.SystemInit
                0x08004fac       0x40 Src\system_stm32f2xx.o
                0x08004fac                SystemInit
 .text.Reset_Handler
                0x08004fec       0x50 startup\startup_stm32f207xx.o
                0x08004fec                Reset_Handler
 .text.Default_Handler
                0x0800503c        0x2 startup\startup_stm32f207xx.o
                0x0800503c                RTC_Alarm_IRQHandler
                0x0800503c                HASH_RNG_IRQHandler
                0x0800503c                EXTI2_IRQHandler
                0x0800503c                TIM8_CC_IRQHandler
                0x0800503c                TIM1_CC_IRQHandler
                0x0800503c                DMA2_Stream5_IRQHandler
                0x0800503c                DMA1_Stream5_IRQHandler
                0x0800503c                PVD_IRQHandler
                0x0800503c                SDIO_IRQHandler
                0x0800503c                TAMP_STAMP_IRQHandler
                0x0800503c                CAN2_RX1_IRQHandler
                0x0800503c                EXTI3_IRQHandler
                0x0800503c                TIM8_TRG_COM_TIM14_IRQHandler
                0x0800503c                TIM1_UP_TIM10_IRQHandler
                0x0800503c                TIM8_UP_TIM13_IRQHandler
                0x0800503c                I2C3_ER_IRQHandler
                0x0800503c                EXTI0_IRQHandler
                0x0800503c                I2C2_EV_IRQHandler
                0x0800503c                DMA1_Stream2_IRQHandler
                0x0800503c                CAN1_RX0_IRQHandler
                0x0800503c                OTG_HS_WKUP_IRQHandler
                0x0800503c                CAN2_SCE_IRQHandler
                0x0800503c                DMA2_Stream2_IRQHandler
                0x0800503c                SPI1_IRQHandler
                0x0800503c                TIM1_BRK_TIM9_IRQHandler
                0x0800503c                DCMI_IRQHandler
                0x0800503c                CAN2_RX0_IRQHandler
                0x0800503c                DMA2_Stream3_IRQHandler
                0x0800503c                USART6_IRQHandler
                0x0800503c                USART3_IRQHandler
                0x0800503c                CAN1_RX1_IRQHandler
                0x0800503c                UART5_IRQHandler
                0x0800503c                DMA2_Stream0_IRQHandler
                0x0800503c                TIM4_IRQHandler
                0x0800503c                I2C1_EV_IRQHandler
                0x0800503c                DMA1_Stream6_IRQHandler
                0x0800503c                DMA1_Stream1_IRQHandler
                0x0800503c                UART4_IRQHandler
                0x0800503c                TIM3_IRQHandler
                0x0800503c                RCC_IRQHandler
                0x0800503c                TIM8_BRK_TIM12_IRQHandler
                0x0800503c                Default_Handler
                0x0800503c                EXTI15_10_IRQHandler
                0x0800503c                ADC_IRQHandler
                0x0800503c                DMA1_Stream7_IRQHandler
                0x0800503c                TIM7_IRQHandler
                0x0800503c                CAN2_TX_IRQHandler
                0x0800503c                TIM5_IRQHandler
                0x0800503c                DMA2_Stream7_IRQHandler
                0x0800503c                I2C3_EV_IRQHandler
                0x0800503c                EXTI9_5_IRQHandler
                0x0800503c                RTC_WKUP_IRQHandler
                0x0800503c                ETH_WKUP_IRQHandler
                0x0800503c                SPI2_IRQHandler
                0x0800503c                OTG_HS_EP1_IN_IRQHandler
                0x0800503c                DMA1_Stream0_IRQHandler
                0x0800503c                CAN1_TX_IRQHandler
                0x0800503c                EXTI4_IRQHandler
                0x0800503c                FSMC_IRQHandler
                0x0800503c                ETH_IRQHandler
                0x0800503c                OTG_HS_EP1_OUT_IRQHandler
                0x0800503c                WWDG_IRQHandler
                0x0800503c                TIM2_IRQHandler
                0x0800503c                OTG_FS_WKUP_IRQHandler
                0x0800503c                TIM1_TRG_COM_TIM11_IRQHandler
                0x0800503c                OTG_HS_IRQHandler
                0x0800503c                EXTI1_IRQHandler
                0x0800503c                USART2_IRQHandler
                0x0800503c                I2C2_ER_IRQHandler
                0x0800503c                DMA2_Stream1_IRQHandler
                0x0800503c                CAN1_SCE_IRQHandler
                0x0800503c                FLASH_IRQHandler
                0x0800503c                DMA2_Stream4_IRQHandler
                0x0800503c                OTG_FS_IRQHandler
                0x0800503c                SPI3_IRQHandler
                0x0800503c                DMA1_Stream4_IRQHandler
                0x0800503c                I2C1_ER_IRQHandler
                0x0800503c                DMA2_Stream6_IRQHandler
                0x0800503c                DMA1_Stream3_IRQHandler
 *fill*         0x0800503e        0x2 
 .text.__libc_init_array
                0x08005040       0x48 c:/program files (x86)/atollic/truestudio for stm32 9.2.0/armtools/bin/../lib/gcc/arm-atollic-eabi/6.3.1/../../../../arm-atollic-eabi/lib/armv7-m\libc_nano.a(lib_a-init.o)
                0x08005040                __libc_init_array
 .text.memset   0x08005088       0x10 c:/program files (x86)/atollic/truestudio for stm32 9.2.0/armtools/bin/../lib/gcc/arm-atollic-eabi/6.3.1/../../../../arm-atollic-eabi/lib/armv7-m\libc_nano.a(lib_a-memset.o)
                0x08005088                memset
 .text.printf   0x08005098       0x30 c:/program files (x86)/atollic/truestudio for stm32 9.2.0/armtools/bin/../lib/gcc/arm-atollic-eabi/6.3.1/../../../../arm-atollic-eabi/lib/armv7-m\libc_nano.a(lib_a-printf.o)
                0x08005098                iprintf
                0x08005098                printf
 .text._puts_r  0x080050c8       0xb8 c:/program files (x86)/atollic/truestudio for stm32 9.2.0/armtools/bin/../lib/gcc/arm-atollic-eabi/6.3.1/../../../../arm-atollic-eabi/lib/armv7-m\libc_nano.a(lib_a-puts.o)
                0x080050c8                _puts_r
 .text.puts     0x08005180       0x10 c:/program files (x86)/atollic/truestudio for stm32 9.2.0/armtools/bin/../lib/gcc/arm-atollic-eabi/6.3.1/../../../../arm-atollic-eabi/lib/armv7-m\libc_nano.a(lib_a-puts.o)
                0x08005180                puts
 .text.setbuf   0x08005190       0x10 c:/program files (x86)/atollic/truestudio for stm32 9.2.0/armtools/bin/../lib/gcc/arm-atollic-eabi/6.3.1/../../../../arm-atollic-eabi/lib/armv7-m\libc_nano.a(lib_a-setbuf.o)
                0x08005190                setbuf
 .text.setvbuf  0x080051a0      0x15c c:/program files (x86)/atollic/truestudio for stm32 9.2.0/armtools/bin/../lib/gcc/arm-atollic-eabi/6.3.1/../../../../arm-atollic-eabi/lib/armv7-m\libc_nano.a(lib_a-setvbuf.o)
                0x080051a0                setvbuf
 .text.__swbuf_r
                0x080052fc       0xa4 c:/program files (x86)/atollic/truestudio for stm32 9.2.0/armtools/bin/../lib/gcc/arm-atollic-eabi/6.3.1/../../../../arm-atollic-eabi/lib/armv7-m\libc_nano.a(lib_a-wbuf.o)
                0x080052fc                __swbuf_r
 .text.__swsetup_r
                0x080053a0       0xdc c:/program files (x86)/atollic/truestudio for stm32 9.2.0/armtools/bin/../lib/gcc/arm-atollic-eabi/6.3.1/../../../../arm-atollic-eabi/lib/armv7-m\libc_nano.a(lib_a-wsetup.o)
                0x080053a0                __swsetup_r
 .text.__sflush_r
                0x0800547c      0x110 c:/program files (x86)/atollic/truestudio for stm32 9.2.0/armtools/bin/../lib/gcc/arm-atollic-eabi/6.3.1/../../../../arm-atollic-eabi/lib/armv7-m\libc_nano.a(lib_a-fflush.o)
                0x0800547c                __sflush_r
 .text._fflush_r
                0x0800558c       0x54 c:/program files (x86)/atollic/truestudio for stm32 9.2.0/armtools/bin/../lib/gcc/arm-atollic-eabi/6.3.1/../../../../arm-atollic-eabi/lib/armv7-m\libc_nano.a(lib_a-fflush.o)
                0x0800558c                _fflush_r
 .text._cleanup_r
                0x080055e0        0xc c:/program files (x86)/atollic/truestudio for stm32 9.2.0/armtools/bin/../lib/gcc/arm-atollic-eabi/6.3.1/../../../../arm-atollic-eabi/lib/armv7-m\libc_nano.a(lib_a-findfp.o)
                0x080055e0                _cleanup_r
 .text.std.isra.0
                0x080055ec       0x48 c:/program files (x86)/atollic/truestudio for stm32 9.2.0/armtools/bin/../lib/gcc/arm-atollic-eabi/6.3.1/../../../../arm-atollic-eabi/lib/armv7-m\libc_nano.a(lib_a-findfp.o)
 .text.__sfmoreglue
                0x08005634       0x2c c:/program files (x86)/atollic/truestudio for stm32 9.2.0/armtools/bin/../lib/gcc/arm-atollic-eabi/6.3.1/../../../../arm-atollic-eabi/lib/armv7-m\libc_nano.a(lib_a-findfp.o)
                0x08005634                __sfmoreglue
 .text.__sinit  0x08005660       0x60 c:/program files (x86)/atollic/truestudio for stm32 9.2.0/armtools/bin/../lib/gcc/arm-atollic-eabi/6.3.1/../../../../arm-atollic-eabi/lib/armv7-m\libc_nano.a(lib_a-findfp.o)
                0x08005660                __sinit
 .text.__sfp    0x080056c0       0x78 c:/program files (x86)/atollic/truestudio for stm32 9.2.0/armtools/bin/../lib/gcc/arm-atollic-eabi/6.3.1/../../../../arm-atollic-eabi/lib/armv7-m\libc_nano.a(lib_a-findfp.o)
                0x080056c0                __sfp
 .text._fwalk_reent
                0x08005738       0x3c c:/program files (x86)/atollic/truestudio for stm32 9.2.0/armtools/bin/../lib/gcc/arm-atollic-eabi/6.3.1/../../../../arm-atollic-eabi/lib/armv7-m\libc_nano.a(lib_a-fwalk.o)
                0x08005738                _fwalk_reent
 .text.__swhatbuf_r
                0x08005774       0x48 c:/program files (x86)/atollic/truestudio for stm32 9.2.0/armtools/bin/../lib/gcc/arm-atollic-eabi/6.3.1/../../../../arm-atollic-eabi/lib/armv7-m\libc_nano.a(lib_a-makebuf.o)
                0x08005774                __swhatbuf_r
 .text.__smakebuf_r
                0x080057bc       0x80 c:/program files (x86)/atollic/truestudio for stm32 9.2.0/armtools/bin/../lib/gcc/arm-atollic-eabi/6.3.1/../../../../arm-atollic-eabi/lib/armv7-m\libc_nano.a(lib_a-makebuf.o)
                0x080057bc                __smakebuf_r
 .text.malloc   0x0800583c       0x10 c:/program files (x86)/atollic/truestudio for stm32 9.2.0/armtools/bin/../lib/gcc/arm-atollic-eabi/6.3.1/../../../../arm-atollic-eabi/lib/armv7-m\libc_nano.a(lib_a-malloc.o)
                0x0800583c                malloc
 .text._free_r  0x0800584c       0x98 c:/program files (x86)/atollic/truestudio for stm32 9.2.0/armtools/bin/../lib/gcc/arm-atollic-eabi/6.3.1/../../../../arm-atollic-eabi/lib/armv7-m\libc_nano.a(lib_a-nano-freer.o)
                0x0800584c                _free_r
 .text._malloc_r
                0x080058e4       0xbc c:/program files (x86)/atollic/truestudio for stm32 9.2.0/armtools/bin/../lib/gcc/arm-atollic-eabi/6.3.1/../../../../arm-atollic-eabi/lib/armv7-m\libc_nano.a(lib_a-nano-mallocr.o)
                0x080058e4                _malloc_r
 .text.__sfputc_r
                0x080059a0       0x2c c:/program files (x86)/atollic/truestudio for stm32 9.2.0/armtools/bin/../lib/gcc/arm-atollic-eabi/6.3.1/../../../../arm-atollic-eabi/lib/armv7-m\libc_nano.a(lib_a-nano-vfprintf.o)
 .text.__sfputs_r
                0x080059cc       0x24 c:/program files (x86)/atollic/truestudio for stm32 9.2.0/armtools/bin/../lib/gcc/arm-atollic-eabi/6.3.1/../../../../arm-atollic-eabi/lib/armv7-m\libc_nano.a(lib_a-nano-vfprintf.o)
                0x080059cc                __sfputs_r
 .text._vfprintf_r
                0x080059f0      0x22c c:/program files (x86)/atollic/truestudio for stm32 9.2.0/armtools/bin/../lib/gcc/arm-atollic-eabi/6.3.1/../../../../arm-atollic-eabi/lib/armv7-m\libc_nano.a(lib_a-nano-vfprintf.o)
                0x080059f0                _vfprintf_r
                0x080059f0                _vfiprintf_r
 .text._printf_common
                0x08005c1c       0xee c:/program files (x86)/atollic/truestudio for stm32 9.2.0/armtools/bin/../lib/gcc/arm-atollic-eabi/6.3.1/../../../../arm-atollic-eabi/lib/armv7-m\libc_nano.a(lib_a-nano-vfprintf_i.o)
                0x08005c1c                _printf_common
 *fill*         0x08005d0a        0x2 
 .text._printf_i
                0x08005d0c      0x240 c:/program files (x86)/atollic/truestudio for stm32 9.2.0/armtools/bin/../lib/gcc/arm-atollic-eabi/6.3.1/../../../../arm-atollic-eabi/lib/armv7-m\libc_nano.a(lib_a-nano-vfprintf_i.o)
                0x08005d0c                _printf_i
 .text._sbrk_r  0x08005f4c       0x20 c:/program files (x86)/atollic/truestudio for stm32 9.2.0/armtools/bin/../lib/gcc/arm-atollic-eabi/6.3.1/../../../../arm-atollic-eabi/lib/armv7-m\libc_nano.a(lib_a-sbrkr.o)
                0x08005f4c                _sbrk_r
 .text.__sread  0x08005f6c       0x22 c:/program files (x86)/atollic/truestudio for stm32 9.2.0/armtools/bin/../lib/gcc/arm-atollic-eabi/6.3.1/../../../../arm-atollic-eabi/lib/armv7-m\libc_nano.a(lib_a-stdio.o)
                0x08005f6c                __sread
 .text.__swrite
                0x08005f8e       0x38 c:/program files (x86)/atollic/truestudio for stm32 9.2.0/armtools/bin/../lib/gcc/arm-atollic-eabi/6.3.1/../../../../arm-atollic-eabi/lib/armv7-m\libc_nano.a(lib_a-stdio.o)
                0x08005f8e                __swrite
 .text.__sseek  0x08005fc6       0x24 c:/program files (x86)/atollic/truestudio for stm32 9.2.0/armtools/bin/../lib/gcc/arm-atollic-eabi/6.3.1/../../../../arm-atollic-eabi/lib/armv7-m\libc_nano.a(lib_a-stdio.o)
                0x08005fc6                __sseek
 .text.__sclose
                0x08005fea        0x8 c:/program files (x86)/atollic/truestudio for stm32 9.2.0/armtools/bin/../lib/gcc/arm-atollic-eabi/6.3.1/../../../../arm-atollic-eabi/lib/armv7-m\libc_nano.a(lib_a-stdio.o)
                0x08005fea                __sclose
 *fill*         0x08005ff2        0x2 
 .text._write_r
                0x08005ff4       0x24 c:/program files (x86)/atollic/truestudio for stm32 9.2.0/armtools/bin/../lib/gcc/arm-atollic-eabi/6.3.1/../../../../arm-atollic-eabi/lib/armv7-m\libc_nano.a(lib_a-writer.o)
                0x08005ff4                _write_r
 .text._close_r
                0x08006018       0x20 c:/program files (x86)/atollic/truestudio for stm32 9.2.0/armtools/bin/../lib/gcc/arm-atollic-eabi/6.3.1/../../../../arm-atollic-eabi/lib/armv7-m\libc_nano.a(lib_a-closer.o)
                0x08006018                _close_r
 .text._fstat_r
                0x08006038       0x24 c:/program files (x86)/atollic/truestudio for stm32 9.2.0/armtools/bin/../lib/gcc/arm-atollic-eabi/6.3.1/../../../../arm-atollic-eabi/lib/armv7-m\libc_nano.a(lib_a-fstatr.o)
                0x08006038                _fstat_r
 .text._isatty_r
                0x0800605c       0x20 c:/program files (x86)/atollic/truestudio for stm32 9.2.0/armtools/bin/../lib/gcc/arm-atollic-eabi/6.3.1/../../../../arm-atollic-eabi/lib/armv7-m\libc_nano.a(lib_a-isattyr.o)
                0x0800605c                _isatty_r
 .text._lseek_r
                0x0800607c       0x24 c:/program files (x86)/atollic/truestudio for stm32 9.2.0/armtools/bin/../lib/gcc/arm-atollic-eabi/6.3.1/../../../../arm-atollic-eabi/lib/armv7-m\libc_nano.a(lib_a-lseekr.o)
                0x0800607c                _lseek_r
 .text.memchr   0x080060a0       0x1c c:/program files (x86)/atollic/truestudio for stm32 9.2.0/armtools/bin/../lib/gcc/arm-atollic-eabi/6.3.1/../../../../arm-atollic-eabi/lib/armv7-m\libc_nano.a(lib_a-memchr-stub.o)
                0x080060a0                memchr
 .text.__malloc_lock
                0x080060bc        0x2 c:/program files (x86)/atollic/truestudio for stm32 9.2.0/armtools/bin/../lib/gcc/arm-atollic-eabi/6.3.1/../../../../arm-atollic-eabi/lib/armv7-m\libc_nano.a(lib_a-mlock.o)
                0x080060bc                __malloc_lock
 .text.__malloc_unlock
                0x080060be        0x2 c:/program files (x86)/atollic/truestudio for stm32 9.2.0/armtools/bin/../lib/gcc/arm-atollic-eabi/6.3.1/../../../../arm-atollic-eabi/lib/armv7-m\libc_nano.a(lib_a-mlock.o)
                0x080060be                __malloc_unlock
 .text._read_r  0x080060c0       0x24 c:/program files (x86)/atollic/truestudio for stm32 9.2.0/armtools/bin/../lib/gcc/arm-atollic-eabi/6.3.1/../../../../arm-atollic-eabi/lib/armv7-m\libc_nano.a(lib_a-readr.o)
                0x080060c0                _read_r
 .text._close   0x080060e4       0x10 c:/program files (x86)/atollic/truestudio for stm32 9.2.0/armtools/bin/../lib/gcc/arm-atollic-eabi/6.3.1/../../../../arm-atollic-eabi/lib/armv7-m\libnosys.a(close.o)
                0x080060e4                _close
 .text._fstat   0x080060f4       0x10 c:/program files (x86)/atollic/truestudio for stm32 9.2.0/armtools/bin/../lib/gcc/arm-atollic-eabi/6.3.1/../../../../arm-atollic-eabi/lib/armv7-m\libnosys.a(fstat.o)
                0x080060f4                _fstat
 .text._isatty  0x08006104       0x10 c:/program files (x86)/atollic/truestudio for stm32 9.2.0/armtools/bin/../lib/gcc/arm-atollic-eabi/6.3.1/../../../../arm-atollic-eabi/lib/armv7-m\libnosys.a(isatty.o)
                0x08006104                _isatty
 .text._lseek   0x08006114       0x10 c:/program files (x86)/atollic/truestudio for stm32 9.2.0/armtools/bin/../lib/gcc/arm-atollic-eabi/6.3.1/../../../../arm-atollic-eabi/lib/armv7-m\libnosys.a(lseek.o)
                0x08006114                _lseek
 .text._read    0x08006124       0x10 c:/program files (x86)/atollic/truestudio for stm32 9.2.0/armtools/bin/../lib/gcc/arm-atollic-eabi/6.3.1/../../../../arm-atollic-eabi/lib/armv7-m\libnosys.a(read.o)
                0x08006124                _read
 .text._sbrk    0x08006134       0x1c c:/program files (x86)/atollic/truestudio for stm32 9.2.0/armtools/bin/../lib/gcc/arm-atollic-eabi/6.3.1/../../../../arm-atollic-eabi/lib/armv7-m\libnosys.a(sbrk.o)
                0x08006134                _sbrk
 *(.glue_7)
 .glue_7        0x08006150        0x0 linker stubs
 *(.glue_7t)
 .glue_7t       0x08006150        0x0 linker stubs
 *(.eh_frame)
 .eh_frame      0x08006150        0x0 c:/program files (x86)/atollic/truestudio for stm32 9.2.0/armtools/bin/../lib/gcc/arm-atollic-eabi/6.3.1/armv7-m/crtbegin.o
 *(.init)
 .init          0x08006150        0x4 c:/program files (x86)/atollic/truestudio for stm32 9.2.0/armtools/bin/../lib/gcc/arm-atollic-eabi/6.3.1/armv7-m/crti.o
                0x08006150                _init
 .init          0x08006154        0x8 c:/program files (x86)/atollic/truestudio for stm32 9.2.0/armtools/bin/../lib/gcc/arm-atollic-eabi/6.3.1/armv7-m/crtn.o
 *(.fini)
 .fini          0x0800615c        0x4 c:/program files (x86)/atollic/truestudio for stm32 9.2.0/armtools/bin/../lib/gcc/arm-atollic-eabi/6.3.1/armv7-m/crti.o
                0x0800615c                _fini
 .fini          0x08006160        0x8 c:/program files (x86)/atollic/truestudio for stm32 9.2.0/armtools/bin/../lib/gcc/arm-atollic-eabi/6.3.1/armv7-m/crtn.o
                0x08006168                . = ALIGN (0x4)
                0x08006168                _etext = .

.vfp11_veneer   0x08006168        0x0
 .vfp11_veneer  0x08006168        0x0 linker stubs

.v4_bx          0x08006168        0x0
 .v4_bx         0x08006168        0x0 linker stubs

.iplt           0x08006168        0x0
 .iplt          0x08006168        0x0 c:/program files (x86)/atollic/truestudio for stm32 9.2.0/armtools/bin/../lib/gcc/arm-atollic-eabi/6.3.1/armv7-m/crtbegin.o

.rodata         0x08006168      0x1e0
                0x08006168                . = ALIGN (0x4)
 *(.rodata)
 *(.rodata*)
 .rodata.Atten_Offset_QPC6614.str1.1
                0x08006168       0x10 Src\atten_ctrl.o
 .rodata.Atten_Operate.str1.1
                0x08006178        0xc Src\atten_ctrl.o
 .rodata.Atten_Operate_Mem_RW.str1.1
                0x08006184       0x27 Src\atten_ctrl.o
 .rodata.__func__.9078
                0x080061ab       0x15 Src\atten_ctrl.o
 .rodata.main.str1.1
                0x080061c0       0xd8 Src\main.o
                                 0xda (size before relaxing)
 .rodata.AHBPrescTable
                0x08006298       0x10 Src\system_stm32f2xx.o
                0x08006298                AHBPrescTable
 .rodata.APBPrescTable
                0x080062a8        0x8 Src\system_stm32f2xx.o
                0x080062a8                APBPrescTable
 .rodata._global_impure_ptr
                0x080062b0        0x4 c:/program files (x86)/atollic/truestudio for stm32 9.2.0/armtools/bin/../lib/gcc/arm-atollic-eabi/6.3.1/../../../../arm-atollic-eabi/lib/armv7-m\libc_nano.a(lib_a-impure.o)
                0x080062b0                _global_impure_ptr
 .rodata.__sf_fake_stderr
                0x080062b4       0x20 c:/program files (x86)/atollic/truestudio for stm32 9.2.0/armtools/bin/../lib/gcc/arm-atollic-eabi/6.3.1/../../../../arm-atollic-eabi/lib/armv7-m\libc_nano.a(lib_a-findfp.o)
                0x080062b4                __sf_fake_stderr
 .rodata.__sf_fake_stdin
                0x080062d4       0x20 c:/program files (x86)/atollic/truestudio for stm32 9.2.0/armtools/bin/../lib/gcc/arm-atollic-eabi/6.3.1/../../../../arm-atollic-eabi/lib/armv7-m\libc_nano.a(lib_a-findfp.o)
                0x080062d4                __sf_fake_stdin
 .rodata.__sf_fake_stdout
                0x080062f4       0x20 c:/program files (x86)/atollic/truestudio for stm32 9.2.0/armtools/bin/../lib/gcc/arm-atollic-eabi/6.3.1/../../../../arm-atollic-eabi/lib/armv7-m\libc_nano.a(lib_a-findfp.o)
                0x080062f4                __sf_fake_stdout
 .rodata._vfprintf_r.str1.1
                0x08006314       0x11 c:/program files (x86)/atollic/truestudio for stm32 9.2.0/armtools/bin/../lib/gcc/arm-atollic-eabi/6.3.1/../../../../arm-atollic-eabi/lib/armv7-m\libc_nano.a(lib_a-nano-vfprintf.o)
 .rodata._printf_i.str1.1
                0x08006325       0x22 c:/program files (x86)/atollic/truestudio for stm32 9.2.0/armtools/bin/../lib/gcc/arm-atollic-eabi/6.3.1/../../../../arm-atollic-eabi/lib/armv7-m\libc_nano.a(lib_a-nano-vfprintf_i.o)
                0x08006348                . = ALIGN (0x4)
 *fill*         0x08006347        0x1 

.ARM.extab
 *(.ARM.extab* .gnu.linkonce.armextab.*)

.ARM            0x08006348        0x8
                0x08006348                __exidx_start = .
 *(.ARM.exidx*)
 .ARM.exidx     0x08006348        0x8 c:/program files (x86)/atollic/truestudio for stm32 9.2.0/armtools/bin/../lib/gcc/arm-atollic-eabi/6.3.1/armv7-m\libgcc.a(_udivmoddi4.o)
                0x08006350                __exidx_end = .

.rel.dyn        0x08006350        0x0
 .rel.iplt      0x08006350        0x0 c:/program files (x86)/atollic/truestudio for stm32 9.2.0/armtools/bin/../lib/gcc/arm-atollic-eabi/6.3.1/armv7-m/crtbegin.o

.preinit_array  0x08006350        0x0
                0x08006350                PROVIDE (__preinit_array_start, .)
 *(.preinit_array*)
                0x08006350                PROVIDE (__preinit_array_end, .)

.init_array     0x08006350        0x4
                0x08006350                PROVIDE (__init_array_start, .)
 *(SORT(.init_array.*))
 *(.init_array*)
 .init_array    0x08006350        0x4 c:/program files (x86)/atollic/truestudio for stm32 9.2.0/armtools/bin/../lib/gcc/arm-atollic-eabi/6.3.1/armv7-m/crtbegin.o
                0x08006354                PROVIDE (__init_array_end, .)

.fini_array     0x08006354        0x4
                [!provide]                PROVIDE (__fini_array_start, .)
 *(SORT(.fini_array.*))
 *(.fini_array*)
 .fini_array    0x08006354        0x4 c:/program files (x86)/atollic/truestudio for stm32 9.2.0/armtools/bin/../lib/gcc/arm-atollic-eabi/6.3.1/armv7-m/crtbegin.o
                [!provide]                PROVIDE (__fini_array_end, .)
                0x08006358                _sidata = LOADADDR (.data)

.data           0x20000000       0x68 load address 0x08006358
                0x20000000                . = ALIGN (0x4)
                0x20000000                _sdata = .
 *(.data)
 *(.data*)
 .data.SystemCoreClock
                0x20000000        0x4 Src\system_stm32f2xx.o
                0x20000000                SystemCoreClock
 .data._impure_ptr
                0x20000004        0x4 c:/program files (x86)/atollic/truestudio for stm32 9.2.0/armtools/bin/../lib/gcc/arm-atollic-eabi/6.3.1/../../../../arm-atollic-eabi/lib/armv7-m\libc_nano.a(lib_a-impure.o)
                0x20000004                _impure_ptr
 .data.impure_data
                0x20000008       0x60 c:/program files (x86)/atollic/truestudio for stm32 9.2.0/armtools/bin/../lib/gcc/arm-atollic-eabi/6.3.1/../../../../arm-atollic-eabi/lib/armv7-m\libc_nano.a(lib_a-impure.o)
                0x20000068                . = ALIGN (0x4)
                0x20000068                _edata = .

.igot.plt       0x20000068        0x0 load address 0x080063c0
 .igot.plt      0x20000068        0x0 c:/program files (x86)/atollic/truestudio for stm32 9.2.0/armtools/bin/../lib/gcc/arm-atollic-eabi/6.3.1/armv7-m/crtbegin.o
                0x20000068                . = ALIGN (0x4)

.bss            0x20000068      0xc50 load address 0x080063c0
                0x20000068                _sbss = .
                0x20000068                __bss_start__ = _sbss
 *(.bss)
 .bss           0x20000068       0x1c c:/program files (x86)/atollic/truestudio for stm32 9.2.0/armtools/bin/../lib/gcc/arm-atollic-eabi/6.3.1/armv7-m/crtbegin.o
 *(.bss*)
 .bss.printf_if
                0x20000084        0x1 Src\atten_ctrl.o
                0x20000084                printf_if
 *fill*         0x20000085        0x3 
 .bss.LedTimerCnt
                0x20000088        0x4 Src\main.o
                0x20000088                LedTimerCnt
 .bss.UartTimerCnt
                0x2000008c        0x4 Src\main.o
                0x2000008c                UartTimerCnt
 .bss.buf       0x20000090       0x40 Src\main.o
                0x20000090                buf
 .bss.__malloc_free_list
                0x200000d0        0x4 c:/program files (x86)/atollic/truestudio for stm32 9.2.0/armtools/bin/../lib/gcc/arm-atollic-eabi/6.3.1/../../../../arm-atollic-eabi/lib/armv7-m\libc_nano.a(lib_a-nano-mallocr.o)
                0x200000d0                __malloc_free_list
 .bss.__malloc_sbrk_start
                0x200000d4        0x4 c:/program files (x86)/atollic/truestudio for stm32 9.2.0/armtools/bin/../lib/gcc/arm-atollic-eabi/6.3.1/../../../../arm-atollic-eabi/lib/armv7-m\libc_nano.a(lib_a-nano-mallocr.o)
                0x200000d4                __malloc_sbrk_start
 .bss.heap_end.4116
                0x200000d8        0x4 c:/program files (x86)/atollic/truestudio for stm32 9.2.0/armtools/bin/../lib/gcc/arm-atollic-eabi/6.3.1/../../../../arm-atollic-eabi/lib/armv7-m\libnosys.a(sbrk.o)
 *(COMMON)
 COMMON         0x200000dc        0x4 Drivers\STM32F2xx_HAL_Driver\Src\stm32f2xx_hal.o
                0x200000dc                uwTick
 COMMON         0x200000e0      0xab1 Src\atten_ctrl.o
                0x200000e0                ATT_B_EN_WIFI4_2_4Ghz_Table
                0x20000120                ATT_A_EN_30G3_29_29_5Ghz_Table
                0x20000160                ATT_B_EN_30G1_28_28_5Ghz_Table
                0x200001a0                ATT_A_EN_WIFI4_2_4Ghz_Table
                0x200001e0                ATT_A_EN_30G3_29_5_30Ghz_Table
                0x20000220                ATT_B_EN_WIFI3_5_8Ghz_Table
                0x20000260                ATT_B_EN_30G3_28_5_29Ghz_Table
                0x200002a0                ATT_A_EN_WIFI1_2_4Ghz_Table
                0x200002e0                ATT_B_EN_30G2_28_28_5Ghz_Table
                0x20000320                ATT_B_EN_WIFI4_5_8Ghz_Table
                0x20000360                ATT_A_EN_WIFI3_2_4Ghz_Table
                0x200003a0                ATT_B_EN_WIFI2_2_4Ghz_Table
                0x200003e0                ATT_B_EN_30G1_28_5_29Ghz_Table
                0x20000420                ATT_A_EN_30G2_28_5_29Ghz_Table
                0x20000460                ATT_B_EN_WIFI1_2_4Ghz_Table
                0x200004a0                ATT_A_EN_30G2_29_29_5Ghz_Table
                0x200004e0                ATT_B_EN_30G3_29_29_5Ghz_Table
                0x20000520                ATT_B_EN_30G2_28_5_29Ghz_Table
                0x20000560                ATT_A_EN_30G3_28_5_29Ghz_Table
                0x200005a0                ATT_B_EN_WIFI2_5_8Ghz_Table
                0x200005e0                ATT_A_EN_30G1_28_28_5Ghz_Table
                0x20000620                ATT_B_EN_30G1_29_29_5Ghz_Table
                0x20000660                ATT_B_EN_30G2_29_29_5Ghz_Table
                0x200006a0                ATT_A_EN_WIFI3_5_8Ghz_Table
                0x200006e0                ATT_A_EN_30G3_28_28_5Ghz_Table
                0x20000720                ATT_A_EN_WIFI4_5_8Ghz_Table
                0x20000760                Atten_Setting
                0x20000791                ATT_A_EN_150M_Table
                0x200007d1                ATT_B_EN_WIFI3_2_4Ghz_Table
                0x20000811                ATT_A_EN_30G2_29_5_30Ghz_Table
                0x20000851                ATT_A_EN_30G1_29_5_30Ghz_Table
                0x20000891                ATT_B_EN_30G3_29_5_30Ghz_Table
                0x200008d1                ATT_A_EN_30G1_28_5_29Ghz_Table
                0x20000911                ATT_B_EN_30G1_29_5_30Ghz_Table
                0x20000951                ATT_B_EN_150M_Table
                0x20000991                ATT_B_EN_30G3_28_28_5Ghz_Table
                0x200009d1                ATT_A_EN_WIFI1_5_8Ghz_Table
                0x20000a11                ATT_B_EN_WIFI1_5_8Ghz_Table
                0x20000a51                ATT_B_EN_30G2_29_5_30Ghz_Table
                0x20000a91                ATT_A_EN_30G2_28_28_5Ghz_Table
                0x20000ad1                ATT_A_EN_WIFI2_2_4Ghz_Table
                0x20000b11                ATT_A_EN_30G1_29_29_5Ghz_Table
                0x20000b51                ATT_A_EN_WIFI2_5_8Ghz_Table
 *fill*         0x20000b91        0x3 
 COMMON         0x20000b94      0x120 Src\main.o
                0x20000b94                hi2c3
                0x20000be8                UartDataisReved
                0x20000be9                rx2_data
                0x20000beb                count_out
                0x20000bec                count_in
                0x20000bf0                huart1
                0x20000c30                ring_buf
                0x20000c70                htim6
                0x20000cb0                Timer10ms
 COMMON         0x20000cb4        0x4 c:/program files (x86)/atollic/truestudio for stm32 9.2.0/armtools/bin/../lib/gcc/arm-atollic-eabi/6.3.1/../../../../arm-atollic-eabi/lib/armv7-m\libc_nano.a(lib_a-reent.o)
                0x20000cb4                errno
                0x20000cb8                . = ALIGN (0x4)
                0x20000cb8                _ebss = .
                0x20000cb8                __bss_end__ = _ebss

._user_heap_stack
                0x20000cb8      0x600 load address 0x080063c0
                0x20000cb8                . = ALIGN (0x4)
                0x20000cb8                PROVIDE (end, .)
                [!provide]                PROVIDE (_end, .)
                0x20000eb8                . = (. + _Min_Heap_Size)
 *fill*         0x20000cb8      0x200 
                0x200012b8                . = (. + _Min_Stack_Size)
 *fill*         0x20000eb8      0x400 
                0x200012b8                . = ALIGN (0x4)

/DISCARD/
 libc.a(*)
 libm.a(*)
 libgcc.a(*)

.ARM.attributes
                0x00000000       0x29
 *(.ARM.attributes)
 .ARM.attributes
                0x00000000       0x1d c:/program files (x86)/atollic/truestudio for stm32 9.2.0/armtools/bin/../lib/gcc/arm-atollic-eabi/6.3.1/armv7-m/crti.o
 .ARM.attributes
                0x0000001d       0x2d c:/program files (x86)/atollic/truestudio for stm32 9.2.0/armtools/bin/../lib/gcc/arm-atollic-eabi/6.3.1/armv7-m/crtbegin.o
 .ARM.attributes
                0x0000004a       0x33 Drivers\STM32F2xx_HAL_Driver\Src\stm32f2xx_hal.o
 .ARM.attributes
                0x0000007d       0x33 Drivers\STM32F2xx_HAL_Driver\Src\stm32f2xx_hal_cortex.o
 .ARM.attributes
                0x000000b0       0x33 Drivers\STM32F2xx_HAL_Driver\Src\stm32f2xx_hal_dma.o
 .ARM.attributes
                0x000000e3       0x33 Drivers\STM32F2xx_HAL_Driver\Src\stm32f2xx_hal_gpio.o
 .ARM.attributes
                0x00000116       0x33 Drivers\STM32F2xx_HAL_Driver\Src\stm32f2xx_hal_i2c.o
 .ARM.attributes
                0x00000149       0x33 Drivers\STM32F2xx_HAL_Driver\Src\stm32f2xx_hal_rcc.o
 .ARM.attributes
                0x0000017c       0x33 Drivers\STM32F2xx_HAL_Driver\Src\stm32f2xx_hal_tim.o
 .ARM.attributes
                0x000001af       0x33 Drivers\STM32F2xx_HAL_Driver\Src\stm32f2xx_hal_tim_ex.o
 .ARM.attributes
                0x000001e2       0x33 Drivers\STM32F2xx_HAL_Driver\Src\stm32f2xx_hal_uart.o
 .ARM.attributes
                0x00000215       0x33 Src\atten_ctrl.o
 .ARM.attributes
                0x00000248       0x33 Src\eeprom.o
 .ARM.attributes
                0x0000027b       0x33 Src\main.o
 .ARM.attributes
                0x000002ae       0x33 Src\sth30_crc.o
 .ARM.attributes
                0x000002e1       0x33 Src\stm32f2xx_hal_msp.o
 .ARM.attributes
                0x00000314       0x33 Src\stm32f2xx_it.o
 .ARM.attributes
                0x00000347       0x33 Src\system_stm32f2xx.o
 .ARM.attributes
                0x0000037a       0x21 startup\startup_stm32f207xx.o
 .ARM.attributes
                0x0000039b       0x2d c:/program files (x86)/atollic/truestudio for stm32 9.2.0/armtools/bin/../lib/gcc/arm-atollic-eabi/6.3.1/../../../../arm-atollic-eabi/lib/armv7-m\libc_nano.a(lib_a-impure.o)
 .ARM.attributes
                0x000003c8       0x2d c:/program files (x86)/atollic/truestudio for stm32 9.2.0/armtools/bin/../lib/gcc/arm-atollic-eabi/6.3.1/../../../../arm-atollic-eabi/lib/armv7-m\libc_nano.a(lib_a-init.o)
 .ARM.attributes
                0x000003f5       0x2d c:/program files (x86)/atollic/truestudio for stm32 9.2.0/armtools/bin/../lib/gcc/arm-atollic-eabi/6.3.1/../../../../arm-atollic-eabi/lib/armv7-m\libc_nano.a(lib_a-memset.o)
 .ARM.attributes
                0x00000422       0x2d c:/program files (x86)/atollic/truestudio for stm32 9.2.0/armtools/bin/../lib/gcc/arm-atollic-eabi/6.3.1/../../../../arm-atollic-eabi/lib/armv7-m\libc_nano.a(lib_a-printf.o)
 .ARM.attributes
                0x0000044f       0x2d c:/program files (x86)/atollic/truestudio for stm32 9.2.0/armtools/bin/../lib/gcc/arm-atollic-eabi/6.3.1/../../../../arm-atollic-eabi/lib/armv7-m\libc_nano.a(lib_a-puts.o)
 .ARM.attributes
                0x0000047c       0x2d c:/program files (x86)/atollic/truestudio for stm32 9.2.0/armtools/bin/../lib/gcc/arm-atollic-eabi/6.3.1/../../../../arm-atollic-eabi/lib/armv7-m\libc_nano.a(lib_a-setbuf.o)
 .ARM.attributes
                0x000004a9       0x2d c:/program files (x86)/atollic/truestudio for stm32 9.2.0/armtools/bin/../lib/gcc/arm-atollic-eabi/6.3.1/../../../../arm-atollic-eabi/lib/armv7-m\libc_nano.a(lib_a-setvbuf.o)
 .ARM.attributes
                0x000004d6       0x2d c:/program files (x86)/atollic/truestudio for stm32 9.2.0/armtools/bin/../lib/gcc/arm-atollic-eabi/6.3.1/../../../../arm-atollic-eabi/lib/armv7-m\libc_nano.a(lib_a-wbuf.o)
 .ARM.attributes
                0x00000503       0x2d c:/program files (x86)/atollic/truestudio for stm32 9.2.0/armtools/bin/../lib/gcc/arm-atollic-eabi/6.3.1/../../../../arm-atollic-eabi/lib/armv7-m\libc_nano.a(lib_a-wsetup.o)
 .ARM.attributes
                0x00000530       0x2d c:/program files (x86)/atollic/truestudio for stm32 9.2.0/armtools/bin/../lib/gcc/arm-atollic-eabi/6.3.1/../../../../arm-atollic-eabi/lib/armv7-m\libc_nano.a(lib_a-fflush.o)
 .ARM.attributes
                0x0000055d       0x2d c:/program files (x86)/atollic/truestudio for stm32 9.2.0/armtools/bin/../lib/gcc/arm-atollic-eabi/6.3.1/../../../../arm-atollic-eabi/lib/armv7-m\libc_nano.a(lib_a-findfp.o)
 .ARM.attributes
                0x0000058a       0x2d c:/program files (x86)/atollic/truestudio for stm32 9.2.0/armtools/bin/../lib/gcc/arm-atollic-eabi/6.3.1/../../../../arm-atollic-eabi/lib/armv7-m\libc_nano.a(lib_a-fwalk.o)
 .ARM.attributes
                0x000005b7       0x2d c:/program files (x86)/atollic/truestudio for stm32 9.2.0/armtools/bin/../lib/gcc/arm-atollic-eabi/6.3.1/../../../../arm-atollic-eabi/lib/armv7-m\libc_nano.a(lib_a-makebuf.o)
 .ARM.attributes
                0x000005e4       0x2d c:/program files (x86)/atollic/truestudio for stm32 9.2.0/armtools/bin/../lib/gcc/arm-atollic-eabi/6.3.1/../../../../arm-atollic-eabi/lib/armv7-m\libc_nano.a(lib_a-malloc.o)
 .ARM.attributes
                0x00000611       0x2d c:/program files (x86)/atollic/truestudio for stm32 9.2.0/armtools/bin/../lib/gcc/arm-atollic-eabi/6.3.1/../../../../arm-atollic-eabi/lib/armv7-m\libc_nano.a(lib_a-nano-freer.o)
 .ARM.attributes
                0x0000063e       0x2d c:/program files (x86)/atollic/truestudio for stm32 9.2.0/armtools/bin/../lib/gcc/arm-atollic-eabi/6.3.1/../../../../arm-atollic-eabi/lib/armv7-m\libc_nano.a(lib_a-nano-mallocr.o)
 .ARM.attributes
                0x0000066b       0x2d c:/program files (x86)/atollic/truestudio for stm32 9.2.0/armtools/bin/../lib/gcc/arm-atollic-eabi/6.3.1/../../../../arm-atollic-eabi/lib/armv7-m\libc_nano.a(lib_a-nano-vfprintf.o)
 .ARM.attributes
                0x00000698       0x2d c:/program files (x86)/atollic/truestudio for stm32 9.2.0/armtools/bin/../lib/gcc/arm-atollic-eabi/6.3.1/../../../../arm-atollic-eabi/lib/armv7-m\libc_nano.a(lib_a-nano-vfprintf_i.o)
 .ARM.attributes
                0x000006c5       0x2d c:/program files (x86)/atollic/truestudio for stm32 9.2.0/armtools/bin/../lib/gcc/arm-atollic-eabi/6.3.1/../../../../arm-atollic-eabi/lib/armv7-m\libc_nano.a(lib_a-sbrkr.o)
 .ARM.attributes
                0x000006f2       0x2d c:/program files (x86)/atollic/truestudio for stm32 9.2.0/armtools/bin/../lib/gcc/arm-atollic-eabi/6.3.1/../../../../arm-atollic-eabi/lib/armv7-m\libc_nano.a(lib_a-stdio.o)
 .ARM.attributes
                0x0000071f       0x2d c:/program files (x86)/atollic/truestudio for stm32 9.2.0/armtools/bin/../lib/gcc/arm-atollic-eabi/6.3.1/../../../../arm-atollic-eabi/lib/armv7-m\libc_nano.a(lib_a-writer.o)
 .ARM.attributes
                0x0000074c       0x2d c:/program files (x86)/atollic/truestudio for stm32 9.2.0/armtools/bin/../lib/gcc/arm-atollic-eabi/6.3.1/../../../../arm-atollic-eabi/lib/armv7-m\libc_nano.a(lib_a-closer.o)
 .ARM.attributes
                0x00000779       0x2d c:/program files (x86)/atollic/truestudio for stm32 9.2.0/armtools/bin/../lib/gcc/arm-atollic-eabi/6.3.1/../../../../arm-atollic-eabi/lib/armv7-m\libc_nano.a(lib_a-fstatr.o)
 .ARM.attributes
                0x000007a6       0x2d c:/program files (x86)/atollic/truestudio for stm32 9.2.0/armtools/bin/../lib/gcc/arm-atollic-eabi/6.3.1/../../../../arm-atollic-eabi/lib/armv7-m\libc_nano.a(lib_a-isattyr.o)
 .ARM.attributes
                0x000007d3       0x2d c:/program files (x86)/atollic/truestudio for stm32 9.2.0/armtools/bin/../lib/gcc/arm-atollic-eabi/6.3.1/../../../../arm-atollic-eabi/lib/armv7-m\libc_nano.a(lib_a-lseekr.o)
 .ARM.attributes
                0x00000800       0x2d c:/program files (x86)/atollic/truestudio for stm32 9.2.0/armtools/bin/../lib/gcc/arm-atollic-eabi/6.3.1/../../../../arm-atollic-eabi/lib/armv7-m\libc_nano.a(lib_a-memchr-stub.o)
 .ARM.attributes
                0x0000082d       0x2d c:/program files (x86)/atollic/truestudio for stm32 9.2.0/armtools/bin/../lib/gcc/arm-atollic-eabi/6.3.1/../../../../arm-atollic-eabi/lib/armv7-m\libc_nano.a(lib_a-mlock.o)
 .ARM.attributes
                0x0000085a       0x2d c:/program files (x86)/atollic/truestudio for stm32 9.2.0/armtools/bin/../lib/gcc/arm-atollic-eabi/6.3.1/../../../../arm-atollic-eabi/lib/armv7-m\libc_nano.a(lib_a-readr.o)
 .ARM.attributes
                0x00000887       0x2d c:/program files (x86)/atollic/truestudio for stm32 9.2.0/armtools/bin/../lib/gcc/arm-atollic-eabi/6.3.1/../../../../arm-atollic-eabi/lib/armv7-m\libc_nano.a(lib_a-reent.o)
 .ARM.attributes
                0x000008b4       0x1d c:/program files (x86)/atollic/truestudio for stm32 9.2.0/armtools/bin/../lib/gcc/arm-atollic-eabi/6.3.1/armv7-m\libgcc.a(_aeabi_uldivmod.o)
 .ARM.attributes
                0x000008d1       0x2d c:/program files (x86)/atollic/truestudio for stm32 9.2.0/armtools/bin/../lib/gcc/arm-atollic-eabi/6.3.1/armv7-m\libgcc.a(_udivmoddi4.o)
 .ARM.attributes
                0x000008fe       0x1d c:/program files (x86)/atollic/truestudio for stm32 9.2.0/armtools/bin/../lib/gcc/arm-atollic-eabi/6.3.1/armv7-m\libgcc.a(_dvmd_tls.o)
 .ARM.attributes
                0x0000091b       0x2d c:/program files (x86)/atollic/truestudio for stm32 9.2.0/armtools/bin/../lib/gcc/arm-atollic-eabi/6.3.1/../../../../arm-atollic-eabi/lib/armv7-m\libnosys.a(close.o)
 .ARM.attributes
                0x00000948       0x2d c:/program files (x86)/atollic/truestudio for stm32 9.2.0/armtools/bin/../lib/gcc/arm-atollic-eabi/6.3.1/../../../../arm-atollic-eabi/lib/armv7-m\libnosys.a(fstat.o)
 .ARM.attributes
                0x00000975       0x2d c:/program files (x86)/atollic/truestudio for stm32 9.2.0/armtools/bin/../lib/gcc/arm-atollic-eabi/6.3.1/../../../../arm-atollic-eabi/lib/armv7-m\libnosys.a(isatty.o)
 .ARM.attributes
                0x000009a2       0x2d c:/program files (x86)/atollic/truestudio for stm32 9.2.0/armtools/bin/../lib/gcc/arm-atollic-eabi/6.3.1/../../../../arm-atollic-eabi/lib/armv7-m\libnosys.a(lseek.o)
 .ARM.attributes
                0x000009cf       0x2d c:/program files (x86)/atollic/truestudio for stm32 9.2.0/armtools/bin/../lib/gcc/arm-atollic-eabi/6.3.1/../../../../arm-atollic-eabi/lib/armv7-m\libnosys.a(read.o)
 .ARM.attributes
                0x000009fc       0x2d c:/program files (x86)/atollic/truestudio for stm32 9.2.0/armtools/bin/../lib/gcc/arm-atollic-eabi/6.3.1/../../../../arm-atollic-eabi/lib/armv7-m\libnosys.a(sbrk.o)
 .ARM.attributes
                0x00000a29       0x1d c:/program files (x86)/atollic/truestudio for stm32 9.2.0/armtools/bin/../lib/gcc/arm-atollic-eabi/6.3.1/armv7-m/crtn.o
OUTPUT(STM32F207_ChannelCtrl.elf elf32-littlearm)

.debug_info     0x00000000    0x1dc6e
 .debug_info    0x00000000     0x1179 Drivers\STM32F2xx_HAL_Driver\Src\stm32f2xx_hal.o
 .debug_info    0x00001179     0x1742 Drivers\STM32F2xx_HAL_Driver\Src\stm32f2xx_hal_cortex.o
 .debug_info    0x000028bb     0x125c Drivers\STM32F2xx_HAL_Driver\Src\stm32f2xx_hal_dma.o
 .debug_info    0x00003b17      0xf88 Drivers\STM32F2xx_HAL_Driver\Src\stm32f2xx_hal_gpio.o
 .debug_info    0x00004a9f     0x377c Drivers\STM32F2xx_HAL_Driver\Src\stm32f2xx_hal_i2c.o
 .debug_info    0x0000821b     0x14d1 Drivers\STM32F2xx_HAL_Driver\Src\stm32f2xx_hal_rcc.o
 .debug_info    0x000096ec     0x3bae Drivers\STM32F2xx_HAL_Driver\Src\stm32f2xx_hal_tim.o
 .debug_info    0x0000d29a     0x19b1 Drivers\STM32F2xx_HAL_Driver\Src\stm32f2xx_hal_tim_ex.o
 .debug_info    0x0000ec4b     0x1e9f Drivers\STM32F2xx_HAL_Driver\Src\stm32f2xx_hal_uart.o
 .debug_info    0x00010aea     0x33e7 Src\atten_ctrl.o
 .debug_info    0x00013ed1     0x1e9b Src\eeprom.o
 .debug_info    0x00015d6c     0x2a5e Src\main.o
 .debug_info    0x000187ca      0xa0e Src\sth30_crc.o
 .debug_info    0x000191d8     0x21e5 Src\stm32f2xx_hal_msp.o
 .debug_info    0x0001b3bd     0x1b26 Src\stm32f2xx_it.o
 .debug_info    0x0001cee3      0xd1c Src\system_stm32f2xx.o
 .debug_info    0x0001dbff       0x6f startup\startup_stm32f207xx.o

.debug_abbrev   0x00000000     0x3044
 .debug_abbrev  0x00000000      0x324 Drivers\STM32F2xx_HAL_Driver\Src\stm32f2xx_hal.o
 .debug_abbrev  0x00000324      0x3a2 Drivers\STM32F2xx_HAL_Driver\Src\stm32f2xx_hal_cortex.o
 .debug_abbrev  0x000006c6      0x34a Drivers\STM32F2xx_HAL_Driver\Src\stm32f2xx_hal_dma.o
 .debug_abbrev  0x00000a10      0x268 Drivers\STM32F2xx_HAL_Driver\Src\stm32f2xx_hal_gpio.o
 .debug_abbrev  0x00000c78      0x3b4 Drivers\STM32F2xx_HAL_Driver\Src\stm32f2xx_hal_i2c.o
 .debug_abbrev  0x0000102c      0x375 Drivers\STM32F2xx_HAL_Driver\Src\stm32f2xx_hal_rcc.o
 .debug_abbrev  0x000013a1      0x3bd Drivers\STM32F2xx_HAL_Driver\Src\stm32f2xx_hal_tim.o
 .debug_abbrev  0x0000175e      0x300 Drivers\STM32F2xx_HAL_Driver\Src\stm32f2xx_hal_tim_ex.o
 .debug_abbrev  0x00001a5e      0x3a0 Drivers\STM32F2xx_HAL_Driver\Src\stm32f2xx_hal_uart.o
 .debug_abbrev  0x00001dfe      0x3b5 Src\atten_ctrl.o
 .debug_abbrev  0x000021b3      0x22d Src\eeprom.o
 .debug_abbrev  0x000023e0      0x3d6 Src\main.o
 .debug_abbrev  0x000027b6      0x201 Src\sth30_crc.o
 .debug_abbrev  0x000029b7      0x28b Src\stm32f2xx_hal_msp.o
 .debug_abbrev  0x00002c42      0x226 Src\stm32f2xx_it.o
 .debug_abbrev  0x00002e68      0x1ca Src\system_stm32f2xx.o
 .debug_abbrev  0x00003032       0x12 startup\startup_stm32f207xx.o

.debug_loc      0x00000000     0xb8f0
 .debug_loc     0x00000000       0x91 Drivers\STM32F2xx_HAL_Driver\Src\stm32f2xx_hal.o
 .debug_loc     0x00000091      0x48c Drivers\STM32F2xx_HAL_Driver\Src\stm32f2xx_hal_cortex.o
 .debug_loc     0x0000051d      0x735 Drivers\STM32F2xx_HAL_Driver\Src\stm32f2xx_hal_dma.o
 .debug_loc     0x00000c52      0x3cd Drivers\STM32F2xx_HAL_Driver\Src\stm32f2xx_hal_gpio.o
 .debug_loc     0x0000101f     0x2bba Drivers\STM32F2xx_HAL_Driver\Src\stm32f2xx_hal_i2c.o
 .debug_loc     0x00003bd9      0x4b0 Drivers\STM32F2xx_HAL_Driver\Src\stm32f2xx_hal_rcc.o
 .debug_loc     0x00004089     0x30d0 Drivers\STM32F2xx_HAL_Driver\Src\stm32f2xx_hal_tim.o
 .debug_loc     0x00007159      0x84a Drivers\STM32F2xx_HAL_Driver\Src\stm32f2xx_hal_tim_ex.o
 .debug_loc     0x000079a3     0x1338 Drivers\STM32F2xx_HAL_Driver\Src\stm32f2xx_hal_uart.o
 .debug_loc     0x00008cdb     0x2558 Src\atten_ctrl.o
 .debug_loc     0x0000b233      0x15e Src\eeprom.o
 .debug_loc     0x0000b391      0x145 Src\main.o
 .debug_loc     0x0000b4d6      0x222 Src\sth30_crc.o
 .debug_loc     0x0000b6f8       0xdc Src\stm32f2xx_hal_msp.o
 .debug_loc     0x0000b7d4      0x11c Src\system_stm32f2xx.o

.debug_aranges  0x00000000      0xb38
 .debug_aranges
                0x00000000       0xc0 Drivers\STM32F2xx_HAL_Driver\Src\stm32f2xx_hal.o
 .debug_aranges
                0x000000c0       0xa8 Drivers\STM32F2xx_HAL_Driver\Src\stm32f2xx_hal_cortex.o
 .debug_aranges
                0x00000168       0x80 Drivers\STM32F2xx_HAL_Driver\Src\stm32f2xx_hal_dma.o
 .debug_aranges
                0x000001e8       0x58 Drivers\STM32F2xx_HAL_Driver\Src\stm32f2xx_hal_gpio.o
 .debug_aranges
                0x00000240      0x190 Drivers\STM32F2xx_HAL_Driver\Src\stm32f2xx_hal_i2c.o
 .debug_aranges
                0x000003d0       0x88 Drivers\STM32F2xx_HAL_Driver\Src\stm32f2xx_hal_rcc.o
 .debug_aranges
                0x00000458      0x250 Drivers\STM32F2xx_HAL_Driver\Src\stm32f2xx_hal_tim.o
 .debug_aranges
                0x000006a8       0xf0 Drivers\STM32F2xx_HAL_Driver\Src\stm32f2xx_hal_tim_ex.o
 .debug_aranges
                0x00000798      0x170 Drivers\STM32F2xx_HAL_Driver\Src\stm32f2xx_hal_uart.o
 .debug_aranges
                0x00000908       0x80 Src\atten_ctrl.o
 .debug_aranges
                0x00000988       0x30 Src\eeprom.o
 .debug_aranges
                0x000009b8       0x58 Src\main.o
 .debug_aranges
                0x00000a10       0x30 Src\sth30_crc.o
 .debug_aranges
                0x00000a40       0x50 Src\stm32f2xx_hal_msp.o
 .debug_aranges
                0x00000a90       0x58 Src\stm32f2xx_it.o
 .debug_aranges
                0x00000ae8       0x28 Src\system_stm32f2xx.o
 .debug_aranges
                0x00000b10       0x28 startup\startup_stm32f207xx.o

.debug_ranges   0x00000000     0x1168
 .debug_ranges  0x00000000       0xb0 Drivers\STM32F2xx_HAL_Driver\Src\stm32f2xx_hal.o
 .debug_ranges  0x000000b0      0x140 Drivers\STM32F2xx_HAL_Driver\Src\stm32f2xx_hal_cortex.o
 .debug_ranges  0x000001f0       0xd8 Drivers\STM32F2xx_HAL_Driver\Src\stm32f2xx_hal_dma.o
 .debug_ranges  0x000002c8       0x78 Drivers\STM32F2xx_HAL_Driver\Src\stm32f2xx_hal_gpio.o
 .debug_ranges  0x00000340      0x3f0 Drivers\STM32F2xx_HAL_Driver\Src\stm32f2xx_hal_i2c.o
 .debug_ranges  0x00000730      0x178 Drivers\STM32F2xx_HAL_Driver\Src\stm32f2xx_hal_rcc.o
 .debug_ranges  0x000008a8      0x340 Drivers\STM32F2xx_HAL_Driver\Src\stm32f2xx_hal_tim.o
 .debug_ranges  0x00000be8       0xe0 Drivers\STM32F2xx_HAL_Driver\Src\stm32f2xx_hal_tim_ex.o
 .debug_ranges  0x00000cc8      0x190 Drivers\STM32F2xx_HAL_Driver\Src\stm32f2xx_hal_uart.o
 .debug_ranges  0x00000e58       0x70 Src\atten_ctrl.o
 .debug_ranges  0x00000ec8       0x20 Src\eeprom.o
 .debug_ranges  0x00000ee8      0x118 Src\main.o
 .debug_ranges  0x00001000       0x20 Src\sth30_crc.o
 .debug_ranges  0x00001020       0xc8 Src\stm32f2xx_hal_msp.o
 .debug_ranges  0x000010e8       0x48 Src\stm32f2xx_it.o
 .debug_ranges  0x00001130       0x18 Src\system_stm32f2xx.o
 .debug_ranges  0x00001148       0x20 startup\startup_stm32f207xx.o

.debug_line     0x00000000     0x7811
 .debug_line    0x00000000      0x462 Drivers\STM32F2xx_HAL_Driver\Src\stm32f2xx_hal.o
 .debug_line    0x00000462      0x4e8 Drivers\STM32F2xx_HAL_Driver\Src\stm32f2xx_hal_cortex.o
 .debug_line    0x0000094a      0x617 Drivers\STM32F2xx_HAL_Driver\Src\stm32f2xx_hal_dma.o
 .debug_line    0x00000f61      0x495 Drivers\STM32F2xx_HAL_Driver\Src\stm32f2xx_hal_gpio.o
 .debug_line    0x000013f6     0x1a16 Drivers\STM32F2xx_HAL_Driver\Src\stm32f2xx_hal_i2c.o
 .debug_line    0x00002e0c      0x64a Drivers\STM32F2xx_HAL_Driver\Src\stm32f2xx_hal_rcc.o
 .debug_line    0x00003456     0x121f Drivers\STM32F2xx_HAL_Driver\Src\stm32f2xx_hal_tim.o
 .debug_line    0x00004675      0x704 Drivers\STM32F2xx_HAL_Driver\Src\stm32f2xx_hal_tim_ex.o
 .debug_line    0x00004d79      0xc6a Drivers\STM32F2xx_HAL_Driver\Src\stm32f2xx_hal_uart.o
 .debug_line    0x000059e3      0x8de Src\atten_ctrl.o
 .debug_line    0x000062c1      0x338 Src\eeprom.o
 .debug_line    0x000065f9      0x564 Src\main.o
 .debug_line    0x00006b5d      0x241 Src\sth30_crc.o
 .debug_line    0x00006d9e      0x3fd Src\stm32f2xx_hal_msp.o
 .debug_line    0x0000719b      0x37c Src\stm32f2xx_it.o
 .debug_line    0x00007517      0x27b Src\system_stm32f2xx.o
 .debug_line    0x00007792       0x7f startup\startup_stm32f207xx.o

.debug_str      0x00000000     0x718a
 .debug_str     0x00000000      0xe2f Drivers\STM32F2xx_HAL_Driver\Src\stm32f2xx_hal.o
                                0xef0 (size before relaxing)
 .debug_str     0x00000e2f      0x3ca Drivers\STM32F2xx_HAL_Driver\Src\stm32f2xx_hal_cortex.o
                               0x1070 (size before relaxing)
 .debug_str     0x000011f9      0x522 Drivers\STM32F2xx_HAL_Driver\Src\stm32f2xx_hal_dma.o
                                0xbc1 (size before relaxing)
 .debug_str     0x0000171b      0x1d3 Drivers\STM32F2xx_HAL_Driver\Src\stm32f2xx_hal_gpio.o
                                0x93b (size before relaxing)
 .debug_str     0x000018ee      0xa6d Drivers\STM32F2xx_HAL_Driver\Src\stm32f2xx_hal_i2c.o
                               0x1392 (size before relaxing)
 .debug_str     0x0000235b      0x2bb Drivers\STM32F2xx_HAL_Driver\Src\stm32f2xx_hal_rcc.o
                                0xb02 (size before relaxing)
 .debug_str     0x00002616      0xf03 Drivers\STM32F2xx_HAL_Driver\Src\stm32f2xx_hal_tim.o
                               0x1812 (size before relaxing)
 .debug_str     0x00003519      0x50d Drivers\STM32F2xx_HAL_Driver\Src\stm32f2xx_hal_tim_ex.o
                               0x10d2 (size before relaxing)
 .debug_str     0x00003a26      0x6c3 Drivers\STM32F2xx_HAL_Driver\Src\stm32f2xx_hal_uart.o
                               0x1047 (size before relaxing)
 .debug_str     0x000040e9     0x2d85 Src\atten_ctrl.o
                               0x3a93 (size before relaxing)
 .debug_str     0x00006e6e       0x42 Src\eeprom.o
                               0x1d85 (size before relaxing)
 .debug_str     0x00006eb0      0x152 Src\main.o
                               0x29c5 (size before relaxing)
 .debug_str     0x00007002       0x52 Src\sth30_crc.o
                                0x630 (size before relaxing)
 .debug_str     0x00007054       0x25 Src\stm32f2xx_hal_msp.o
                               0x25d3 (size before relaxing)
 .debug_str     0x00007079       0xcc Src\stm32f2xx_it.o
                               0x1fa0 (size before relaxing)
 .debug_str     0x00007145       0x45 Src\system_stm32f2xx.o
                                0x79f (size before relaxing)

.comment        0x00000000       0x7c
 .comment       0x00000000       0x7c Drivers\STM32F2xx_HAL_Driver\Src\stm32f2xx_hal.o
                                 0x7d (size before relaxing)
 .comment       0x0000007c       0x7d Drivers\STM32F2xx_HAL_Driver\Src\stm32f2xx_hal_cortex.o
 .comment       0x0000007c       0x7d Drivers\STM32F2xx_HAL_Driver\Src\stm32f2xx_hal_dma.o
 .comment       0x0000007c       0x7d Drivers\STM32F2xx_HAL_Driver\Src\stm32f2xx_hal_gpio.o
 .comment       0x0000007c       0x7d Drivers\STM32F2xx_HAL_Driver\Src\stm32f2xx_hal_i2c.o
 .comment       0x0000007c       0x7d Drivers\STM32F2xx_HAL_Driver\Src\stm32f2xx_hal_rcc.o
 .comment       0x0000007c       0x7d Drivers\STM32F2xx_HAL_Driver\Src\stm32f2xx_hal_tim.o
 .comment       0x0000007c       0x7d Drivers\STM32F2xx_HAL_Driver\Src\stm32f2xx_hal_tim_ex.o
 .comment       0x0000007c       0x7d Drivers\STM32F2xx_HAL_Driver\Src\stm32f2xx_hal_uart.o
 .comment       0x0000007c       0x7d Src\atten_ctrl.o
 .comment       0x0000007c       0x7d Src\eeprom.o
 .comment       0x0000007c       0x7d Src\main.o
 .comment       0x0000007c       0x7d Src\sth30_crc.o
 .comment       0x0000007c       0x7d Src\stm32f2xx_hal_msp.o
 .comment       0x0000007c       0x7d Src\stm32f2xx_it.o
 .comment       0x0000007c       0x7d Src\system_stm32f2xx.o

.debug_frame    0x00000000     0x2bc0
 .debug_frame   0x00000000      0x194 Drivers\STM32F2xx_HAL_Driver\Src\stm32f2xx_hal.o
 .debug_frame   0x00000194      0x158 Drivers\STM32F2xx_HAL_Driver\Src\stm32f2xx_hal_cortex.o
 .debug_frame   0x000002ec      0x150 Drivers\STM32F2xx_HAL_Driver\Src\stm32f2xx_hal_dma.o
 .debug_frame   0x0000043c       0xd8 Drivers\STM32F2xx_HAL_Driver\Src\stm32f2xx_hal_gpio.o
 .debug_frame   0x00000514      0x684 Drivers\STM32F2xx_HAL_Driver\Src\stm32f2xx_hal_i2c.o
 .debug_frame   0x00000b98      0x14c Drivers\STM32F2xx_HAL_Driver\Src\stm32f2xx_hal_rcc.o
 .debug_frame   0x00000ce4      0x854 Drivers\STM32F2xx_HAL_Driver\Src\stm32f2xx_hal_tim.o
 .debug_frame   0x00001538      0x330 Drivers\STM32F2xx_HAL_Driver\Src\stm32f2xx_hal_tim_ex.o
 .debug_frame   0x00001868      0x4a0 Drivers\STM32F2xx_HAL_Driver\Src\stm32f2xx_hal_uart.o
 .debug_frame   0x00001d08      0x244 Src\atten_ctrl.o
 .debug_frame   0x00001f4c       0x68 Src\eeprom.o
 .debug_frame   0x00001fb4       0xc0 Src\main.o
 .debug_frame   0x00002074       0x5c Src\sth30_crc.o
 .debug_frame   0x000020d0       0xd8 Src\stm32f2xx_hal_msp.o
 .debug_frame   0x000021a8       0xc0 Src\stm32f2xx_it.o
 .debug_frame   0x00002268       0x38 Src\system_stm32f2xx.o
 .debug_frame   0x000022a0       0x2c c:/program files (x86)/atollic/truestudio for stm32 9.2.0/armtools/bin/../lib/gcc/arm-atollic-eabi/6.3.1/../../../../arm-atollic-eabi/lib/armv7-m\libc_nano.a(lib_a-init.o)
 .debug_frame   0x000022cc       0x20 c:/program files (x86)/atollic/truestudio for stm32 9.2.0/armtools/bin/../lib/gcc/arm-atollic-eabi/6.3.1/../../../../arm-atollic-eabi/lib/armv7-m\libc_nano.a(lib_a-memset.o)
 .debug_frame   0x000022ec       0x74 c:/program files (x86)/atollic/truestudio for stm32 9.2.0/armtools/bin/../lib/gcc/arm-atollic-eabi/6.3.1/../../../../arm-atollic-eabi/lib/armv7-m\libc_nano.a(lib_a-printf.o)
 .debug_frame   0x00002360       0x3c c:/program files (x86)/atollic/truestudio for stm32 9.2.0/armtools/bin/../lib/gcc/arm-atollic-eabi/6.3.1/../../../../arm-atollic-eabi/lib/armv7-m\libc_nano.a(lib_a-puts.o)
 .debug_frame   0x0000239c       0x20 c:/program files (x86)/atollic/truestudio for stm32 9.2.0/armtools/bin/../lib/gcc/arm-atollic-eabi/6.3.1/../../../../arm-atollic-eabi/lib/armv7-m\libc_nano.a(lib_a-setbuf.o)
 .debug_frame   0x000023bc       0x38 c:/program files (x86)/atollic/truestudio for stm32 9.2.0/armtools/bin/../lib/gcc/arm-atollic-eabi/6.3.1/../../../../arm-atollic-eabi/lib/armv7-m\libc_nano.a(lib_a-setvbuf.o)
 .debug_frame   0x000023f4       0x40 c:/program files (x86)/atollic/truestudio for stm32 9.2.0/armtools/bin/../lib/gcc/arm-atollic-eabi/6.3.1/../../../../arm-atollic-eabi/lib/armv7-m\libc_nano.a(lib_a-wbuf.o)
 .debug_frame   0x00002434       0x2c c:/program files (x86)/atollic/truestudio for stm32 9.2.0/armtools/bin/../lib/gcc/arm-atollic-eabi/6.3.1/../../../../arm-atollic-eabi/lib/armv7-m\libc_nano.a(lib_a-wsetup.o)
 .debug_frame   0x00002460       0x68 c:/program files (x86)/atollic/truestudio for stm32 9.2.0/armtools/bin/../lib/gcc/arm-atollic-eabi/6.3.1/../../../../arm-atollic-eabi/lib/armv7-m\libc_nano.a(lib_a-fflush.o)
 .debug_frame   0x000024c8      0x11c c:/program files (x86)/atollic/truestudio for stm32 9.2.0/armtools/bin/../lib/gcc/arm-atollic-eabi/6.3.1/../../../../arm-atollic-eabi/lib/armv7-m\libc_nano.a(lib_a-findfp.o)
 .debug_frame   0x000025e4       0x54 c:/program files (x86)/atollic/truestudio for stm32 9.2.0/armtools/bin/../lib/gcc/arm-atollic-eabi/6.3.1/../../../../arm-atollic-eabi/lib/armv7-m\libc_nano.a(lib_a-fwalk.o)
 .debug_frame   0x00002638       0x58 c:/program files (x86)/atollic/truestudio for stm32 9.2.0/armtools/bin/../lib/gcc/arm-atollic-eabi/6.3.1/../../../../arm-atollic-eabi/lib/armv7-m\libc_nano.a(lib_a-makebuf.o)
 .debug_frame   0x00002690       0x30 c:/program files (x86)/atollic/truestudio for stm32 9.2.0/armtools/bin/../lib/gcc/arm-atollic-eabi/6.3.1/../../../../arm-atollic-eabi/lib/armv7-m\libc_nano.a(lib_a-malloc.o)
 .debug_frame   0x000026c0       0x38 c:/program files (x86)/atollic/truestudio for stm32 9.2.0/armtools/bin/../lib/gcc/arm-atollic-eabi/6.3.1/../../../../arm-atollic-eabi/lib/armv7-m\libc_nano.a(lib_a-nano-freer.o)
 .debug_frame   0x000026f8       0x2c c:/program files (x86)/atollic/truestudio for stm32 9.2.0/armtools/bin/../lib/gcc/arm-atollic-eabi/6.3.1/../../../../arm-atollic-eabi/lib/armv7-m\libc_nano.a(lib_a-nano-mallocr.o)
 .debug_frame   0x00002724       0xac c:/program files (x86)/atollic/truestudio for stm32 9.2.0/armtools/bin/../lib/gcc/arm-atollic-eabi/6.3.1/../../../../arm-atollic-eabi/lib/armv7-m\libc_nano.a(lib_a-nano-vfprintf.o)
 .debug_frame   0x000027d0       0x60 c:/program files (x86)/atollic/truestudio for stm32 9.2.0/armtools/bin/../lib/gcc/arm-atollic-eabi/6.3.1/../../../../arm-atollic-eabi/lib/armv7-m\libc_nano.a(lib_a-nano-vfprintf_i.o)
 .debug_frame   0x00002830       0x2c c:/program files (x86)/atollic/truestudio for stm32 9.2.0/armtools/bin/../lib/gcc/arm-atollic-eabi/6.3.1/../../../../arm-atollic-eabi/lib/armv7-m\libc_nano.a(lib_a-sbrkr.o)
 .debug_frame   0x0000285c       0x88 c:/program files (x86)/atollic/truestudio for stm32 9.2.0/armtools/bin/../lib/gcc/arm-atollic-eabi/6.3.1/../../../../arm-atollic-eabi/lib/armv7-m\libc_nano.a(lib_a-stdio.o)
 .debug_frame   0x000028e4       0x2c c:/program files (x86)/atollic/truestudio for stm32 9.2.0/armtools/bin/../lib/gcc/arm-atollic-eabi/6.3.1/../../../../arm-atollic-eabi/lib/armv7-m\libc_nano.a(lib_a-writer.o)
 .debug_frame   0x00002910       0x2c c:/program files (x86)/atollic/truestudio for stm32 9.2.0/armtools/bin/../lib/gcc/arm-atollic-eabi/6.3.1/../../../../arm-atollic-eabi/lib/armv7-m\libc_nano.a(lib_a-closer.o)
 .debug_frame   0x0000293c       0x2c c:/program files (x86)/atollic/truestudio for stm32 9.2.0/armtools/bin/../lib/gcc/arm-atollic-eabi/6.3.1/../../../../arm-atollic-eabi/lib/armv7-m\libc_nano.a(lib_a-fstatr.o)
 .debug_frame   0x00002968       0x2c c:/program files (x86)/atollic/truestudio for stm32 9.2.0/armtools/bin/../lib/gcc/arm-atollic-eabi/6.3.1/../../../../arm-atollic-eabi/lib/armv7-m\libc_nano.a(lib_a-isattyr.o)
 .debug_frame   0x00002994       0x2c c:/program files (x86)/atollic/truestudio for stm32 9.2.0/armtools/bin/../lib/gcc/arm-atollic-eabi/6.3.1/../../../../arm-atollic-eabi/lib/armv7-m\libc_nano.a(lib_a-lseekr.o)
 .debug_frame   0x000029c0       0x28 c:/program files (x86)/atollic/truestudio for stm32 9.2.0/armtools/bin/../lib/gcc/arm-atollic-eabi/6.3.1/../../../../arm-atollic-eabi/lib/armv7-m\libc_nano.a(lib_a-memchr-stub.o)
 .debug_frame   0x000029e8       0x30 c:/program files (x86)/atollic/truestudio for stm32 9.2.0/armtools/bin/../lib/gcc/arm-atollic-eabi/6.3.1/../../../../arm-atollic-eabi/lib/armv7-m\libc_nano.a(lib_a-mlock.o)
 .debug_frame   0x00002a18       0x2c c:/program files (x86)/atollic/truestudio for stm32 9.2.0/armtools/bin/../lib/gcc/arm-atollic-eabi/6.3.1/../../../../arm-atollic-eabi/lib/armv7-m\libc_nano.a(lib_a-readr.o)
 .debug_frame   0x00002a44       0x5c c:/program files (x86)/atollic/truestudio for stm32 9.2.0/armtools/bin/../lib/gcc/arm-atollic-eabi/6.3.1/../../../../arm-atollic-eabi/lib/armv7-m\libc_nano.a(lib_a-reent.o)
 .debug_frame   0x00002aa0       0x2c c:/program files (x86)/atollic/truestudio for stm32 9.2.0/armtools/bin/../lib/gcc/arm-atollic-eabi/6.3.1/armv7-m\libgcc.a(_aeabi_uldivmod.o)
 .debug_frame   0x00002acc       0x34 c:/program files (x86)/atollic/truestudio for stm32 9.2.0/armtools/bin/../lib/gcc/arm-atollic-eabi/6.3.1/armv7-m\libgcc.a(_udivmoddi4.o)
 .debug_frame   0x00002b00       0x20 c:/program files (x86)/atollic/truestudio for stm32 9.2.0/armtools/bin/../lib/gcc/arm-atollic-eabi/6.3.1/../../../../arm-atollic-eabi/lib/armv7-m\libnosys.a(close.o)
 .debug_frame   0x00002b20       0x20 c:/program files (x86)/atollic/truestudio for stm32 9.2.0/armtools/bin/../lib/gcc/arm-atollic-eabi/6.3.1/../../../../arm-atollic-eabi/lib/armv7-m\libnosys.a(fstat.o)
 .debug_frame   0x00002b40       0x20 c:/program files (x86)/atollic/truestudio for stm32 9.2.0/armtools/bin/../lib/gcc/arm-atollic-eabi/6.3.1/../../../../arm-atollic-eabi/lib/armv7-m\libnosys.a(isatty.o)
 .debug_frame   0x00002b60       0x20 c:/program files (x86)/atollic/truestudio for stm32 9.2.0/armtools/bin/../lib/gcc/arm-atollic-eabi/6.3.1/../../../../arm-atollic-eabi/lib/armv7-m\libnosys.a(lseek.o)
 .debug_frame   0x00002b80       0x20 c:/program files (x86)/atollic/truestudio for stm32 9.2.0/armtools/bin/../lib/gcc/arm-atollic-eabi/6.3.1/../../../../arm-atollic-eabi/lib/armv7-m\libnosys.a(read.o)
 .debug_frame   0x00002ba0       0x20 c:/program files (x86)/atollic/truestudio for stm32 9.2.0/armtools/bin/../lib/gcc/arm-atollic-eabi/6.3.1/../../../../arm-atollic-eabi/lib/armv7-m\libnosys.a(sbrk.o)

.stab           0x00000000       0x84
 .stab          0x00000000       0x24 c:/program files (x86)/atollic/truestudio for stm32 9.2.0/armtools/bin/../lib/gcc/arm-atollic-eabi/6.3.1/../../../../arm-atollic-eabi/lib/armv7-m\libnosys.a(close.o)
 .stab          0x00000024       0x18 c:/program files (x86)/atollic/truestudio for stm32 9.2.0/armtools/bin/../lib/gcc/arm-atollic-eabi/6.3.1/../../../../arm-atollic-eabi/lib/armv7-m\libnosys.a(fstat.o)
                                 0x24 (size before relaxing)
 .stab          0x0000003c       0x18 c:/program files (x86)/atollic/truestudio for stm32 9.2.0/armtools/bin/../lib/gcc/arm-atollic-eabi/6.3.1/../../../../arm-atollic-eabi/lib/armv7-m\libnosys.a(isatty.o)
                                 0x24 (size before relaxing)
 .stab          0x00000054       0x18 c:/program files (x86)/atollic/truestudio for stm32 9.2.0/armtools/bin/../lib/gcc/arm-atollic-eabi/6.3.1/../../../../arm-atollic-eabi/lib/armv7-m\libnosys.a(lseek.o)
                                 0x24 (size before relaxing)
 .stab          0x0000006c       0x18 c:/program files (x86)/atollic/truestudio for stm32 9.2.0/armtools/bin/../lib/gcc/arm-atollic-eabi/6.3.1/../../../../arm-atollic-eabi/lib/armv7-m\libnosys.a(read.o)
                                 0x24 (size before relaxing)

.stabstr        0x00000000      0x117
 .stabstr       0x00000000      0x117 c:/program files (x86)/atollic/truestudio for stm32 9.2.0/armtools/bin/../lib/gcc/arm-atollic-eabi/6.3.1/../../../../arm-atollic-eabi/lib/armv7-m\libnosys.a(close.o)
